:020000040800F2
:1000000000040020E1010008090E00080D0E0008A0
:10001000610E00080D0E0008350E0008E30100080F
:10002000E3010008E3010008E3010008392F00089C
:10003000E3010008E3010008E3010008E301000810
:10004000E3010008E3010008E3010008E301000800
:10005000E3010008E301000899310008C5310008F8
:10006000F13100081D32000849320008E3010008A0
:10007000E3010008E3010008E3010008E3010008D0
:10008000E3010008E3010008E3010008E3010008C0
:10009000E3010008E3010008E301000875320008ED
:1000A000E3010008E3010008E3010008E3010008A0
:1000B000B52F0008E3010008E3010008E301000890
:1000C000E3010008E3010008E3010008E301000880
:1000D000E3010008E3010008E3010008E301000870
:1000E000DD320008E3010008E3010008E301000835
:1000F000E3010008E3010008E3010008E301000850
:10010000E3010008E3010008E3010008E30100083F
:10011000E3010008E3010008E3010008E30100082F
:10012000E3010008E3010008E3010008E30100081F
:10013000E3010008E3010008E3010008E30100080F
:10014000E3010008E3010008E30100088D26000830
:10015000E3010008E3010008E3010008E3010008EF
:10016000E3010008E3010008E3010008E3010008DF
:10017000E3010008E3010008E3010008E3010008CF
:10018000E3010008E3010008E3010008E3010008BF
:10019000E3010008E3010008E3010008E3010008AF
:1001A000E3010008E3010008E3010008E30100089F
:1001B000E3010008E3010008E3010008E30100088F
:1001C000E3010008E3010008E3010008E30100087F
:1001D000E3010008E3010008E3010008E30100086F
:1001E00002E000F000F8FEE772B6394880F30888B4
:1001F000384880F3098838484EF60851CEF200019D
:10020000086040F20000CCF200004EF63471CEF2ED
:1002100000010860BFF34F8FBFF36F8F40F2000003
:10022000C0F2F0004EF68851CEF200010860BFF334
:100230004F8FBFF36F8F4FF00000E1EE100A4EF6C4
:100240003C71CEF200010860062080F31488BFF3F1
:100250006F8F01F0E3FE02F005FE4FF055301F49AD
:100260001B4A91423CBF41F8040BFAE71C49194A6A
:1002700091423CBF41F8040BFAE71A491A4A1B4B5A
:100280009A423EBF51F8040B42F8040BF8E70020F5
:100290001749184A91423CBF41F8040BFAE701F0B4
:1002A000C1FE02F03BFE144C144DAC4203DA54F88C
:1002B000041B8847F9E700F03FF8114C114DAC42A0
:1002C00003DA54F8041B8847F9E701F0A9BE0000DF
:1002D000000400200024002000000008000000208E
:1002E00000040020F036000800240020282400200C
:1002F0002824002018300020E0010008E001000858
:10030000E0010008E00100082DE9F04F2DED108A12
:10031000C1F80CD0C3689D46BDEC108ABDE8F08FD3
:10032000002383F311882846A047002001F0FAFA41
:1003300001F0AAFA00DFFEE71A4B6FF0790270B500
:1003400000241A700F225C709C70DC701C715C7150
:100350009C71DC711C725C729A72DC7201F030FE6E
:10036000064601F055FE054650B90F4B9E4217D088
:1003700001339E4241F2883412BF05460024012514
:10038000002001F027FE0DB100F0B4F800F010FDE0
:1003900000F0F4FB204600F00BF900F0ABF8F9E7B1
:1003A0000446EDE728240020010007B008B500F05E
:1003B00087FBA0F120035842584108BD07B5054B03
:1003C00002211B88ADF8043001A800F0C7FB03B080
:1003D0005DF804FBC0330008064991F8243033B1BE
:1003E00000230822086A81F8243000F0E9BB0120CC
:1003F000704700BF482400202DE9F84F234C94F8A3
:1004000024300546884617468BBB2E46DFF87C9085
:10041000002F38D094F824A0BAF1000F05D1202283
:10042000FF214846266200F0B1FCCAF10805BD4232
:1004300028BF3D465FFA85FBAD0041462A4604EBE6
:100440008A0000F079FC94F82430A7EB0B079B445A
:100450005FFA8BFBBBF1080F2E44A844FFB284F86F
:1004600024B0D5D1FFF7B8FF0028D1D108E0266A23
:1004700006EB8306B042C9D0FFF7AEFF0028C4D117
:100480000020BDE8F88F0120BDE8F88F4824002047
:1004900010B5202383F311881248C3680BB101F013
:1004A000C7FA0023104A0F484FF47A7101F084FA1A
:1004B000002383F311880D4C236813B12368013B9B
:1004C0002360636813B16368013B6360084B1B786A
:1004D00033B9636823B9022000F024FC322363603F
:1004E00010BD00BF342400209104000878250020AE
:1004F0007024002010B5254B254953F8042F0132F4
:1005000000D110BD8B42F8D1224C234B22689A4275
:100510003AD9224B9B6803F1006303F580339A427A
:1005200032D2002000F044FB1D4B0220187000F076
:10053000F1FB1C4B1A6C00221A64196E1A66196EB4
:10054000596C5A64596E5A665A6E5A6942F0800262
:100550005A615A6922F080025A615A691A6942F056
:1005600000521A611A6922F000521A611B6972B6B0
:100570000D4A0E4B13601B682268202181F31188FD
:100580009D4683F30888104710BD00BFFCFF00089C
:100590001C00010804000108FFFF000828240020B7
:1005A000702400200038024008ED00E0000001083F
:1005B0002DE9F04F99B0B34C01902022FF2110A8F3
:1005C000A66800F0E3FBB04A1378A346A3B9AF488E
:1005D0000121C3601170202383F31188C3680BB11C
:1005E00001F026FA0023AA4AA8484FF47A7101F0D4
:1005F000E3F9002383F31188019B13B1A54B019A02
:100600001A60A54AA349019F0292002313704B6010
:1006100099461C461D469846012000F07BFB002FA2
:1006200000F012829B4B1B68002B40F00D8219B02A
:10063000BDE8F08F0220FFF7B9FE002840F0FB81F3
:10064000019BB9F1000F08BF1F46944B1B88ADF802
:100650002C3002210BA800F081FADDE74FF47A700C
:1006600000F02EFA031E0393EADB0220FFF79EFE42
:1006700082460028E4D0039B581E042800F2DD8146
:10068000DFE800F0030E1114170018A8052340F846
:10069000343D042100F062FA54464FF0000856E061
:1006A00004217848F6E704217D48F3E704217D48DA
:1006B000F0E71C24204600F07DFA04340B9004215E
:1006C0000BA800F04BFA2C2CF4D1E5E7002DB7D0A5
:1006D000002CB5D00220FFF769FE0546002800F087
:1006E000AF8101206C4C00F063FA0220207000F012
:1006F00011FB4FF000095FFA89FA504600F068FAE2
:10070000074658B1504600F073FA09F10109002874
:10071000F1D12C46A9460027634B97E7012302201D
:10072000237000F0EDFA3E46DBF808309E4206D218
:10073000304600F03FFA0130EBD10436F4E7029B7B
:1007400000261E70534BA9465E602C46374600F0CB
:1007500025FB15B1002C18BF0027FFF72FFE5BE724
:10076000002D3FF46DAF002C3FF46AAF029B0220D6
:10077000187000F0CFFA322000F0A2F9B0F1000AB0
:10078000C0F25E811AF0030540F05A81DBF80820C0
:1007900006EB0A03934200F25381BAF5807F00F220
:1007A0004F8155450DDA4FF47A7000F089F90490C5
:1007B000049B002BC0F244813C4A049BAB5401359E
:1007C000EFE7C820FFF7F2FD0546002800F038816A
:1007D0001F2E11D8C6F12004544528BF544610AB33
:1007E00026F0030022463149184400F0A5FA2246BB
:1007F000FF212E4800F0CAFA4FEAAA0A5FFA8AF2ED
:100800002A493046FFF7F8FD0446002800F01A8117
:1008100006EB8A0605469AE70220FFF7C7FD002887
:100820003FF40EAFFFF7D8FD00283FF409AF4FF0BB
:10083000000A5346DBF8082092451CD2BAF11F0F7C
:1008400012D8109A01320FD02AF0030218A90A44D4
:1008500052F8202C0B92184604220BA900F014FB2E
:100860000AF1040A0346E5E75046039300F0A2F9B3
:10087000039B0B90EFE718A8042140F84C3D00F0D3
:100880006DF964E72824002074250020342400201A
:10089000910400087825002070240020C23300084D
:1008A0002C24002030240020C433000874240020AD
:1008B00018A8002340F8343D642100F02BF90028EB
:1008C0007FF4BEAE0220FFF771FD00283FF4B8AE02
:1008D0000B9800F09FF918AB43F8480D0421184617
:1008E000CDE718A8002340F8343D642100F012F948
:1008F00000287FF4A5AE0220FFF758FD00283FF442
:100900009FAE0B9800F094F918AB43F8440DE5E75F
:100910000220FFF74BFD00283FF492AE00F08EF965
:1009200018AB43F8400DD9E70220FFF73FFD002840
:100930003FF486AE0BA9142000F086F9824618A871
:10094000042140F83CAD00F009F951460BA896E7A8
:10095000322000F0B5F8B0F1000AFFF671AE1AF0DF
:10096000030F7FF46DAEDBF808200AEB0803934217
:100970003FF666AE0220FFF719FD00283FF460AE97
:100980002AF0030AC244D0453FF4E1AE404600F0ED
:1009900011F904210A900AA800F0E0F808F104080F
:1009A000F1E74FF47A70FFF701FD00283FF448AEFD
:1009B000FFF712FD00283FF4AFAE109B01330CD0BF
:1009C000082210A90020FFF717FD00283FF4A4AE6D
:1009D0002022FF2110A800F0D9F9FFF7EFFC3748DB
:1009E00000F0A6FF23E6002D3FF42AAE002C3FF4D2
:1009F00027AE18A8002340F8343D642100F08AF89F
:100A0000824600287FF41CAE0220FFF7CFFC0028AE
:100A10003FF416AE0390FFF7D1FC41F2883000F0AE
:100A200087FF0B9800F0EEF900F0B8F9039B5746EA
:100A30001C461D46F0E5054689E64FF00008FFE537
:100A40002546FDE52C4667E6002000F039F80490C5
:100A5000049B002BFFF6E3AD012000F051F9049B4D
:100A6000213B122B3FF6D8AD01A252F823F000BF74
:100A7000350600085D060008CD06000819060008C6
:100A80001906000819060008610700085109000846
:100A900019080008B1080008E30800081109000857
:100AA000190600082909000819060008A30900080A
:100AB0004F07000819060008E7090008A086010092
:100AC00037B5114B1A780132D2B20024012A0146FF
:100AD0008DF8074011D80D4803681D6A4FF47A73EA
:100AE0004B4301220DF10701A847012805D1084B0E
:100AF0009DF807001C7003B030BD4FF4FA7000F091
:100B000017FF4FF0FF30F6E70024002048260020B2
:100B10008425002038B50E4B1A780132D2B2012A52
:100B200005460ED80B4803681C6A4FF47A734B4392
:100B300004222946A047042803D1074B002018703F
:100B400038BD4FF4FA7000F0F3FE4FF0FF3038BDBF
:100B500000240020482600208425002030B4054CC5
:100B60002368DD69044B0A46AC460146204630BC8A
:100B7000604700BF48260020A086010070B501F044
:100B800023F9094C094E20700025306823788342F0
:100B900008D901F013F9336805440133B5F5803FF6
:100BA0003360F2D370BD00BF852500208025002072
:100BB00001F0B8B900F1006000F5803000687047BE
:100BC00000F10060920000F5803001F043B90000B0
:100BD000054B1A68054B1B789B1A834202D91044B7
:100BE00001F0ECB80020704780250020852500200A
:100BF00038B5074D04462868204401F0E7F828B9C5
:100C000028682044BDE8384001F0F8B838BD00BF7E
:100C10008025002010F0030308D1B0F5007F05D82F
:100C200000F10050A0F508400068704700207047B0
:100C3000014BC058704700BF107AFF1F014B186866
:100C4000704700BF002004E070B52A4B1C68C4F355
:100C50000B03240C63B140F21342934231D040F2B3
:100C6000194293422FD040F2214293422DD10323C7
:100C7000214A0C2505FB03235D6893F9082042F205
:100C800001039C4224D0B4F5805F23D041F20103DC
:100C90009C4221D041F203039C421FD041F2070342
:100CA0009C4208BF3122441E0C44013D0B46A34226
:100CB0001ED215F9016F581C96B1034600F8016C5D
:100CC000F5E70123D4E70223D2E73F220B4DD6E715
:100CD0003322E3E74122E1E75A22E4E75922E2E73F
:100CE0002C2584421D7001D9981C5A70401A70BD81
:100CF0001846FBE7002004E0D4330008C83300089E
:100D0000022802BF024B4FF400129A61704700BFE5
:100D100000040240022802BF014B20229A61704762
:100D200000040240022801BF024A536983F02003F5
:100D3000536170470004024010B50023934203D072
:100D4000CC5CC4540133F9E710BD000030B5441E3B
:100D500014F9010F0B4660B193F90050854201F17F
:100D6000010106D11AB993F90020801A30BD013A69
:100D7000EEE7002AF7D1104630BD000002460346D8
:100D8000981A13F9011B0029FAD17047024403464F
:100D9000934202D003F8011BFAE77047024B1A781E
:100DA000024B1A70704700BF8425002000240020E9
:100DB00038B5104D104C284600F002F9214628465F
:100DC00000F02AF924680D48626DD2F8043843F027
:100DD0000203C2F8043800F0ABFD0949204600F0D8
:100DE00027FA626DD2F8043823F00203C2F80438FF
:100DF00038BD00BF48260020A034000840420F0044
:100E0000C834000870470000FEE7000000B59BB042
:100E1000EFF3098168226846FFF78EFFEFF3058341
:100E2000034B9A6B9A6A9A6A9A6A9A6A9B6AFEE775
:100E300000ED00E000B59BB0EFF309816822684641
:100E4000FFF77AFFEFF30583044B9A6B9A6A9A6A6D
:100E50009A6A9A6A9A6A9B6AFEE700BF00ED00E010
:100E600000B59BB0EFF3098168226846FFF764FF85
:100E7000EFF30583034B5A6B9A6A9A6A9A6A9A6AE5
:100E80009B6AFEE700ED00E030B5084D0A44914250
:100E90000BD011F8013B09245840013CF7D040F336
:100EA00000032B4083EA5000F7E730BD2083B8ED04
:100EB000002304491A465A50C8180833802B426050
:100EC000F9D170478825002002684368114301600A
:100ED00003B118477047000013B5446BD4F894343D
:100EE0001A681178042915D1217C022912D11979A7
:100EF000128901238B4013420CD101A904F14C004B
:100F000001F02AFED4F89444019B2179024620681E
:100F100000F0DAF902B010BD143001F0ADBD0000F0
:100F20004FF0FF33143001F0A7BD00004C3001F04A
:100F30007FBE00004FF0FF334C3001F079BE00005F
:100F4000143001F07BBD00004FF0FF31143001F090
:100F500075BD00004C3001F04BBE00004FF0FF3279
:100F60004C3001F045BE0000D0F8942438B5136829
:100F700019780429054601D0012038BD017C0229D9
:100F8000FAD112795C89012090400440F4D105F136
:100F9000140001F00DFD02460028EDD0D5F8945460
:100FA0004FF480732868697900F07CF9204638BDD9
:100FB000406BFFF7D9BF000000207047704700006A
:100FC0007FB5124B0360002343608360C36001253B
:100FD00002260F4B057404460290019300F184022F
:100FE000294600964FF48073143001F0BDFC094B84
:100FF0000193029400964FF4807304F523722946FE
:1010000004F14C0001F084FD04B070BD24340008EC
:10101000B10F0008D90E00080B68202282F3118856
:101020000A7903EB820290614A79093243F822007F
:101030008A7912B103EB8203986102230374C0F82A
:101040009414002383F311887047000038B5037FA0
:10105000044613B190F85430ABB9201D012502218C
:10106000FFF732FF04F1140025776FF0010100F063
:1010700087FC84F8545004F14C006FF00101BDE886
:10108000384000F07DBC38BD10B501210446043065
:10109000FFF71AFF0023237784F8543010BD0000B7
:1010A00038B504460025143001F076FC04F14C00FC
:1010B000257701F045FD201D84F854500121FFF7EC
:1010C00003FF2046BDE83840FFF74EBF90F844309C
:1010D00003F06003202B19D190F84520212A0AD073
:1010E000222A4FF000030ED0202A0FD1084A826333
:1010F0000722C26304E0064B83630723C363002314
:101100000364012070478363C363F9E700207047DD
:1011100001240020D0F8943437B51A6811780429D6
:1011200004461AD1017C022917D1197912890123A9
:101130008B40134211D100F14C05284601F0C0FD4F
:1011400058B101A9284601F007FDD4F89444019B49
:1011500021790246206800F0B7F803B030BD0000E6
:1011600000EB8103F7B59C6905460E46F4B12023D8
:1011700083F3118805EB8607201D0821FFF7A4FEE5
:10118000FB685B691B684C3413B1204601F0F2FC2C
:1011900001A9204601F0E0FC024648B1019B31461E
:1011A000284600F091F8002383F3118803B0F0BDC6
:1011B000FB685A691268002AF5D01B8A013B13406C
:1011C000F1D105F14402EAE7093138B550F8214080
:1011D000DCB1202383F31188D4F894241368527966
:1011E00003EB8203DB689B695D6845B104216018ED
:1011F000FFF76AFE294604F1140001F0E3FB2046E4
:10120000FFF7B2FE002383F3118838BD704700005A
:1012100000F08EBF0123037000234360C36183622B
:101220000362C3624362036303814381704700002A
:1012300038B50446202383F3118800254160C5603A
:1012400005614561856100F083FF0223237085F30A
:10125000118838BD70B500EB810305465069DA602E
:101260000E46144618B110220021FFF78FFDA06929
:1012700018B110220021FFF789FD31462846BDE84C
:10128000704001F02FB80000028902F001020281D3
:10129000428902F0010242810022026142618261C0
:1012A00001F0B4B8F0B400EB81044789E46801258B
:1012B000A4698D403D43458123600023A2606360A3
:1012C000F0BC01F0CFB80000F0B400EB8104078956
:1012D000E468012564698D403D4305812360002356
:1012E000A2606360F0BC01F049B9000070B5022350
:1012F000002504460370A0F84C5080F84E5080F84A
:101300004F5005814581C56005614561856180F863
:10131000345000F083FF63681B6823B129462046E0
:10132000BDE87040184770BD436802781B6880F8BC
:101330005020052202700BB10421184770470000AD
:10134000436890F850201B6802700BB105211847C4
:101350007047000090F8343070B5044613B1002394
:1013600080F8343004F14402204601F071F86368DB
:101370009B6863BB94F8445015F0600615D194F84F
:10138000453005F07F0545EA032540F202339D42D2
:1013900000F00E815BD8022D00F0DC803FD8002DDC
:1013A00000F08780012D00F0CF800021204601F061
:1013B000A7FA0021204601F099FA63681B6813B16F
:1013C000062120469847062384F8343070BD204615
:1013D00098470028CED094F84B2094F84A3043EA3E
:1013E0000223E26B934238BFE36394F94430E56B28
:1013F000002B4FF0200380F2FD80002D00F0EC80E8
:10140000092284F8342083F311880021E36BA26B56
:101410002046FFF759FF002383F3118870BDB5F50F
:10142000817F00F0B180B5F5407F49D0B5F5807F70
:10143000BBD194F84630012BB7D1B4F84C3023F02F
:101440000203A4F84C30A663E6632664C3E740F2C7
:1014500001639D421ED8B5F5C06F3BD2B5F5A06FB4
:10146000A3D1B4F84430B3F5A06F0ED194F8463050
:1014700084F84E30204600F029FF63681B6813B1E2
:10148000012120469847032323700023A363E363CD
:101490002364A0E7B5F5106F32D040F602439D42B9
:1014A00052D0B5F5006F80D104F14F03A36301233F
:1014B00024E004F14C03A3630223E36325648AE779
:1014C00094F84630012B7FF470AFB4F84C3043F001
:1014D0000203B6E794F84920616894F848304D68F3
:1014E00094F8471043EA0223204694F84620A84780
:1014F00000283FF45AAF4368A3630368E363A4E79B
:101500002378042B10D1202383F311882046FFF782
:10151000BBFE86F31188636884F84F601B68032163
:1015200021700BB12046984794F84630002BACD080
:1015300084F84F300423237063681B68002BA4D009
:10154000022120469847A0E7374BA3630223E363B9
:1015500000239DE794F8481011F0800F204601F019
:101560000F010ED000F066FF012806D002287FF49C
:101570001CAF2E4BA363E06367E72D4BA363E563CA
:1015800063E700F049FFEFE794F84630002B7FF463
:101590000CAF94F8483013F00F013FF476AF1A0601
:1015A000204602D501F0C0F96FE701F0B3F96CE70E
:1015B00094F84630002B7FF4F8AE94F8483013F0DE
:1015C0000F013FF462AF1B06204602D501F098F9E7
:1015D0005BE701F08BF958E7142284F8342083F399
:1015E00011882B462A4629462046FFF75BFE85F3E5
:1015F000118870BD5DB1152284F8342083F3118801
:101600000021E36BA26B2046FFF74CFE03E70B22A1
:1016100084F8342083F311882B462A462946204635
:10162000FFF752FEE3E700BF543400084C340008D3
:101630005034000838B590F834300446152B29D8BA
:10164000DFE803F03E28282828283E28280B2939DF
:1016500028282828282828283E3E90F84B1090F863
:101660004A20C36B42EA01229A4214D9C268128A04
:10167000B3FBF2F502FB15356DB9202383F3118816
:101680002B462A462946FFF71FFE85F311880A23B9
:1016900084F8343038BD142384F83430202383F3A5
:1016A000118800231A4619462046FFF7FBFD002348
:1016B00083F3118838BD036C03B198470023E7E733
:1016C000002101F01DF90021204601F00FF96368A7
:1016D0001B6813B10621204698470623D8E700006F
:1016E00090F83420152A38B5044622D801239340B7
:1016F00040F6416213421DD113F480150FD19B02B5
:1017000017D50B2380F83430202383F311882B4620
:101710002A462946FFF7D8FD85F3118838BDC368EE
:101720009B695B682BB9036C03B19847002384F86D
:10173000343038BD002101F0E3F80021204601F0EB
:10174000D5F863681B6813B1062120469847062325
:10175000EDE70000024B00221B605B609A6070475F
:1017600008260020002303748268054B1B689968D3
:101770009142FBD25A680360426010605860704723
:101780000826002008B5202383F31188037C032B4F
:1017900005D0042B0DD02BB983F3118808BD436904
:1017A00000221A604FF0FF334361FFF7DBFF002395
:1017B000F2E790E80C001A6002685360F2E700005C
:1017C000002303748268054B1B6899689142FBD81B
:1017D0005A68036042601060586070470826002015
:1017E000054B19690874186802681A60536018611B
:1017F00001230374FEF788BD0826002030B54B1C7A
:1018000087B005460A4C10D023690A4A01A800F0A7
:10181000D3F82846FFF7E4FF049B13B101A800F0BA
:1018200007F92369586907B030BDFFF7D9FFF8E71A
:10183000082600208517000838B50C4D41612B693A
:1018400081689A689142044603D8BDE83840FFF7A2
:1018500089BF1846FFF786FF01232C6101462374D8
:101860002046BDE83840FEF74FBD00BF08260020E7
:10187000044B1A681B6990689B68984294BF0020CB
:10188000012070470826002010B5084C2368206905
:101890001A6822605460012223611A74FFF790FFD6
:1018A00001462069BDE81040FEF72EBD0826002045
:1018B0008260022202740022427470478368A3F19E
:1018C0007C0243F80C2C026943F83C2C426943F833
:1018D000382C074A43F81C2CC26843F8102C02220B
:1018E00003F8082C002203F8072CA3F11800704716
:1018F0002103000810B5202383F31188FFF7DEFFD2
:1019000000210446FFF798FF002383F31188204647
:1019100010BD0000024B1B6958610F20FFF760BF2C
:1019200008260020202383F31188FFF7F3BF00006F
:1019300008B50146202383F311880820FFF75EFFD6
:10194000002383F3118808BD49B1064B42681B6927
:1019500018605A60136043600420FFF74FBF4FF0D8
:10196000FF307047082600200368984206D01A68A6
:101970000260506059611846FFF7F4BE70470000DE
:1019800038B504460D462068844200D138BD03684E
:1019900023605C604561FFF7E5FEF4E7054B03F16A
:1019A00014025A619A614FF0FF32DA6100221A6222
:1019B000704700BF08260020F8B503614FF0804350
:1019C000C2605C6A194B1A46022952F8145F38BF8C
:1019D0000221954206461F460AD1586198611C6251
:1019E0000560456081600819BDE8F84001F08AB9DA
:1019F000186AAB68241A0C1902D3E41A2D6804E0A3
:101A00009C4202D2204401F08BF9AB689C42F4D88E
:101A10006B68736035601E606E60B460A9684FF0DB
:101A2000FF33091BA960FB61F8BD00BF0826002039
:101A300010B41B4C234653F8141F814210D0416848
:101A400002680A60026851609A424FF00001C1606A
:101A500003D0936881680B4493605DF8044B704732
:101A60000A68626100209A425360C86003D15DF841
:101A7000044B01F04FB993688868034493604FF0BA
:101A80008042206A526A121A9342E6D9991A0129B1
:101A900098BF931C18445DF8044B01F041B900BF96
:101AA0000826002000207047FEE700007047000075
:101AB0004FF0FF3070470000022906D0032906D0FE
:101AC0000129064818BF0020704705487047032ABF
:101AD0009ABF044800EBC20000207047243500087C
:101AE000D83400080824002070B59AB001AD06462D
:101AF00008462946144600F095F82846FFF73EF9B7
:101B0000C0B2431C5B0086E8180023700323637097
:101B1000002302341946DAB2904204F1020401D8DB
:101B20001AB070BDEA5C04F8022C04F8011C013301
:101B3000F1E7000008B5202383F311880348FFF77D
:101B4000E9FA002383F3118808BD00BF482600206E
:101B500010B50446052916D8DFE801F0161503165E
:101B6000161D202383F311880E4A0121FFF772FB13
:101B700020460D4A0221FFF76DFB0C48FFF790FA53
:101B8000002383F3118810BD202383F311880748B5
:101B9000FFF75CFAF4E7202383F311880348FFF78B
:101BA00073FAEDE7583400087C340008482600201A
:101BB00038B50C4D0C4C0D492A4604F10800FFF7CE
:101BC00093FF05F1CA0204F110000949FFF78CFFE9
:101BD00005F5CA7204F118000649BDE83840FFF760
:101BE00083BF00BF102B002008240020A834000869
:101BF000B2340008BD34000870B5044608460D46EE
:101C0000FFF7BCF8C6B22046013403780BB918467A
:101C100070BD32462946FFF799F80028F3D101201C
:101C200070BD00002DE9F84F05460C46FFF7A6F8F9
:101C30002C49C6B22846FFF7DFFF08B10436F6B2DA
:101C400029492846FFF7D8FF08B11036F6B2632EAF
:101C50000DD8DFF89090DFF890A0DFF89880DFF8DB
:101C600098B0224F2E7846B92670BDE8F88F2946E5
:101C70002046BDE8F84F01F09BBB252E2DD1072251
:101C800049462846FFF762F850B93B6823607B68F5
:101C900063603B892381BB7AA37207350B34E1E78C
:101CA000082251462846FFF751F8B0B9104BA21C44
:101CB00013F8011F09095B4511F8081002F8021C0E
:101CC000197801F00F0102F1020211F8081002F870
:101CD000031CEDD118340835C4E7267001350134F2
:101CE000C0E700BF44350008BD3400084C3500088B
:101CF0000F7AFF1F583500081B7AFF1FBFF34F8F65
:101D0000024AD368DB03FCD4704700BF003C0240AA
:101D100008B5094B1B7873B9FFF7F0FF074B1A6939
:101D2000002ABFBF064A5A6002F188325A601A6818
:101D300022F480621A6008BD6E2D0020003C024033
:101D40002301674508B50B4B1B7893B9FFF7D6FF06
:101D5000094B1A6942F000421A611A6842F4805233
:101D60001A601A6822F480521A601A6842F480627B
:101D70001A6008BD6E2D0020003C02400B2870B593
:101D800013D80B4A0B4C137863B90B4E4FF000611C
:101D900044F8231056F8235001330C2B2944F7D173
:101DA0000123137054F8200070BD002070BD00BFE7
:101DB000A02D0020702D00206C350008014B53F839
:101DC000200070476C3500080C2070470B2810B5B8
:101DD000044601D9002010BDFFF7D0FF064B53F891
:101DE00024301844C21A0BB9012010BD1268013208
:101DF000F0D1043BF6E700BF6C3500080B2810B5A6
:101E0000044621D8FFF77AFFFFF782FF0F4AF3233A
:101E1000D360C300DBB243F4007343F002031361E9
:101E2000136943F480331361FFF768FFFFF7A6FFE0
:101E3000074B53F8241000F0DDF8FFF783FF20462E
:101E4000BDE81040FFF7C2BF002010BD003C0240BB
:101E50006C3500082DE9F84312F00103154640D116
:101E60008218B2F1016F3CD22C4B1B6813F00103B6
:101E700037D02B4CFFF74CFFF323E360FFF73EFF17
:101E800040F20127032D01D9830713D0244C0F46BC
:101E9000401A40F20118EB1B0B44012B00EB070624
:101EA000236924D823F001032361FFF74BFF0120AE
:101EB000BDE8F883236923F44073236123693B431E
:101EC000236151F8046B0660BFF34F8FFFF716FFD5
:101ED00003689E4208D0236923F001032361FFF7C2
:101EE00031FF0020BDE8F883043D0430CAE723F445
:101EF00040732361236943EA08032361B94637F835
:101F0000023B3380BFF34F8FFFF7F8FE3688B9F8F6
:101F10000030B6B2B342BED0DDE700BF00380240A9
:101F2000003C0240084908B50B7828B153B9FFF7C7
:101F3000EFFE01230B7008BD23B1BDE80840087017
:101F4000FFF700BF08BD00BF6E2D002010B5024492
:101F5000064B0439D2B2904200D110BD441C00B2ED
:101F600053F8200041F8040FE0B2F4E75028004095
:101F7000104B30B51C6F240407D41C6F44F400745C
:101F80001C671C6F44F400441C670B4C236843F42B
:101F9000807323600244094B0439D2B2904200D1CD
:101FA00030BD441C00B251F8045F43F82050E0B249
:101FB000F4E700BF003802400070004050280040A5
:101FC00007B5012201A90020FFF7C0FF019803B067
:101FD0005DF804FB13B50446FFF7F2FFA04206D0FC
:101FE00002A9012241F8044D0020FFF7C1FF02B011
:101FF00010BD000070470000034B1B689B0042BFF0
:10200000024B01221A70704774380240A12D002043
:10201000014B1878704700BFA12D002070470000C9
:10202000FEE70000084A094B09498B4204D3094ADC
:102030000021934205D3704752F8040F43F8040B74
:10204000F3E743F8041BF4E71437000818300020C6
:102050001830002018300020836D30B500229D68B4
:10206000446D11464FF0FF3004EB421301329542AC
:10207000C3F80019C3F81019C3F80809C3F8001B06
:10208000C3F8101BC3F8080BEED24FF00113C4F8CD
:102090001C3830BD890141F02001016103699B06B4
:1020A000FCD4122000F0C4BE204B03EB80022DE9CB
:1020B000F047D2F80CE05D6DDEF81420461CD2F833
:1020C00000C005EB063605EB4018516861450BD39F
:1020D000D5F83428012303FA00F022EA0000C5F8FD
:1020E00034081846BDE8F087BEF81040ACEB010399
:1020F000A34228BF2346D8F81849A4B2B3EB840FF3
:1021000010D894681F46A4F1040959F804AFC6F822
:1021100000A0042F01D9043FF7E71C440B4494604E
:102120005360D2E70020BDE8F08700BFA42D002057
:1021300010B5054C2046FFF76DF84FF0A0436365DE
:10214000024BA36510BD00BFA42D0020C0350008C0
:102150000378012B70B5054650D12A4B446D984247
:102160001BD1294B5A6B42F080025A635A6D42F0E0
:1021700080025A655A6D5A6942F080025A615A6962
:1021800022F080025A610E2143205B6900F0D6FBE9
:102190001E4BE3601E4BC4F800380023C4F8003E19
:1021A000C02323606E6D4FF40413A3633369002BC7
:1021B000FCDA012333610C2000F03AFE3369DB07BF
:1021C000FCD4122000F034FE3369002BFCDA002628
:1021D000A6602846FFF740FF6B68C4F81068DB680C
:1021E000C4F81468C4F81C684BB90A4BA3614FF0DB
:1021F000FF336361A36843F00103A36070BD064B26
:10220000F4E700BFA42D0020003802404014004035
:1022100003002002003C30C0083C30C0F8B5446DDB
:10222000054600212046FFF735FFA96D00234FF03A
:1022300001128F68C4F834384FF00066C4F81C28C7
:102240004FF0FF3004EB431201339F42C2F80069A4
:10225000C2F8006BC2F80809C2F8080BF2D20B688A
:102260006A6DEB65636210231361166916F0100640
:10227000FBD1122000F0DCFDD4F8003823F4FE631B
:10228000C4F80038A36943F4402343F01003A3616A
:102290000923C4F81038C4F814380A4BEB604FF027
:1022A000C043C4F8103B084BC4F8003BC4F81069A5
:1022B000C4F80039EB6D03F1100243F48013EA65B2
:1022C000A362F8BD9C35000840800010426D90F874
:1022D0004E10D2F8003823F4FE6343EA0113C2F82B
:1022E000003870472DE9F0410EB200EB86080D462C
:1022F000D8F80C100F6807F00303022B50D0032B03
:1023000050D03D4A3D4F012B18BF1746446D4FEA50
:10231000451E04EB0E030022C3F8102B8A6905F159
:10232000100C002A40D04A8A05F158035B013A4359
:10233000E2500123D4F81C2803FA0CF31343A644FB
:102340004A69C4F81C380023CEF8103905F13F0360
:10235000002A39D00A8A898B9208012988BF4A430A
:10236000C16D04EB8303561841EA0242C665294653
:102370005A602046FFF78EFED8F80C301B8A43EADD
:1023800085531F4305F148035B01E7500123D4F84F
:102390001C2803FA05F51543C4F81C58BDE8F08164
:1023A000174FB3E7174FB1E704EB4613D3F8002BF1
:1023B00022F40042C3F8002BD4F81C28012303FAAE
:1023C0000CF322EA0303BAE704EB83030E4A5A60D4
:1023D00004EB461629462046FFF75CFED6F8003986
:1023E00023F40043C6F80039D4F81C38012202FA5D
:1023F00005F523EA0505CFE70080001000800410F2
:102400000080081000800C1000040002826D126829
:10241000C265FFF721BE00005831436D49015B588A
:1024200013F4004004D013F4001F14BF0120022055
:10243000704700004831436D49015B5813F4004078
:1024400004D013F4001F14BF0120022070470000C5
:1024500000EB8101CB68196A0B6813604B6853600D
:102460007047000000EB810330B5DD68AA6913688E
:10247000D36019B9402B84BF402313606B8A146862
:10248000426D1C44013CB4FBF3F46343033323F07B
:10249000030302EB411043EAC44343F0C043C0F8D6
:1024A000103B2B6803F00303012B09B20ED1D2F8C5
:1024B000083802EB411013F4807FD0F8003B14BFC2
:1024C00043F0805343F00053C0F8003B02EB41124D
:1024D000D2F8003B43F00443C2F8003B30BD00009B
:1024E0002DE9F041244D6E6D06EB40130446D3F800
:1024F000087BC3F8087B38070AD5D6F814381907C3
:1025000006D505EB84032146DB6828465B689847BF
:10251000FA072FD5D6F81438DB072BD505EB840343
:10252000D968CCB98B69488A5E68B6FBF0F200FBCB
:1025300012628AB91868DA6890420DD2121A83E8DA
:102540001400202383F311880B482146FFF78AFFEC
:1025500084F31188BDE8F081012303FA04F26B894A
:1025600023EA02036B81CB6823B121460248BDE810
:10257000F0411847BDE8F081A42D002000EB810355
:1025800070B5DD68436D6C692668E6604A0156BB2C
:102590001A444FF40020C2F810092A6802F003021E
:1025A000012A0AB20ED1D3F8080803EB421410F442
:1025B000807FD4F8000914BF40F0805040F00050F4
:1025C000C4F8000903EB4212D2F8000940F00440BD
:1025D000C2F80009D3F83408012202FA01F10143DC
:1025E000C3F8341870BD19B9402E84BF4020206054
:1025F00020682E8A841940F00050013C1A44B4FB34
:10260000F6F440EAC440C6E7F8B504461E48456DF6
:1026100005EB4413D3F80869C3F80869F10717D527
:10262000D5F81038DA0713D500EB8403D9684B6965
:102630001F68DA68974218D2D21B00271A605F60C1
:10264000202383F311882146FFF798FF87F3118831
:10265000330617D5D5F834280123A340134211D0EF
:102660002046BDE8F840FFF71FBD012303FA04F23E
:10267000038923EA020303818B68002BE8D02146FB
:102680009847E5E7F8BD00BFA42D002096482DE946
:10269000F84F456D6E69AB691E4016F4805F6E6140
:1026A000044605D0FEF722FEBDE8F84F00F054BC0A
:1026B000002E12DAD5F8003E8B489B071EBFD5F8D6
:1026C000003E23F00303C5F8003ED5F8043823F09C
:1026D0000103C5F80438FEF733FE370502D58248FA
:1026E000FEF722FEB0040CD5D5F8083813F0060F1B
:1026F000EB6823F470530CBF43F4105343F4A0531E
:10270000EB60310704D56368DB680BB17648984706
:10271000F2025AD4B3020CD5D4F85480DFF8C8A121
:1027200000274FF00109A36D9B68F9B28B4280F03E
:102730008780F70619D5616D0A6AC2F30A1702F09D
:102740000F0302F4F012B2F5802F00F0A180B2F571
:10275000402F0AD104EB830301F58051DB68186A2E
:1027600000231A469F4240F087803003D5F818486E
:1027700013D5E10302D50020FFF7B2FEA20302D574
:102780000120FFF7ADFE630302D50220FFF7A8FE8C
:10279000270302D50320FFF7A3FE750384D5E007C6
:1027A00002D50020FFF730FFA10702D50120FFF777
:1027B0002BFF620702D50220FFF726FF23077FF5D4
:1027C00073AF0320FFF720FF6EE7D4F85480DFF8E3
:1027D00018A100274FF00109A36D9B685FFA87FBE2
:1027E0005B4597D308EB4B13D3F8002902F4402242
:1027F000B2F5802F22D1D3F80029002A1EDAD3F8AF
:10280000002942F09042C3F80029D3F80029002A99
:10281000FBDB5946606DFFF73DFC228909FA0BF39B
:1028200022EA0303238104EB8B03DB689B6813B16B
:102830005946504698475846FFF736FC0137CBE7D4
:1028400008EB4112D2F8003B03F44023B3F5802F8C
:1028500010D1D2F8003B002B0CDA628909FA01F39F
:1028600022EA0303638104EB8103DB68DB680BB1BD
:1028700050469847013756E79C0708BF0A68072B60
:1028800098BF027003F101039CBF120A013069E78F
:10289000023304EB830201F58051526890690268AB
:1028A000D0F808C04068A2EB000E00221046974204
:1028B0000AD104EB830463689B699A683A449A607E
:1028C0005A6817445F6050E712F0030F08BF0868AA
:1028D000964588BF8CF8000002F1010284BF000A0F
:1028E0000CF1010CE3E700BFA42D0020436D03EBC6
:1028F0004111D1F8003B43F40013C1F8003B70478D
:10290000436D03EB4111D1F8003943F40013C1F8D2
:1029100000397047436D03EB4111D1F8003B23F4BC
:102920000013C1F8003B7047436D03EB4111D1F830
:10293000003923F40013C1F80039704700F16043F7
:1029400000F01F02400903F5614309018000C9B28C
:1029500000F1604083F8001300F5614001239340CB
:10296000C0F880310360704730B5039C01720433B6
:1029700004FB0325C361049B03630021059B0060E6
:102980004060C160426102618561046242628162AD
:10299000C162436330BD00000022416A41610161B0
:1029A000C2608262C2626FF00101FEF7E9BF0000FF
:1029B00003694269934203D1C2680AB1002070479B
:1029C000181D704703691960C2680132C260C2698C
:1029D000134482690361934224BF436A0361002167
:1029E000FEF7C2BF38B504460D46E3683BB16269E5
:1029F000131D1268A3621344E362002038BD237ADA
:102A000033B929462046FEF79FFF0028EDDA38BD8E
:102A10006FF00100FBE70000C368C269013BC360BF
:102A20004369134482694361934224BF436A43610B
:102A300000238362036B03B11847704770B52023EE
:102A4000044683F31188866A3EB9FFF7CBFF05463B
:102A500018B186F31188284670BDA36AE26A13F89C
:102A6000015BA362934202D32046FFF7D5FF002308
:102A700083F31188EFE700002DE9F84F04460E4676
:102A800090469946202787F311880025AA46D4F856
:102A900028B0BBF1000F09D149462046FFF7A2FF3D
:102AA00020B18BF311882846BDE8F88FA16AE36A4C
:102AB000A8EB050B5B1A9B4528BF9B46BBF1400F5B
:102AC0001BD9334601F1400251F8040B43F8040BC3
:102AD0009142F9D1A36A40334036A3624035A26ADD
:102AE000E36A9A4202D32046FFF796FF8AF31188E1
:102AF0004545D8D287F31188C9E730465A46FEF7D4
:102B00001BF9A36A5B445E44A3625D44E7E70000EF
:102B100010B5029C0172043303FB0421C36100233E
:102B20008362C362039B0363049B00604060C460D4
:102B300042610261816104624262436310BD000030
:102B4000026AC260426A4261026100228262C2621B
:102B50006FF00101FEF714BF436902699A4203D185
:102B6000C2680AB100207047184650F8043B0B6059
:102B700070470000C368C2690133C36043691344EE
:102B800082694361934224BF436A43610021FEF797
:102B9000EBBE000038B504460D46E3683BB123693F
:102BA0001A1DA262E2691344E362002038BD237A51
:102BB00033B929462046FEF7C7FE0028EDDA38BDB6
:102BC0006FF00100FBE7000003691960C268013A79
:102BD000C260C269134482690361934224BF436A9D
:102BE000036100238362036B03B118477047000041
:102BF00070B5202304460E4683F31188856A35B9E3
:102C00001146FFF7C7FF10B185F3118870BDA36AA5
:102C10001E70A36AE26A01339342A36204D3E1699E
:102C200020460439FFF7D0FF002080F3118870BDE3
:102C30002DE9F84F04460D4691469A464FF020087C
:102C400088F311880026B346A76A4FB9514620463B
:102C5000FFF7A0FF20B187F311883046BDE8F88F59
:102C6000A06AE76AA9EB06033F1A9F4228BF1F46E6
:102C7000402F1BD905F1400355F8042B40F8042BD5
:102C80009D42F9D1A36A4033A3624036A26AE36A47
:102C90009A4204D3E16920460439FFF795FF8BF38C
:102CA00011884E45D9D288F31188CDE729463A4696
:102CB000FEF742F8A36A3B443D44A3623E44E5E785
:102CC000026943699A4203D1C3681BB91846704729
:102CD0000023FBE7836A002BF8D0043B9B1AF5D056
:102CE0001360C368013BC360C3691A44836902610E
:102CF0009A4224BF436A0361002383620123E5E70C
:102D000000F06CB94FF08043002258631A61022230
:102D1000DA6070474FF080430022DA6070470000AD
:102D20004FF0804358637047FEE7000010B5174C22
:102D3000FEF710FDFEF732FE802215492046FEF711
:102D4000B7FD012344F8180C0374124B124AD968DA
:102D500021F4E0610904090C0A431049DA60CA68E9
:102D600042F08072CA600E490A6842F001020A60AD
:102D70001022DA77202283F82220002383F311889F
:102D800062B60848BDE81040FEF7B4BD302600200A
:102D9000CC35000800ED00E00003FA05F0ED00E09E
:102DA000001000E0D43500082DE9F84F1F4C4FF01B
:102DB0000008656904F11407C1464FF08043266A94
:102DC0005B6AAA689E1B96421DD34FF0200AAA6830
:102DD000236AD5F80CB0134423622B68BB425F60B2
:102DE000A6EB02066361C5F80C8001D1FFF792FFE4
:102DF00089F311882869D8478AF311886569AB6817
:102E00009E42E4D2D9E76269BA420CD0916823624B
:102E10008E1B9660A86802282CBF1818981CBDE865
:102E2000F84FFFF77DBFBDE8F88F00BF08260020F0
:102E3000034B59685A68521A9042FBD8704700BF3A
:102E4000001000E04B6843608B688360CB68C36010
:102E50000B6943614B6903628B6943620B680360D2
:102E60007047000008B5224B22481A6940F2FF1152
:102E70000A431A611A6922F4FF7222F001021A61F0
:102E80001A691A6B0A431A631A6D0A431A651A4AB9
:102E90001B6D1146FFF7D6FF184802F11C01FFF722
:102EA000D1FF174802F13801FFF7CCFF154802F1B6
:102EB0005401FFF7C7FF144802F17001FFF7C2FF8A
:102EC000124802F18C01FFF7BDFF114802F1A80181
:102ED000FFF7B8FF0F4802F1C401FFF7B3FF0E4838
:102EE00002F1E001FFF7AEFFBDE8084000F0E0B8F6
:102EF0000038024000000240F4350008000402409F
:102F000000080240000C0240001002400014024081
:102F100000180240001C02400020024008B500F0EA
:102F200037FAFFF703FFFFF767F8BDE80840FEF741
:102F30003FBE000070470000064A536823F00103BB
:102F40005360EFF30983683383F30988002383F325
:102F50001188704730EF00E010B5202383F311880B
:102F6000104B5B6813F4006318D0F1EE103AEFF3E6
:102F700009844FF0807344F84C3C0B4BDB6844F8F9
:102F8000083CA4F1680383F30988FEF771FC18B1CB
:102F9000064B44F8503C10BD054BFAE783F311880B
:102FA00010BD00BF00ED00E030EF00E0310300088D
:102FB000340300084FF0804310B51A69920708D512
:102FC00000241C61202383F31188FFF7EDFE84F3B6
:102FD0001188BDE81040FFF7BFBF0000104B1A6C0E
:102FE00042F001021A641A6E42F001021A660D4A9A
:102FF0001B6E936843F0010393604FF080435322AC
:103000009A624FF0FF32DA6200229A615A63DA6004
:103010005A6001225A6108211A601C20FFF78EBCF9
:1030200000380240002004E01F4B1A696FEAC252C8
:103030006FEAD2521A611A69C2F308021A614FF09C
:10304000FF301A695A69586100215A6959615A69F1
:103050001A6A62F080521A621A6A02F080521A6288
:103060001A6A5A6A58625A6A59625A6A1A6C42F063
:1030700080521A641A6E42F080521A661A6E0B4A17
:10308000106840F480701060186F00F44070B0F564
:10309000007F1EBF4FF4803018671967536823F410
:1030A0000073536000F054B90038024000700040D3
:1030B000304B4FF080521A642F4A4FF44041116058
:1030C0001A6842F001021A601A689207FCD59A68E1
:1030D00022F003029A60274B19469A6812F00C02FC
:1030E000FBD1186800F0F90018609A601A6842F481
:1030F00080321A600B689B03FCD54B6F43F00103D1
:103100004B671C4B5A6F9007FCD51C4A5A601A68D3
:1031100042F080721A60184A53685904FCD5154B66
:103120001A689201FCD5164A9A60164B1A68164B1B
:103130009A42164B1BD1164A1168164A914216D173
:1031400040F205121A600B4B9A6842F002029A6034
:103150009A6802F00C02082AFAD15A6C42F48042B2
:103160005A645A6E42F480425A665B6E704740F26F
:103170000572E7E70038024000700040085440073D
:1031800000948838002004E011640020003C0240D4
:1031900000ED00E041C20F41084A08B553691168CB
:1031A0000B4003F00103536123B1054A13680BB1CF
:1031B00050689847BDE80840FFF7CEBE003C01408C
:1031C00088250020084A08B5536911680B4003F0B0
:1031D0000203536123B1054A93680BB1D068984745
:1031E000BDE80840FFF7B8BE003C0140882500203C
:1031F000084A08B5536911680B4003F00403536192
:1032000023B1054A13690BB150699847BDE80840DE
:10321000FFF7A2BE003C014088250020084A08B5FF
:10322000536911680B4003F00803536123B1054A49
:1032300093690BB1D0699847BDE80840FFF78CBE91
:10324000003C014088250020084A08B553691168F0
:103250000B4003F01003536123B1054A136A0BB10D
:10326000506A9847BDE80840FFF776BE003C014031
:1032700088250020174B10B55C691A68144004F4C7
:1032800078725A61A30604D5134A936A0BB1D06AC7
:103290009847600604D5104A136B0BB1506B9847E2
:1032A000210604D50C4A936B0BB1D06B9847E2050D
:1032B00004D5094A136C0BB1506C9847A30504D58B
:1032C000054A936C0BB1D06C9847BDE81040FFF7EE
:1032D00043BE00BF003C0140882500201A4B10B5BA
:1032E0005C691A68144004F47C425A61620504D592
:1032F000164A136D0BB1506D9847230504D5134A38
:10330000936D0BB1D06D9847E00404D50F4A136E4E
:103310000BB1506E9847A10404D50C4A936E0BB1C3
:10332000D06E9847620404D5084A136F0BB1506FF2
:103330009847230404D5054A936F0BB1D06F984783
:10334000BDE81040FFF708BE003C01408825002082
:10335000062108B50846FFF7F1FA06210720FFF716
:10336000EDFA06210820FFF7E9FA06210920FFF708
:10337000E5FA06210A20FFF7E1FA06211720FFF7F8
:10338000DDFA06212820BDE80840FFF7D7BA000083
:1033900008B5FFF749FEFDF78BFDFDF739FFFDF797
:1033A0000DFEFFF7C7FDBDE80840FFF7A9BC000010
:1033B000034611F8012B03F8012B002AF9D17047BD
:1033C000121012131211000053544D3332463F3F76
:1033D0003F00000000000000C83300083F0000006C
:1033E00013040000043400083F000000190400002A
:1033F0000E3400083F0000002104000018340008CB
:103400003F00000053544D3332463430780053545B
:103410004D3332463432780053544D3332463434CF
:103420003658580000000000350F0008210F000832
:103430005D0F0008490F0008550F0008410F0008F4
:103440002D0F0008190F0008B90F00080000000038
:103450000100000000000000020000000000000069
:1034600061110008C911000840004000E02A002056
:10347000F02A00200200000000000000030000000D
:10348000000000000D120008000000001000000005
:10349000002B0020000000000100000000000000E0
:1034A000A42D0020010102004172647550696C6F07
:1034B000740025424F415244252D424C002553456E
:1034C0005249414C25000000511B0008B91A000860
:1034D000CD100008351B000843000000E034000850
:1034E00009024300020100C0320904000001020287
:1034F000010005240010010524010001042402023A
:103500000524060001070582030800FF09040100E5
:10351000020A0000000705010240000007058102C1
:1035200040000000120000002C35000812011001BC
:10353000020000400912415700020102030100008D
:103540000403090425424F41524425007370656508
:10355000647962656566340030313233343536372C
:103560003839414243444546000000000040000015
:10357000004000000040000000400000000001008A
:103580000000020000000200000002000000020033
:103590000000020000000200000002000000000025
:1035A0005513000835160008E116000840004000D9
:1035B000042E0020042E002001000000142E002004
:1035C0008000000040010000030000006D61696E92
:1035D00000000000EC350008202E002018300020EC
:1035E00001000000292D00080000000069646C65DE
:1035F000000000000000800200000000AAAAAAAAA1
:1036000000000000FFFF00000000000000A00A0012
:103610000004500000000000AAAAAAAA000050005E
:10362000DFFF0000000000000000000001000000BB
:1036300000000000AAAAAAAA01000000FFFF0000E3
:10364000000000000000000000000000000000007A
:10365000AAAAAAAA00000000FFFF000000000000C4
:10366000000000000000000000000000AAAAAAAAB2
:1036700000000000FFFF000000000000000000004C
:103680000000000000000000AAAAAAAA0000000092
:10369000FFFF00000000000000000000000000002C
:1036A00000000000AAAAAAAA00000000FFFF000074
:1036B000000000000000000000000000000000000A
:1036C0000A000000000000000300000000000000ED
:1036D00000000000000000000000000000000000EA
:1036E00000000000000000000000000000000000DA
:1036F000FF009600000000080400000040350008AC
:1037000000000000000000000000000000000000B9
:103710000000000000000000FFFFFFFFFFFFFFFFB1
:10372000FFFFFFFFFFFFFFFFFFFFFFFFFFFFFFFFA9
:10373000FFFFFFFFFFFFFFFFFFFFFFFFFFFFFFFF99
:10374000FFFFFFFFFFFFFFFFFFFFFFFFFFFFFFFF89
:10375000FFFFFFFFFFFFFFFFFFFFFFFFFFFFFFFF79
:020000040801F1
:10000000000600209912010809A9090865A8090835
:10001000D1A8090865A809089DA809089B1201082C
:100020009B1201089B1201089B12010885B80B085E
:100030009B1201089B1201089B1201089B120108E8
:100040009B1201089B1201089B1201089B120108D8
:100050009B1201089B120108A1CA0B08C9CA0B0810
:10006000F1CA0B0819CB0B0841CB0B08A5740B0880
:10007000CD740B08F9740B0825750B0851750B0826
:1000800079750B08A5750B0829740B089B120108DC
:100090009B1201089B1201089B12010869CB0B08F7
:1000A0008DCC0B08A1CC0B08B5CC0B08B9CC0B0838
:1000B000BDCC0B089B1201089B120108317B0B0879
:1000C000D97C0B089B1201089B1201089B120108A6
:1000D0009B1201083DCC0B089B12010851CC0B0868
:1000E000CDCB0B089B1201089B120108E1CC0B0839
:1000F000E5CC0B08F9CC0B08FDCC0B08D1750B082F
:100100009B1201089B120108D1CC0B089B1201081D
:1001100065CC0B0879CC0B089B1201089B120108D7
:10012000FD750B0825760B0851760B087D760B08BC
:10013000A9760B089B1201089B1201089B1201086B
:100140009B1201089B1201089B120108B1BF0B080A
:10015000D1760B08FD760B0829770B089B12010856
:100160009B1201089B1201089B1201089B120108B7
:100170009B1201089B1201089B1201089B120108A7
:100180009B1201089B1201089B1201089B12010897
:100190009B1201089B1201089B1201089B12010887
:1001A0009B1201089B1201089B1201089B12010877
:1001B0009B1201089B1201089B1201089B12010867
:1001C0009B1201089B1201089B1201089B12010857
:1001D0009B1201089B1201089B1201089B12010847
:1001E000093501081D6501082DEC0108353A0208A2
:1001F00095B90208C92E04086DB3050875B905083C
:100200009924060801750608C57C0608FD7F0608C6
:1002100061E00608DDFE0608B5950708DD0308085D
:10022000D5A1090821900A088DF10A08E5170B08E5
:1002300065220B0825500B08ED550B080000000047
:1002400081F0004102E000BF83F0004330B54FEA87
:1002500041044FEA430594EA050F08BF90EA020FF4
:100260001FBF54EA000C55EA020C7FEA645C7FEA87
:10027000655C00F0E2804FEA5454D4EB5555B8BFAA
:100280006D420CDD2C4480EA020281EA030382EA1B
:10029000000083EA010180EA020281EA0303362DAD
:1002A00088BF30BD11F0004F4FEA01314FF4801C80
:1002B0004CEA113102D0404261EB410113F0004F92
:1002C0004FEA03334CEA133302D0524263EB430349
:1002D00094EA050F00F0A780A4F10104D5F1200EE7
:1002E0000DDB02FA0EFC22FA05F2801841F1000142
:1002F00003FA0EF2801843FA05F359410EE0A5F116
:1003000020050EF1200E012A03FA0EFC28BF4CF046
:10031000020C43FA05F3C01851EBE37101F00045FC
:1003200007D54FF0000EDCF1000C7EEB00006EEB09
:100330000101B1F5801F1BD3B1F5001F0CD3490893
:100340005FEA30004FEA3C0C04F101044FEA4452EA
:1003500012F5800F80F09A80BCF1004F08BF5FEA71
:10036000500C50F1000041EB045141EA050130BD51
:100370005FEA4C0C404141EB0101013C28BFB1F563
:10038000801FE9D291F0000F04BF01460020B1FAAE
:1003900081F308BF2033A3F10B03B3F120020CDA81
:1003A0000C3208DD02F1140CC2F10C0201FA0CF05F
:1003B00021FA02F10CE002F11402D8BFC2F1200CC4
:1003C00001FA02F120FA0CFCDCBF41EA0C0190407A
:1003D000E41AA2BF01EB0451294330BD6FEA0404C3
:1003E0001F3C1CDA0C340EDC04F11404C4F12002AE
:1003F00020FA04F001FA02F340EA030021FA04F3C0
:1004000045EA030130BDC4F10C04C4F1200220FA16
:1004100002F001FA04F340EA0300294630BD21FA54
:1004200004F0294630BD94F0000F83F4801306BF1A
:1004300081F480110134013D4EE77FEA645C18BF0E
:100440007FEA655C29D094EA050F08BF90EA020FA5
:1004500005D054EA000C04BF1946104630BD91EA9D
:10046000030F1EBF0021002030BD5FEA545C05D1A0
:100470004000494128BF41F0004130BD14F58004DF
:100480003CBF01F5801130BD01F0004545F0FE4153
:1004900041F470014FF0000030BD7FEA645C1ABF88
:1004A000194610467FEA655C1CBF0B46024650EABF
:1004B000013406BF52EA033591EA030F41F40021EB
:1004C00030BD00BF90F0000F04BF0021704730B571
:1004D0004FF4806404F132044FF000054FF0000146
:1004E00050E700BF90F0000F04BF0021704730B507
:1004F0004FF4806404F1320410F0004548BF4042DC
:100500004FF000013EE700BF42004FEAE2014FEA30
:1005100031014FEA02701FBF12F07F4393F07F4F0B
:1005200081F06051704732F07F4208BF704793F00E
:100530007F4F04BF41F40021704730B54FF4607421
:1005400001F0004521F000411CE700BF50EA010224
:1005500008BF704730B54FF000050AE050EA0102CD
:1005600008BF704730B511F0004502D5404261EB3D
:1005700041014FF4806404F132045FEA915C3FF47E
:10058000D8AE4FF003025FEADC0C18BF03325FEA1B
:10059000DC0C18BF033202EBDC02C2F1200300FACC
:1005A00003FC20FA02F001FA03FE40EA0E0021FAF1
:1005B00002F11444BDE600BF70B54FF0FF0C4CF4DF
:1005C000E06C1CEA11541DBF1CEA135594EA0C0F91
:1005D00095EA0C0F00F0DEF82C4481EA030621EACC
:1005E0004C5123EA4C5350EA013518BF52EA033507
:1005F00041F4801143F4801338D0A0FB02CE4FF0B9
:100600000005E1FB02E506F00042E0FB03E54FF0E8
:100610000006E1FB03569CF0000F18BF4EF0010EE0
:10062000A4F1FF04B6F5007F64F5407404D25FEADC
:100630004E0E6D4146EB060642EAC62141EA55518F
:100640004FEAC52040EA5E504FEACE2EB4F1FD0CD1
:1006500088BFBCF5E06F1ED8BEF1004F08BF5FEA4F
:10066000500E50F1000041EB045170BD06F0004601
:1006700046EA010140EA020081EA0301B4EB5C04AE
:10068000C2BFD4EB0C0541EA045170BD41F48011A6
:100690004FF0000E013C00F3AB8014F1360FDEBFCB
:1006A000002001F0004170BDC4F10004203C35DAA7
:1006B0000C341BDC04F11404C4F1200500FA05F32A
:1006C00020FA04F001FA05F240EA020001F00042CB
:1006D00021F0004110EBD37021FA04F642EB060141
:1006E0005EEA430E08BF20EAD37070BDC4F10C046B
:1006F000C4F1200500FA04F320FA05F001FA04F22F
:1007000040EA020001F0004110EBD37041F100011A
:100710005EEA430E08BF20EAD37070BDC4F1200525
:1007200000FA05F24EEA020E20FA04F301FA05F28D
:1007300043EA020321FA04F001F0004121FA04F235
:1007400020EA020000EBD3705EEA430E08BF20EA05
:10075000D37070BD94F0000F0FD101F0004640003F
:1007600041EB010111F4801F08BF013CF7D041EAC1
:10077000060195F0000F18BF704703F000465200C5
:1007800043EB030313F4801F08BF013DF7D043EA96
:100790000603704794EA0C0F0CEA135518BF95EA4C
:1007A0000C0F0CD050EA410618BF52EA4306D1D1D3
:1007B00081EA030101F000414FF0000070BD50EAF2
:1007C000410606BF1046194652EA430619D094EA7C
:1007D0000C0F02D150EA013613D195EA0C0F05D166
:1007E00052EA03361CBF104619460AD181EA0301BA
:1007F00001F0004141F0FE4141F470014FF0000072
:1008000070BD41F0FE4141F4780170BD70B54FF00C
:10081000FF0C4CF4E06C1CEA11541DBF1CEA13558C
:1008200094EA0C0F95EA0C0F00F0A7F8A4EB05046E
:1008300081EA030E52EA03354FEA013100F0888065
:100840004FEA03334FF0805545EA131343EA12632E
:100850004FEA022245EA111545EA10654FEA0026E3
:100860000EF000419D4208BF964244F1FD0404F59C
:10087000407402D25B084FEA3202B61A65EB0305F8
:100880005B084FEA32024FF480104FF4002CB6EBB5
:10089000020E75EB030E22BFB61A754640EA0C0035
:1008A0005B084FEA3202B6EB020E75EB030E22BF75
:1008B000B61A754640EA5C005B084FEA3202B6EBB6
:1008C000020E75EB030E22BFB61A754640EA9C0075
:1008D0005B084FEA3202B6EB020E75EB030E22BF45
:1008E000B61A754640EADC0055EA060E18D04FEA03
:1008F000051545EA16754FEA06164FEAC30343EAA3
:1009000052734FEAC2025FEA1C1CC0D111F4801F6F
:100910000BD141EA00014FF000004FF0004CB6E768
:1009200011F4801F04BF01430020B4F1FD0C88BF07
:10093000BCF5E06F3FF6AFAEB5EB030C04BFB6EB12
:10094000020C5FEA500C50F1000041EB045170BD05
:100950000EF0004E4EEA113114EB5C04C2BFD4EB32
:100960000C0541EA045170BD41F480114FF0000EB6
:10097000013C90E645EA060E8DE60CEA135594EA32
:100980000C0F08BF95EA0C0F3FF43BAF94EA0C0F35
:100990000AD150EA01347FF434AF95EA0C0F7FF4AA
:1009A00025AF104619462CE795EA0C0F06D152EAFE
:1009B00003353FF4FDAE1046194622E750EA4106E2
:1009C00018BF52EA43067FF4C5AE50EA41047FF4F3
:1009D0000DAF52EA43057FF4EBAE12E74FF0FF3C58
:1009E00006E000BF4FF0010C02E000BF4FF0010C29
:1009F0004DF804CD4FEA410C7FEA6C5C4FEA430CA2
:100A000018BF7FEA6C5C1BD001B050EA410C0CBFF0
:100A100052EA430C91EA030F02BF90EA020F002052
:100A2000704710F1000F91EA030F58BF994208BFB9
:100A300090422CBFD8176FEAE37040F00100704776
:100A40004FEA410C7FEA6C5C02D150EA013C07D1CD
:100A50004FEA430C7FEA6C5CD6D152EA033CD3D018
:100A60005DF8040B704700BF8446104662468C4612
:100A70001946634600E000BF01B5FFF7B7FF002845
:100A800048BF10F1000F01BD4DF808EDFFF7F4FF6E
:100A90000CBF012000205DF808FB00BF4DF808EDF9
:100AA000FFF7EAFF34BF012000205DF808FB00BF1C
:100AB0004DF808EDFFF7E0FF94BF012000205DF83E
:100AC00008FB00BF4DF808EDFFF7CEFF94BF0120F3
:100AD00000205DF808FB00BF4DF808EDFFF7C4FFEC
:100AE00034BF012000205DF808FB00BF4FEA410C35
:100AF0007FEA6C5C02D150EA013C0AD14FEA430C18
:100B00007FEA6C5C02D152EA033C02D14FF0000054
:100B100070474FF0010070474FEA410212F5001292
:100B200015D211D56FF47873B3EB625212D94FEA34
:100B3000C12343F0004343EA505311F0004F23FA1E
:100B400002F018BF404270474FF00000704750EA73
:100B5000013005D111F0004008BF6FF00040704730
:100B60004FF00000704700BF4A0011D212F500128A
:100B700011D20DD56FF47873B3EB62520ED44FEAF5
:100B8000C12343F0004343EA505323FA02F0704775
:100B90004FF00000704750EA013002D14FF0FF30B3
:100BA00070474FF0000070474FEA4102B2F1E04356
:100BB00024BFB3F5001CDCF1FE5C0DD901F0004C44
:100BC0004FEAC0024CEA5070B2F1004F40EB830094
:100BD00008BF20F00100704711F0804F21D113F1C0
:100BE0003872BCBF01F00040704741F480114FEAF9
:100BF0005252C2F11802C2F1200C10FA0CF320FA82
:100C000002F018BF40F001004FEAC1234FEAD3239E
:100C100003FA0CFC40EA0C0023FA02F34FEA430308
:100C2000CCE77FEA625307D150EA01331EBF4FF091
:100C3000FE4040F44000704701F0004040F0FE40AC
:100C400040F40000704700BF80F0004002E000BFA9
:100C500081F0004142001FBF5FEA410392EA030FA7
:100C60007FEA226C7FEA236C6AD04FEA1262D2EBF1
:100C70001363C1BFD218414048404140B8BF5B42F6
:100C8000192B88BF704710F0004F40F4000020F08F
:100C90007F4018BF404211F0004F41F4000121F0A5
:100CA0007F4118BF494292EA030F3FD0A2F10102EF
:100CB00041FA03FC10EB0C00C3F1200301FA03F12D
:100CC00000F0004302D5494260EB4000B0F5000F50
:100CD00013D3B0F1807F06D340084FEA310102F10F
:100CE0000102FE2A51D2B1F1004F40EBC25008BFC1
:100CF00020F0010040EA03007047490040EB00008B
:100D0000013A28BFB0F5000FEDD2B0FA80FCACF18B
:100D1000080CB2EB0C0200FA0CF0AABF00EBC250B8
:100D200052421843BCBFD0401843704792F0000FA6
:100D300081F4000106BF80F400000132013BB5E7F9
:100D40004FEA41037FEA226C18BF7FEA236C21D06F
:100D500092EA030F04D092F0000F08BF08467047D4
:100D600090EA010F1CBF0020704712F07F4F04D1A2
:100D7000400028BF40F00040704712F100723CBFB5
:100D800000F50000704700F0004343F0FE4040F4DF
:100D9000000070477FEA226216BF08467FEA23639D
:100DA0000146420206BF5FEA412390EA010F40F488
:100DB000800070474FF0000304E000BF10F00043D4
:100DC00048BF40425FEA000C08BF704743F09643BB
:100DD00001464FF000001CE050EA010208BF7047D6
:100DE0004FF000030AE000BF50EA010208BF70475D
:100DF00011F0004302D5404261EB41015FEA010C72
:100E000002BF84460146002043F0B64308BFA3F169
:100E10008053A3F50003BCFA8CF2083AA3EBC2534B
:100E200010DB01FA02FC634400FA02FCC2F120026A
:100E3000BCF1004F20FA02F243EB020008BF20F0A1
:100E40000100704702F1200201FA02FCC2F1200207
:100E500050EA4C0021FA02F243EB020008BF20EAFC
:100E6000DC7070477BB972B90029BEBF00204FF01B
:100E7000004106E008BF00281CBF6FF000414FF0A2
:100E8000FF3000F007BAADF1080C6DE904CE00297F
:100E900009DB002B1ADB00F095F8DDF804E0DDE952
:100EA000022304B07047404261EB4101002B1BDB81
:100EB00000F088F8DDF804E0DDE9022304B04042E8
:100EC00061EB4101524263EB43037047524263EBD3
:100ED000430300F077F8DDF804E0DDE9022304B015
:100EE000404261EB41017047524263EB430300F023
:100EF00069F8DDF804E0DDE9022304B0524263EB57
:100F00004303704753B94AB9002908BF00281CBFE2
:100F10004FF0FF314FF0FF3000F0BCB9ADF1080CDD
:100F20006DE904CE00F04EF8DDF804E0DDE90223BF
:100F300004B07047430803F05533C01A830803F028
:100F4000333300F03330184400EB101000F00F3052
:100F500000EB002000EB0040000E704707EE900A07
:100F6000F5EEC07AF1EE10FA01D400F00BB8F1EE14
:100F7000677A08B517EE900A00F004F8404261EB7A
:100F8000410108BDD0B5FFF7BFFA0C4B0022064661
:100F90000F46FFF711FBFFF7E7FD0446FFF792FA54
:100FA000074B0022FFF708FB02460B463046394646
:100FB000FFF74AF9FFF7D8FD2146D0BD0000F03D0C
:100FC0000000F0412DE9F047089D04468E46002BB5
:100FD0004DD18A42944669D9B2FA82F252B101FAED
:100FE00002F3C2F1200120FA01F10CFA02FC41EAFD
:100FF000030E94404FEA1C48210CBEFBF8F61FFA82
:101000008CF708FB16E341EA034306FB07F199421C
:101010000AD91CEB030306F1FF3080F01F819942CF
:1010200040F21C81023E63445B1AA4B2B3FBF8F0A9
:1010300008FB103344EA034400FB07F7A7420AD930
:101040001CEB040400F1FF3380F00A81A74240F258
:1010500007816444023840EA0640E41B00261DB1C3
:10106000D4400023C5E900433146BDE8F0878B42F8
:1010700009D9002D00F0EF800026C5E900013046B7
:101080003146BDE8F087B3FA83F6002E4AD18B4291
:1010900002D3824200F2F980841A61EB030301203B
:1010A0009E46002DE0D0C5E9004EDDE702B9FFDE27
:1010B000B2FA82F2002A40F09280A1EB0C014FEAD2
:1010C0001C471FFA8CFE0126200CB1FBF7F307FB2F
:1010D000131140EA01410EFB03F0884208D91CEBD2
:1010E000010103F1FF3802D2884200F2CB8043466F
:1010F000091AA4B2B1FBF7F007FB101144EA01444E
:101100000EFB00FEA64508D91CEB040400F1FF31DC
:1011100002D2A64500F2BB800846A4EB0E0440EACA
:1011200003409CE7C6F12007B34022FA07FC4CEAD3
:10113000030C20FA07F401FA06F31C43F9404FEAC6
:101140001C4900FA06F3B1FBF9F8200C1FFA8CFEDB
:1011500009FB181140EA014108FB0EF0884202FA2F
:1011600006F20BD91CEB010108F1FF3A80F08880F0
:10117000884240F28580A8F102086144091AA4B2AD
:10118000B1FBF9F009FB101144EA014100FB0EFE2E
:101190008E4508D91CEB010100F1FF346CD28E455D
:1011A0006AD90238614440EA0840A0FB0294A1EBEE
:1011B0000E01A142C846A64656D353D05DB1B3EB4B
:1011C000080261EB0E0101FA07F722FA06F3F1407B
:1011D0001F43C5E9007100263146BDE8F087C2F122
:1011E0002003D8400CFA02FC21FA03F3914001439A
:1011F0004FEA1C471FFA8CFEB3FBF7F007FB1036D3
:101200000B0C43EA064300FB0EF69E4204FA02F47E
:1012100008D91CEB030300F1FF382FD29E422DD9D1
:10122000023863449B1B89B2B3FBF7F607FB163306
:1012300041EA034106FB0EF38B4208D91CEB010186
:1012400006F1FF3816D28B4214D9023E6144C91A06
:1012500046EA004638E72E46284605E70646E3E616
:101260001846F8E64B45A9D2B9EB020864EB0C0E20
:101270000138A3E74646EAE7204694E74046D1E72F
:10128000D0467BE7023B614432E7304609E76444DD
:10129000023842E7704700BF02E000F000F8FEE7C6
:1012A00072B6374880F30888364880F30988364894
:1012B0003649086040F20000CCF200004EF634716E
:1012C000CEF200010860BFF34F8FBFF36F8F40F283
:1012D0000000C0F2F0004EF68851CEF20001086026
:1012E000BFF34F8FBFF36F8F4FF00000E1EE100A96
:1012F0004EF63C71CEF200010860062080F314889F
:10130000BFF36F8FAAF01CFBABF066FA4FF05530BD
:101310001F491B4A91423CBF41F8040BFAE71D49A3
:10132000184A91423CBF41F8040BFAE71A491B4A9C
:101330001B4B9A423EBF51F8040B42F8040BF8E7EE
:1013400000201849184A91423CBF41F8040BFAE7C3
:10135000AAF0FAFAABF094FA144C154DAC4203DA49
:1013600054F8041B8847F9E702F0BEF8114C124DFF
:10137000AC4203DA54F8041B8847F9E7AAF0E2BA52
:1013800000060020002200200000010808ED00E017
:101390000000002000060020D0340E0800220020AB
:1013A000AC2B0020B02B0020B0400120E001010850
:1013B0003C0201083C0201083C0201082DE9F04F03
:1013C0002DED108AC1F80CD0C3689D46BDEC108A83
:1013D000BDE8F08F002383F311882846A047002042
:1013E000A9F032FAFEE7A9F08FF800DFFEE700006F
:1013F00001F0FF01102A2BDB10F0070F08D010F8C6
:10140000013B013A8B422DD010F0070F42B3F6D1C9
:10141000F0B441EA012141EA014122F007047FF0E2
:1014200000070023F0E80256083C85EA010586EA39
:10143000010685FA47F5A3FA87F586FA47F6A5FA75
:1014400087F68EB9EED1F0BC01F0FF0102F0070281
:1014500032B110F8013B013A83EA010313B1F8D12C
:101460000020704701387047002D06BF354603380D
:10147000073815F0010F07D1013015F4807F02BF46
:10148000013015F4C03F0130F0BC0138704700BF97
:1014900010F8012B11F8013B012A28BF9A42F7D01E
:1014A000D01A7047034613F8012B002AFBD1181AF3
:1014B0000138704738B50022002304460D46FFF777
:1014C000EDFA28B920462946BDE8384000F00AB8B0
:1014D000204605F1004100F005F8404261EB410172
:1014E00038BD00BFD0B50C4B002206460F46FFF7B3
:1014F00063F8FFF739FB0446FEF7E4FF074B0022D1
:10150000FFF75AF802460B4630463946FEF79CFE76
:10151000FFF72AFB2146D0BD0000F03D0000F0415E
:10152000036800221B6818477FB5039140210546D8
:1015300078F034FD039A18B90124204604B070BD38
:10154000134E039296F98231002BF5D05CF0BEFF6A
:10155000437A039A53B95CF0B9FF847A039A2CB9A1
:101560000C4B4021284678F021FDE6E7D6F8D03A2A
:10157000B6F98411B3F906309942DDDD064B0093CC
:101580004021064B284678F011FD0024D5E700BF26
:10159000B84B0020643E0C08833E0C08713E0C08DA
:1015A000F0B50D469DB02021044678F0F7FC0028E8
:1015B00000F09D804F4E96F98231ABB1D6F8D02A1B
:1015C000B6F98431B2F90A1003F10A02914203DD3F
:1015D00040F28D32934207DC474B2A4620212046B9
:1015E00078F0E4FC002080E096F97131022B05D1FF
:1015F000424B2A462021204678F0D8FCB6F84431E8
:10160000A3F57A739BB241F6583293420DD83C4F02
:1016100096ED6C7AD7F83839D3ED097AB4EEE77ADB
:10162000F1EE10FA03DD374BD7E7374BD5E796EDF0
:101630006D7AD3ED0B7AB4EEE77AF1EE10FAF2DCC4
:10164000B6F97E31002B01DC304BC6E796F810224C
:101650000D2A06D80123934013F4215F01D02C4BAF
:10166000BBE72C480EF0B2FD012806D1D7F844099B
:101670007FF064FC98B101281AD00021602204A8F0
:101680000391AEF0F3F82449D7F84009642303AA84
:101690007FF076F800BB03AB0093204B02E0204BB9
:1016A0000093204B2A462021204678F07FFC99E7C2
:1016B00096F8E43A73B11C4819214AF0A5FB48B1E9
:1016C0001948D6F85C6119214AF0C4FB8642D4DD82
:1016D000164BE5E7164BE3E71649D7F838096423BC
:1016E00003AA7BF00DFF0028D5D01DB0F0BD01206E
:1016F000FBE700BFB84B00208C3E0C089F3E0C0857
:10170000B86B0020D73E0C08C73E0C08F13E0C0811
:10171000063F0C08E07C0020803F0C08843F0C084A
:101720004B3F0C08263F0C08C83800206A3F0C08C5
:101730005B3F0C08963F0C0807B5044880F056FF45
:1017400000F0010003B05DF804FB00BFD47400207A
:101750002DE9F043474F0446D7F8940E0368A5B02F
:101760001B690D469847814614F0A0FA0021804677
:1017700060220CA80B91AEF079F864230BAA4946BD
:10178000404613F095FD064648B93B4A0BAB294647
:10179000204678F0EDFD304625B0BDE8F08307F136
:1017A000480066F085F9B9F1000F03D194F91E30B5
:1017B000012B0AD1314811F09FFA80B9304A2946ED
:1017C000204678F0D5FD0026E5E710F0060FE2D0C0
:1017D000A7F5005011F090FA08B92A4AEFE703A9DB
:1017E000404613F09BFB28B19DF80D305B0601D5F8
:1017F000254AE4E7D7ED687AF5EEC07AF1EE10FA03
:101800004FF00003C7DD089309930A930DF12009F7
:1018100007AB019305AA06AB04A9CDF8009040469A
:1018200013F05AFF48462EF063FBD7ED687AB4EE0A
:10183000E70AF1EE10FA01DB144AC0E79DED057AE4
:10184000F4EEC77AF1EE10FA01D8114AB7E79DED30
:10185000047AF4EEC77AF1EE10FA01D80D4AAEE739
:101860009DED067AF4EEC77AF1EE10FA93D80A4AA3
:10187000A5E700BFB84B00209C3F0C08B82B002008
:10188000A53F0C08BC3F0C08E23F0C08F03F0C08D9
:1018900005400C081B400C0831400C0808B5064BED
:1018A00093F8AD3E9B0704D5044A78F061FD002013
:1018B00008BD0120FCE700BFB84B002048400C08E1
:1018C00070B50C4C0546D4F8940E03685B690E465F
:1018D000984710B10124204670BDA4F5005011F0C6
:1018E0001DFA04460028F5D1034A3146284678F00F
:1018F0003FFDF0E7B84B002058400C082DE9F046BA
:10190000464ED6F8B83E93F8CB509BB081468A46F7
:1019100065B9434B1B68986A03685B6B984704463C
:1019200040B9404A5146484678F022FD28461BB04F
:10193000BDE8F0865CF0CAFD20215DF07FFD58B166
:101940005CF0C4FD1F215DF079FD88B3364A514635
:10195000484678F00DFD002496F88A3E03F0140303
:10196000142B05D1314A5146484678F001FD002438
:101970005146484679F08AFB002188424FF06002C8
:1019800002A808BF0C460191ADF070FFD6F8B80E62
:10199000036801AA1B6864219847054680B9244A58
:1019A00001AB5146484678F0E3FC2C462546BDE79E
:1019B0005CF08CFDA5215DF041FD0028C6D1CBE790
:1019C000002CF3D0D9F808303BB9D9F80030514693
:1019D0005B6B484698470446E8E751464846FFF7A0
:1019E000DFFD514607464846FFF758FF3840C4B26E
:1019F00051464846FFF798FD514604404846FFF7D8
:101A00005FFF51460440484678F0DAFC51460440F6
:101A1000484679F053FB0440C8E700BFB84B0020AC
:101A2000E07E00206C400C0883400C089D400C08B0
:101A3000B5400C0808B5FFF761FF054A92F8881E0B
:101A400060F3041182F8881E024A907108BD00BF3D
:101A5000B84B00209D800020F7B505460F4678F072
:101A600041FA044678B10221284678F097FA0646F2
:101A700048B1154880F0BAFDC205C0F30723C0F392
:101A8000002403D53446204603B0F0BD9B07F9D5AA
:101A90000D4880F0B9FD0D4B03F6E803D3ED007A55
:101AA000F8EEE77A30EE670ADFED097AB0EEC00AA9
:101AB000B4EEE70AF1EE10FAE4DD064B3A460221F5
:101AC000284678F073FADEE7D4740020B86B002063
:101AD0000000C842C0400C08F8B504460F4678F034
:101AE0000FFD10210546204678F058FA58B12046DF
:101AF000FFF722FE064630B9044B3A461021204635
:101B000078F054FA35462846F8BD00BFD4400C089A
:101B100070B505460E4678F0E5F9044678B18021A7
:101B2000284678F03BFA50B1074B93F80D3443B197
:101B3000064B32468021284678F038FA00242046A9
:101B400070BD0446FBE700BFB85B0020E8400C080E
:101B500038B50D4D0446D5F844097FF0EFF901285A
:101B600010D0D5F844097FF0E9F9022804D02046C6
:101B7000BDE8384078F0B8B904480EF027FB0128DA
:101B8000F5D138BD0020FCE7B86B0020E07C0020D8
:101B9000F0B5114C85B0D4F8C83A0093D4F8CC3ADB
:101BA0000193D4F8D03A02936A46D4F8D43A039316
:101BB00006460F4679F01CFA39460546304678F05D
:101BC00029FA94F8883E284060F3C303C3F3C000A9
:101BD00084F8883E05B0F0BDB84B00202DE9F843ED
:101BE00006462648DFF8A480DFF8A4900F4665F08B
:101BF0005FFF0446D8F8940E03681B6998470546B2
:101C000030B914F0060F03D1D8F8C83E022B09D121
:101C10003946304678F0D0FA054618B9002489F8DC
:101C200007400AE039463046FFF792FD0446002897
:101C3000F4D02DB9012389F807302046BDE8F88398
:101C40000821304678F0AAF90028F3D00C4821F09A
:101C500049FE0028EED00B4B93F8E423B02101FBA2
:101C60000233B3F8EE21B8F972319A42E2DD064B45
:101C70003A460821304678F099F9CFE7004C002029
:101C8000D82C0020B82B0020FC400C08B84B0020BA
:101C90009D8000202DE9F3410F46054614F006F81B
:101CA000804613F0FDF8044640B94F4A012128460A
:101CB00078F05EFB204602B0BDE8F0814B4ED6F8CE
:101CC000940E036839469B699847044658B9D6F87C
:101CD000940E03681B6C9847454A03460121284629
:101CE00078F046FBE6E7AB68002BE3D010212846EE
:101CF00078F054F910B3D8ED937A98ED920A20EE6B
:101D0000270AABF051FBDFED3B7AB6F9443120EE08
:101D1000270ADFED397A20EE270A07EE903AF8EE2F
:101D2000E77AB4EEE70AF1EE10FA07DD334B012251
:101D30001021284678F03AF90024BBE740212846D4
:101D400078F02CF928B3012F1CD0232F1AD0042FA0
:101D500018D0D6F8D03A2A48B3F9083000EE103A35
:101D6000B8EEC00A00F0BEFBB5EEC00AF1EE10FA04
:101D70001DDD244B00930122234B4021284678F09F
:101D800015F9D9E7D6F8940E0368DB6B984700285D
:101D9000DFD01E4B1B68D86A0368DB6998470128AF
:101DA000014619D11A4A284678F0E2FAC4E7D6F873
:101DB000940E03685B69984730B1D6F8D03AB3F90E
:101DC0000830002BE5DDD4E7D6F8940E03681B68D5
:101DD00098470B28DDD1F0E73946284602B0BDE828
:101DE000F04178F055BE00BF0C410C08B84B002004
:101DF0001D410C08E02E65420000C84231410C082C
:101E0000B82B0020833E0C0839410C08E07E0020EE
:101E100045410C0870B505460E46FFF799FC084B86
:101E20000446D87131462846FFF74AFD314600285E
:101E3000284608BF002478F0C3FF204070BD00BFD3
:101E40009D800020F8B54E4F3B78002B40F09580E8
:101E50004C4CD4F8B85E95F8CB5001263E7015B1C5
:101E60003B702846F8BD79F0D1F9054630B9464AAD
:101E70003870137843F001031370F2E752F06CF9F5
:101E8000314651F0A3FAA4F5005006F07FFC3F4B19
:101E90001E710B2645F018FF013E45F0B3FE16F00B
:101EA000FF06F7D13A4800F069FF13F0FFFED0F8C3
:101EB0000022C4F8E02E90F87C32DA074BD413F0FD
:101EC0006DFA52F049F93C2152F082F804F56A6348
:101ED00000221A6000212E4800F0E4FF2C4810F088
:101EE0000BFF01462B4884F0F3FA2B4B1B68D86A92
:101EF000036801211B689847D4F8B80E03689B6AF1
:101F000098470121D4F8B80E81F02AFB52F024F949
:101F10000646D4F8940E03681B68984794F8042189
:101F20000146304651F02AFC194806F021FC4FF0DA
:101F300039FB4EF075FE00233B7088F01BFD174BFC
:101F4000C3F85009B4F88A3E23F4087343F0200321
:101F5000A4F88A3E85E79B07BCD431460C4804F0C0
:101F6000D5FC0F4880F050FBDFED0E7A20EE270AFB
:101F700004F56A6383ED000AACE7002571E700BF52
:101F8000B02B0020B84B0020BC8000209D8000209A
:101F9000B82B002024550020E07E0020B86B0020E4
:101FA000D47400200AD7233C2DE9F043374DD5F8EF
:101FB000B83E93F8CB3087B0002B64D062B10129D2
:101FC00001D0232908D195F9883E002B04DB002499
:101FD000204607B0BDE8F08379F0C4F90446002834
:101FE000F5D013F063FE07461AF0AEFA8046384685
:101FF00012F068FCD8B198F92430022B17D10026D2
:102000004FF00009F1B203AA38460191CDF80C90C7
:10201000CDF81090CDF8149012F0E6FF019918B1A8
:1020200003AA404619F040FF0136032EEAD11848B2
:10203000012106F015FE1648012106F047FD00219A
:10204000D5F8B80E81F08CFA124830F035FC52F019
:1020500083F8002151F0BAF90F4B1B68D86A036866
:1020600000211B68984795F88A3ED5F8941E0B48C6
:102070006FF3451385F88A3E0B1A594259413C309B
:1020800086F08AFEA4E70124A2E700BFB84B002037
:10209000B82B002014770020E07E0020B0780020CC
:1020A00010B5064CD4F8940E03685B6A984718B1D3
:1020B000D4F8B83E93F8CB0010BD00BFB84B002059
:1020C00030B52DED028B89B00C46B0EE408AFFF79B
:1020D000E7FF0546002838D0B4EE488AF1EE10FA42
:1020E0007CBFDFED1C8ADFED1C7A226863689FED00
:1020F0001A0A68BFDFED198A029278BF68EE288A53
:1021000002A878BF68EEA78AD4ED027A0393F1EEB5
:10211000677ACDED047A2DF0EDFAB4EE488A00220C
:102120000123F1EE10FACDE900238DED050ACDED86
:10213000060A9FED0A0A0A488DED071AF0EE680AB2
:1021400068BF134605A90CF027F9284609B0BDEC75
:10215000028B30BDE02E65420000C8420000000046
:10216000847B002007B50191FFF79AFF30B10199F8
:10217000044803B05DF804EB00F0F2BA03B05DF878
:1021800004FB00BFB82B0020014865F01DBE00BF56
:10219000004C002008B500F5005090F8883EC3F3CD
:1021A00040128A420BD061F3451380F8883E31B16A
:1021B00051F0D2FFBDE808400F2151F009BF08BD22
:1021C00070B500F500560546D6F8C83E8B420C4661
:1021D00012D0012911D0022916D059B951F0BCFFF3
:1021E0001B2151F0F5FE0D4A05F5315006212C302A
:1021F00054F052F8C6F8C84E70BD51F0ADFF1A2128
:1022000051F0E6FE064AEFE7012100F04BFE51F0E7
:10221000A3FF1D2151F0DCFE024AE5E7B0410C08A6
:10222000C5410C08C0410C0810B500F500520C4621
:1022300092F8AD3E03F00101A14209D064F300031E
:1022400082F8AD3EDB0704D405F088FE024B9C7299
:1022500010BD06F05BF8F9E79D80002000F5005006
:1022600090F8AD3E61F3410380F8AD3E014B197328
:10227000704700BF9D80002010B504465CF026F931
:1022800020215DF0DBF804F50053003893F88A2E26
:1022900018BF012060F3820283F88A2E10BD00006F
:1022A00010B504464FF07EF904F50052436FD2F8A2
:1022B000B82E04F58044D360D4F838299366D4F856
:1022C0004029C2F8FC32D4F8380903685B6D98479E
:1022D000D4F838090368BDE810409B6D184700002A
:1022E00070B52DED028B00F500550446D5F8B83ECB
:1022F00093F8CB30002B72D095F9883E002B6EDB23
:1023000000F5804696F8803A002B68D1D5F8940EF7
:1023100003685B699847002861D1324BD3F8940E6B
:1023200003681B6898470B2859D0D6F840399FEDB1
:102330002E7AD3EDDB7AF0EEE77AF4EEC77AF1EE9F
:1023400010FA4CD5D5F8B80E443053F037FB03469D
:10235000DFED260A93ED000A9F20B7EE001A29F060
:10236000C5FFB5EEC00AF1EE10FA38DD04F5924073
:102370001C3080F055F9DFED1E7AB0EEC00AB4EEE5
:10238000E70AF1EE10FA2AD504F58054D6F8380998
:10239000D4F8603407EE903A0368D3F89830B8EE7A
:1023A000E78A984738EE400ADFED127AB0EEC00AAD
:1023B000B4EEE70AF1EE10FA11D5D4F8643440F225
:1023C000E63203F2F313934209D8BDEC028BD5F841
:1023D000B80E9FED090ABDE8704082F0ABBBBDECC2
:1023E000028B70BDB84B00200000003400000000DC
:1023F000000070420000FA430AD7233C08B500F5FC
:102400000050D0F8B80E03681B699847F6EE007AC2
:1024100020EE270AB5EEC00AF1EE10FA48BF9FED94
:10242000010A08BD0000000038B52DED028B00F553
:1024300080450446D5F83839DFED110A93ED370AA7
:1024400004F500547120B7EE001A29F04FFFD4F8BC
:10245000B80ED5F8405903681B69B0EE408A98471A
:1024600038EE400ABDEC028BDFED067A05F5057506
:10247000284620EE270ABDE838406FF095BE00BF21
:102480000000000000007A4400F5805000F59763DA
:1024900000F2C440D3ED005AD2ED007AD0ED006ACC
:1024A00091ED006A26EEE77A67EEA57AA6EE257A28
:1024B000E6EE267A81ED007AC2ED007A70470000E0
:1024C00000F50050B0F91C3A33B9B0F97E0100288C
:1024D000B8BF404280B2704783EAE370A0EBE3707C
:1024E000F8E7000070B52DED028B00F5005482B0C6
:1024F00094F8AD1E11F00106054605D09FED2D0A9A
:1025000002B0BDEC028B70BD8DED010A5BF0DEFF09
:10251000037F002BF2D0DFED288ADFED260A9DED48
:10252000010AB0EE681A4E2029F0E0FE4FF4C8729E
:102530003146B4F98601B0EE408A29F015FFA4F8BF
:102540008601284610F08AF9B4F9863107EE900A20
:10255000B8EEE77A07EE903AF8EEE77A77EE676A38
:10256000B4EEE68AF1EE10FA0DD52846FFF7A8FF83
:1025700007EE900A38EE668AB8EEE70A20EE088A7F
:1025800088EE260ABCE777EE877AB4EEE78AF1EEAA
:1025900010FAB3DDB4F97E3100EE103A38EE678AF6
:1025A000B8EEC00A78EEE77A20EE088A88EE270AAD
:1025B000A6E700BF0000000000007A44002070473A
:1025C000002070477047000000F506501430704737
:1025D000004870475C710C0800F50050D0F8940E6C
:1025E00003681B6818470000034808602F2111701A
:1025F00008221A60704700BF60450C0800F50050C3
:10260000D0F8940E0368DB6C1847000000F500500A
:10261000D0F8940E03689B6C1847000000F5005337
:1026200000F59640D3F8943E20301B1A584258418A
:102630007047000010B500F500500C46D0F8940E1D
:102640000368DB6D984707EE900A9FED057AF8EE78
:10265000677A012067EE877AC4ED007A10BD00BF6B
:102660000AD7233C10B500F500500C46D0F8940E64
:1026700003689B6D984707EE900A9FED057AF8EE88
:10268000E77A012067EE877AC4ED007A10BD00BFBB
:102690000AD7233C10B500F500500C46D0F8940E34
:1026A00003681B6E9847DFED047A20EE270A0120AD
:1026B00084ED000A10BD00BF0AD7233C5EF038BB92
:1026C00062F062BB5DF0DABE4EF0B6BE27F048BDE8
:1026D00050F0FABF17F01AB85BF04ABB59F004BDCE
:1026E0000FF06ABD10F0AAB906F0ECBC11F0AAB95F
:1026F00005F08ABC05F0DCB905F002B960F098B8C5
:102700000EF000BCFFF7ECBD0FF08EBE10F0F4B879
:1027100003F074B80FF016BE0FF094BD5BF024BE4A
:1027200022F07EBB06F09EB802F03EBC10F002B96B
:1027300006F07EBC04F0D6B806F0D8BD05F072B93C
:1027400006F03EB90FF0C4BCFFF7AABD28F026B8CA
:1027500005F05ABE09F080BE09F07ABD09F00EBD41
:102760001FB500F500530446D3F8940E0391036897
:102770005B6A984760B1DFED070A0399002304F50F
:102780009F400093B0EE600A1A464C300BF05AFCA2
:1027900004B010BD0000000010B52DED028B00F557
:1027A00000530446D3F8940E03685B6AB0EE408A87
:1027B000984720B90024BDEC028B204610BD9FED48
:1027C000080A04F59F4028EE000A4C300AF004FF86
:1027D00004460028EED003480121FFF7DBFCEAE7BE
:1027E0000000C842B82B00200A4A92F9882E002A1D
:1027F0000B4605DA00228A604A600A6001207047B1
:1028000000F58040D0F83829783207CA83E80700FD
:10281000F4E700BFB84B002070B51F4B036000F514
:1028200000530446D3F81C0E1C4AC3F86C2C08B1A4
:1028300019F0C2F81A4B236004F5805393F82C2E3C
:1028400042B9D3F8285E2DB1284626F091FA2846E1
:1028500019F0AEF804F58B50103076F0D3FE04F585
:10286000835018305EF03EF804F6C44504F6644622
:10287000B54204D0183D284625F0CEFEF8E7094BB6
:10288000C4F8983804F6941052F074FD04F5106002
:1028900052F070FD204670BD1C490C080C4D0D080F
:1028A000D42D0D0898F60C0838B5484B044640F86E
:1028B000043B5EF05DFB04F1100016F0C9FB04F16F
:1028C00068004EF047FB04F5907020F033FF04F5EC
:1028D000866015F049FA04F2545019F06FF804F6C6
:1028E000980027F0E1FA04F544605EF01FF904F562
:1028F000516049F0AFF904F57C6050F0C7FC04F575
:10290000835018305DF0D6FF04F58550143017F071
:102910009BFE04F58B50103076F060FE04F58C5071
:102920000C304EF0D9FE04F58F505FF0CBFC04F56F
:1029300080530025264A83F8045204F5905004F58C
:10294000905304331430136044F0D0FF04F59350D7
:102950002946083011F0A6FC04F5C55018306FF078
:10296000E1FC04F5E5501C3073F07EFE04F5EE50FA
:10297000143075F08DFF04F5F150183076F0C2FB7D
:1029800004F5F450103011F08FFA04F5FF501030B8
:1029900070F07EF904F50150083064F02DFF04F565
:1029A000005304F5045083F804510A4D1C3077F0AD
:1029B000E9F92B6813B1084887F0AAFF20460749B8
:1029C00047F038FF2C60204638BD00BFD42D0D08DD
:1029D000148A002078810020D4410C08FC2C0D08BA
:1029E00010B50FF0B5FE5BF071FD0368BDE8104057
:1029F0005B681847FFF7F4BF10B5044606F07EF891
:102A0000204610F0A3F9204603F0B6FD2046BDE8AD
:102A1000104003F01DBF0000FFF7EEBF70B500F5DA
:102A20003B5524350446284616F0ECF919F08CFD88
:102A300090F9213093B390F840337BB304F5005301
:102A400004F25456D3F8B80E443052F0B7FF0346A0
:102A5000DFED130A93ED000A9F20B7EE001A29F06C
:102A600045FC94F98835012B284608BF86ED0E0AEF
:102A7000002115F08DFFDFED0B7A04F2AC7494EDBC
:102A8000287A20EE270ADFED087AA7EE270A3046DB
:102A900084ED280ABDE8704019F066BC70BD00BF27
:102AA00000000000CDCCCC3D6666663FFFF7B6BFA8
:102AB00010B50121044610F085F960B1114BD3F82F
:102AC000940E03689B6A984728B9204602F07AF969
:102AD000204602F087F94FF40011204610F072F9F9
:102AE00018B128F0D5FE27F0BBF84FF4802120461E
:102AF00010F068F928B128F0CBFEBDE8104026F0B0
:102B0000BDBF10BDB84B0020FFF7D2BF70B500F5B8
:102B100080450446D5F838099FED540A86B06C30DC
:102B20002CF0E8FD04F5935003A908308DED030A5D
:102B3000CDED040A8DED051A11F060FA0221204650
:102B400010F040F970B10121204610F03BF948B96E
:102B5000474BD3F8940E03689B6A984710B92046F8
:102B600002F030F90121204610F02CF948B9404B11
:102B7000D3F8940E03689B6A984710B9204602F078
:102B800031F90121204610F01DF910B9204602F05C
:102B900081F94FF40031204610F014F930B104F5FA
:102BA0000053D3F8B80E03685B6C98474021204669
:102BB00010F008F960B104F57C6001904FF024FF3B
:102BC00004F58053019893F978300BB150F05EF81A
:102BD0004FF48061204610F0F5F818B104F57C60E0
:102BE0004FF0ACFF2021204610F0ECF858B104F56E
:102BF0000056D6F8940E03681B699847C0B1D5F803
:102C000040097CF0F9FC8021204610F0DBF8E0B1AF
:102C100028F03EFE26F056FF1021204610F0D2F894
:102C200010B3D5F8380906B0BDE8704079F02ABA7B
:102C300020460CF0BFF80028E1D1D6F8940E0368C6
:102C40005B6998470028DAD0DDE74FF48021204601
:102C500010F0B8F80028DBD14FF40021204610F026
:102C6000B1F80028D4D1D7E706B070BDE02E654298
:102C7000B84B0020FFF74ABF10B50121044610F001
:102C8000A1F810B1204602F005F98021204610F08D
:102C900099F858B14FF48021204610F093F828B9E4
:102CA00028F0F6FDBDE8104026F0E8BE10BD00009B
:102CB000FFF7E2BF10B5044605F074FC204605F0AE
:102CC000D7FA204605F0B2FC204610F027FF204638
:102CD000BDE8104003F02CBCFFF7ECBF70B54FF619
:102CE000FF71044610F06EF804F5005528B1D5F8D0
:102CF000882E0721204602F0FDF8D5F8B83E93F85B
:102D0000CB307BB92046FFF7B7FAD5F8B80E95F867
:102D10009A21036895F810121B6A9847D5F8B80EE7
:102D200081F0D4FE5DF0D4F85CF060FE204610F037
:102D3000F3FE95F8883E0F4A04F58044DB43D4F84F
:102D40003859C3F3C01353712B681E6F4EF02AFC21
:102D50004EF092F82846B047D4F840494EF022FC95
:102D600004F505744EF088F82046BDE870406FF019
:102D700081B800BF9D800020FFF7B0BF2DE9F04172
:102D800000F5805600F5005406F5976304F6CC680C
:102D90001B68C8F8003006F2C44304F56D671B6871
:102DA0003B600546D6F8680400F58C40503029F0A9
:102DB00071FA04F6D863C4F8D40ED8F800201A606B
:102DC00004F6DC643B6823604FF6FF7128460FF081
:102DD000F9FF38B1D6F8682428460921BDE8F0414A
:102DE00002F060B8BDE8F08110B500F50053D3F8EB
:102DF000C84E002C55D093F8892ED10751D56FF3CA
:102E0000000283F8892ED3F8CC2AD3F8C81AB2F975
:102E10000820012C06EE902AB1F908400BBF03F6FA
:102E2000CC6203F6D862D2ED007AD2ED007A0CBF04
:102E300003F56D6203F6DC62D2ED005A0CBFF8EECA
:102E4000E66AF8EEE66A07EE104A25EEE66AB8EEA4
:102E5000C77A00F58050A7EE276A00F5976200F266
:102E6000C44067EEA67AD2ED006AE7EE257A90EDCF
:102E7000007A27EE877AA6EE267ABDEEC77A17EE9D
:102E8000104A0C8192ED007AD3F8CC3A67EE877A3B
:102E900090ED007AE6EE477AFDEEE77A17EE902A9B
:102EA0001A8110BD38B505462DED028B00F5005492
:102EB00071B128460FF0DAFAD4F8D43E1B1A03F2A7
:102EC000F31340F2E63293420CD8BDEC028B38BDCE
:102ED000D4F8C83E022BF8D10FF0AAFAB0F57A7FE9
:102EE000E7D2F2E7C4F8D40E00F58C4050306423EA
:102EF00090FBF3F308EE103ADFED0B7AB8EEC88AD8
:102F000028EE278AB0EE480AAAF094F804F6D863AF
:102F100083ED000AB0EE480AAAF0E2F904F6DC6498
:102F200084ED000AD1E700BF35FA8E3C00F59350DE
:102F30000121083012F02CBEFFF7F8BF10B504468F
:102F40000FF092FC102120460FF03CFF70B120469C
:102F500001F092FE4FF4001120460FF033FF28B924
:102F600028F096FCBDE8104026F07ABE10BD0000A7
:102F7000FFF7E4BFF8B50446254606F0DFF8224B1C
:102F800045F83C3B214BA465C4E91734204BC4E908
:102F90001934204BE36604F1800018F0A1F904F124
:102FA0009C0018F09DF904F1B80018F099F94FF65B
:102FB000FF76194BC4F8CC30A4F8D06004F1D400EB
:102FC00018F08EF94FF0FF37144B1549C4F83071E3
:102FD00028461D6047F02EFCA4F87870A4F8946091
:102FE00004F5A27018F07CF904F5B07018F078F9C7
:102FF00004F5BE7018F074F9002384F89031C4F819
:10300000B4312046F8BD00BFC09C0C08552701080C
:10301000592701085D2701080000FFFF6C80002090
:1030200058040D0810B5044606F088F80A4B2360D2
:103030000123A38704F1400018F052F904F1500075
:1030400018F04EF904F1600018F04AF904F170002C
:1030500018F046F9204610BD68A40C082DE9F0438D
:10306000044689B0FFF720FCA24B236004F506500C
:103070003C3004F5005502F071F804F506530833AE
:1030800004F52B57C5F8DC3A062385F8E03A4FF0F3
:103090007C5805A907F12C00CDF8148052F024FDCE
:1030A00007F1440086F01CFE04F5924600231C360E
:1030B00004F52C5785F81C3B192304A985F8283BF7
:1030C000C5F8246B07F13400CDF8108052F00CFDE8
:1030D00007F14C0086F004FE4FF00108182304F5B8
:1030E0002E5004F52F5785F8703B2C3785F8648BEC
:1030F000C5F86C6B04305CF0EFFF384676F0FEFEEE
:1031000006AE7D4BC5F8EC3B3146381D8DF8188076
:1031100048F0A6F904F53050243076F0D9FE774B0C
:10312000774FC5F8243C04F5305031463C300697C3
:1031300052F0DAFC04F5315031460830069752F06F
:10314000D3FC04F531503146143004F5315806975C
:1031500008F12C0852F0C8FC6A4BC5F86C3C08F129
:10316000080086F0BDFD04F5325704F533591837D1
:1031700009F13C093846143757F0CEF94F45F9D1DB
:103180000723C5F8203E0023A5F8243E4FF4CB705A
:1031900018F00CFCC5F81C0E04F53850283086F0E9
:1031A0009FFD04F539502C3086F09AFD564B1A6875
:1031B0000AB9C3F8008004F5A347544BC5F86C3C2A
:1031C000343704F53A50C5F8947E183078F0EAF8B0
:1031D00005F6CC634FF07E58C3F8008005F6D8653D
:1031E0004B4B07934B4BC5F800800694009304F5B6
:1031F0003B5096E80C004FF40071243015F09AFA19
:1032000004F55050103068F083FA04F5914003A99A
:103210006C30CDF80C8052F08DFC03A904F592407F
:10322000CDF80C8052F060FC04F5924004F5804526
:103230000C3018F055F805F61C1300261E605E6071
:103240009E6005F6281304F592401E605E609E6045
:1032500004F593530833C5F83439002385F85539FC
:103260004FF40041583015F0D7FF04F59340583023
:1032700066F0DCFB04F59440143048F027FA264B46
:10328000C5F8143A04F59440244B2549283004F538
:103290009448186008F1480847F0CCFAFF2385F8F5
:1032A000583A85F8603A1F49404647F0C3FA1E4A2B
:1032B000136813B11D4887F02BFB1D491D48C2F848
:1032C000008004F59442703208604FF0140E1FFA2B
:1032D00083FC0EFB0C010133097C0029F7D1164B4E
:1032E000A3F800C0154BD3F80080B8F1000F29D027
:1032F0001348E0E71C490C085C410C089C410C0891
:103300000000A0400C4D0D08948400209C490C083E
:10331000512701080C490C08AC410C08188A002000
:1033200080590D0858B50D08A88A0020E8410C08FE
:1033300038810020508B0C0834810020F48000205C
:1033400009420C0804F595401A6003A9554B0393F4
:10335000043052F0C9FB04F59540243005F0EEFE30
:10336000514BC5F8A43A04F59540643005F0E6FEEB
:1033700004F599494D4BC5F8E43A04F5964009F136
:1033800078092030FFF7F6FD484605F0D7FE484B98
:10339000C5F8F83C09F13C0084F086F9454BC5F8C6
:1033A000343D04F59D40383005F0C8FE424BC5F869
:1033B000B83E04F59D407C3005F0C0FE3F4BC5F89B
:1033C000FC3E04F59E4085F8388F3C3005F0B6FE93
:1033D0003B4BC5F83C3F04F59E40783005F0AEFE0F
:1033E000384BC5F8783F05F6B47304F59F401E606E
:1033F0005E609E604C3005F0A1FE334BC5F8CC3FBB
:1034000004F5A0452846C5F80880103005F096FE62
:103410002E4B2B612846583005F090FE2C4BAB65A7
:1034200004F5A140143005F089FE2A4BC5F894300C
:1034300004F5A240C5F80C61C5F810612830FFF70B
:10344000F1FD384605F07AFE234BC5F8B43104F59A
:10345000A340703005F072FE204BC5F8F03104F542
:10346000A440A5F82C824030FFF7DCFD1C4BC5F8CA
:10347000403204F5A540012385F8C932C5F8D06271
:10348000C5F8D462C5F8D8625C3005F057FE154B1C
:10349000C5F8DC322046C5F81C63C5F8206309B0C6
:1034A000BDE8F083CDCC4C3DBC990C08609A0C086B
:1034B000649D0C08F49D0C08B09E0C08509F0C08ED
:1034C000F09F0C0888A00C0828A10C08B8A10C08D3
:1034D00050A20C08F0A20C08C4A50C0860A70C08A8
:1034E00020A50C0824A80C0838B5054B1C682368D7
:1034F0000A461D68034B01462046A847002038BDF8
:10350000E07E0020B82B002010B586F05FFE064C50
:10351000064B18602046FFF7A1FD2046044A0549E6
:10352000BDE81040A9F060BCB82B0020E07E002070
:1035300034DC0020192801080120704790F89030F1
:103540008B4286BF00EB8100D0F8940000207047CA
:1035500090F890308B4286BF00EB8100D0F8940049
:1035600000207047FA207047014B93F84A017047DA
:10357000B84B0020034BD3F8C80E431E58425841A5
:10358000704700BFB84B0020034BD3F8C80E831E12
:1035900058425841704700BFB84B0020034BD3F846
:1035A000B80E08B180F0D4B801487047B84B00207D
:1035B00088490C0870B5036A2E4D43F4E05202624C
:1035C000426A42F4E0524262826A42F4E05282620B
:1035D000D5F840290446E2B143F4F8430362D5F834
:1035E00040097BF0C9FB38B1636A43F480436362EE
:1035F000A36A43F48043A362D5F840097BF0DEFC64
:1036000038B1636A43F400536362A36A43F400531E
:10361000A362194B1D6845B11921284648F0F4FBF7
:1036200018B1236A43F480732362144E96F8E43A87
:103630006BB1636A43F48073636245B11921284614
:1036400048F01AFC18B1A36A43F48073A362236A9A
:1036500043F080432362636A43F080436362D6F899
:10366000B83E93F8C1301BB9A36A43F08043A3620C
:1036700070BD00BFB86B002044810020B84B002013
:1036800013B54FF44470CDE9002118F089F90446D0
:1036900028B1DDE9002159F075FC024B236020467A
:1036A00002B010BDDC4B0C080020704770470000D2
:1036B0000320704708207047014B93F84C01704776
:1036C000B84B0020034B93F90402003818BF0120C7
:1036D000704700BFB84B0020014B93F94E01704773
:1036E000B84B0020704700007047000008B50C4B35
:1036F000D3F8400970B910230A4AD2F8B82E43F023
:10370000400022B192F8CB200AB143F0C00040F053
:10371000010008BD7BF030FB0028ECD01823EBE75C
:10372000B86B0020B84B002038B5C5780B46352D56
:10373000044628BF3525352200211846ACF096F8FE
:103740002A4604F10C01BDE83840ACF045B8000051
:103750001FB5184C94F8DE1F04F5696010F090FB5B
:1037600078B194F8DE1F04F5696010F08BFB40B16E
:1037700094F8DE1F04F5696004B0BDE8104010F055
:1037800083BB002301930293039312F08FFA01A9E4
:1037900012F066F820B101A82CF0AAFB04B010BD0D
:1037A00021F07CFB90F8C432B02202FB030090EDC4
:1037B0002F0AF3E7B83B002008B50D4BD3F8B80E3D
:1037C000A8B1443052F0FAF8034693ED000ADFED59
:1037D000090A9F20B7EE001A28F088FDDFED067A6F
:1037E00020EE270ABDEEC00A10EE103A18B208BD4E
:1037F000B84B0020000000000000C8422DE9F04F47
:10380000DFF8D880344F8DB00446042508F5005603
:1038100017F8019BB8F9A43109F1FF3A43FA0AF30A
:10382000D90742D5207C53F0C5FC8346207C54F058
:10383000C5FB00F121039B4505D2207C0DB0BDE8FE
:10384000F04F52F033BFBAF1030F2ED8DFE80AF081
:103850000234393ED6F8380903689B68984700F16E
:1038600094035A69D3F800A0D3F804E0D868196922
:10387000D3F818C008925A6A1B6ACDF82520CDF8F3
:10388000293062222123CDE9003206900791207C65
:10389000CDF80CA0192303AAC221CDF810E0CDF871
:1038A00014C08DF8249053F0EFFC013D15F0FF0596
:1038B000AED10DB0BDE8F08FD6F838090368DB68EB
:1038C000CCE7D6F8380903681B69C7E7D6F8403952
:1038D00003F52A73C5E700BFA84C0C08B84B0020BD
:1038E00013B504460748019108F0FAFB30B9019975
:1038F000204602B0BDE8104054F084BD042002B060
:1039000010BD00BFD8760020014808F043BA00BFC0
:10391000D876002058F096BA10B588B0044655F015
:10392000FDFE0C4BD3F8B80E38B90B4A06212046E1
:1039300008B0BDE8104055F0D9BE69461E227FF0A0
:103940000BFF064A6B460621204655F0CFFE08B015
:1039500010BD00BFB84B0020D4490C0832970C08AA
:10396000034A92F8C43A013382F8C43A54F0DABFF9
:10397000B84B002007B50846019117F087FD38B114
:103980000448019902F086FC002003B05DF804FBB6
:103990000420FAE7EC7E0020162A10B40C4605D06D
:1039A000542A03D05DF8044B54F04ABD032323701E
:1039B00001205DF8044B704708B554F0E7FE40F471
:1039C0001C6040F00D0008BD10B5044617F0F0FF74
:1039D000204610BD10B50C4C94F9883E002B0FDB2F
:1039E000D4F8940E0368DB6C984758B9D4F8940E59
:1039F00003689B6C984700280CBF0220032010BD71
:103A00000120FCE70420FAE7B84B002010B44C6911
:103A1000012C05D101465DF8044B034802F0BEBFFE
:103A20005DF8044B54F098BFB82B00202DE9F3410A
:103A3000B1F90430002B06460C46154635DB4FF035
:103A40000008CDE900281A4FB1F902209FED190AAC
:103A5000D7F8C81A4FF47A7358F0CEFC0123CDE999
:103A600000539FED140AB4F90020D7F8CC1A4FF494
:103A70007A73304658F0C0FC9FED0F0AB4F9042069
:103A8000D7F8D01A43463046CDE9005858F0B4FC78
:103A9000CDE900589FED070AB4F90620D7F8D41AEB
:103AA0004FF47A73304658F0A7FC02B0BDE8F081BD
:103AB000B84B00200000FA4400007A44044B187808
:103AC00020B9044B93F88A0EC0F38010704700BFF2
:103AD0003C800020B84B00200C4B93F80D248AB991
:103AE000A3F5805393F8AD2E92060BD193F9882E4F
:103AF000002A09DB93F8893E13F0200F14BF04203D
:103B0000012070470520704703207047B85B0020F4
:103B100008B5074B93F99831032B03D0BDE8084053
:103B200055F05CBE034A022155F0E0FD042008BDBB
:103B3000B84B0020EC490C08094BD3F80822920737
:103B400001D454F06FBC03F5005303F5116393EDFA
:103B5000000ADFED047AB8EEC00A20EE270A7047AB
:103B6000B84B00200AD7233C10B594B0044603A8F4
:103B700017F0B6FB1C4BD3F8940E036803A95B6DDA
:103B8000984778B3002103A817F042FC50B3247C77
:103B900086F0F0FE059BDDED047A0893069B099301
:103BA0000023F8EEE77A9FED117A0B930C930D93B7
:103BB0000E930F931093119312934FF6F853ADF8A1
:103BC0004C300023962267EE877A8DF84E303323EF
:103BD000CDE90032079007AA57212046CDED0A7A99
:103BE00053F052FB14B010BDB84B00200AD7233C51
:103BF00030B52DED0A8B764C0546D4F8940E03684B
:103C000099B05B6A984700285AD004F54054A368DD
:103C1000062B00F2C980DFE803F00404045788ABE8
:103C200053006C489FED6C8A0AF0D4FB9FED6B0A41
:103C30000168426883680D930BA80B910C922BF0DE
:103C400059FDF0EE489AB0EE40CAF0EE60BAB0EE20
:103C5000419AB0EE48AAF0EE488AF0EE48AAB0EEDB
:103C600048BA40F6F8542D7C86F084FE0023159364
:103C7000169301238C228DF85E303323CDE9003278
:103C80000B90B1EE499AF1EE688AB1EE488A0BAA20
:103C9000552128468DED0CCACDED0DBA8DED0E9A4D
:103CA0008DED0FBACDED10AACDED118A8DED12AAD2
:103CB000CDED139A8DED148AADF85C4053F0E4FA23
:103CC00019B0BDEC0A8B30BD42480AF083FB9FED72
:103CD000430A0168426883680D930BA80B910C920C
:103CE0002BF008FD3B48F0EE60BAB0EE419AB0EE22
:103CF00040CA0AF073FB9FED390A2BF0FBFC3548F4
:103D0000B0EE40BAF0EE60AAF0EE418A0AF06AFB2B
:103D10009FED320A2BF0EEFC4FF44064B0EE40AA67
:103D2000F0EE609AB0EE418A9DE72A489FED2A9A0C
:103D30000AF054FB9FED290A2BF0DCFC2548B0EE7D
:103D400040BAF0EE60AAF0EE418A0AF04BFB9FED1C
:103D5000230A2BF0CFFCF0EE49BAB0EE40AAF0EE09
:103D6000609AB0EE418AB0EE49CA40F607447AE75D
:103D70001848DFED198A0AF035FB9FED180A2BF081
:103D8000B9FCF0EE68AAB0EE40AAF0EE609AB0EE90
:103D9000418AB0EE68BAB0EE689AF0EE68BAB0EE5A
:103DA00068CA40F63F445EE79FED0B8A0024F0EEC0
:103DB000489AB0EE48AAF0EE488AF0EE48AAB0EE73
:103DC00048BAB0EE489AF0EE48BAB0EE48CA4AE7B0
:103DD000B84B0020847B0020000000000AD7233C61
:103DE0002DE9F0412DED068B3B4D95F8893E990666
:103DF0008CB004466AD505F500579FED380AD7F810
:103E00003809DFED378A6C302BF074FC8DED041A25
:103E100021EE281AD5F8946E8DED020ABDEEC11A76
:103E2000CDED030A11EE103A1DB2336894F81080FC
:103E30009B6D304660EE289A20EEA89A984707EED0
:103E4000900AF8EEE77A304667EEA87AFDEEE77A58
:103E500017EE903A1CB23368DB6D984707EE900A74
:103E6000B8EE678AD7F84039DFED1E7A93ED0FAAD6
:103E7000336828EE288A1B6EB4EEE78AF1EE10FA5A
:103E800058BFB0EE678A30469847BCEEC88A002318
:103E9000089318EE103AB7222AEE28AA20EE280A34
:103EA000ADF82C301A23CDE900323E2105AA404658
:103EB000CDED059A8DED069A8DED07AA8DED090AD7
:103EC000ADF82850ADF82A4053F0DEF90CB0BDEC47
:103ED000068BBDE8F08100BFB84B00209F0CB345B6
:103EE0000AD7233C00FF7F472DE9F04F2DED028BD1
:103EF0001A4B047CD3F838398DB0D3F88480D3F8CA
:103F00008870D3F88C60D3F8905093ED258AD3F85D
:103F100098B0D3F89CA0D3F8DC9086F02BFD00235A
:103F20008DF82C3016222523CDE90032029002AA0A
:103F3000532120468DED078ACDF820B0CDF824A07E
:103F4000CDF82890CDF80C8004970596069553F08F
:103F50009BF90DB0BDEC028BBDE8F08FB86B002073
:103F6000054BD3F8B83E2BB193F8CA00002808BF20
:103F70000220704702207047B84B002008B5034B61
:103F8000D3F8940E03681B68984708BDB84B00200F
:103F9000024B93F8890EC0F340107047B84B0020D5
:103FA00070B52C4E2DED028B0546D6F8940E91ED92
:103FB000018A036886B05B6A0C46984750B9BDEE2B
:103FC000C88A18EE103ADB0704D4022006B0BDEC14
:103FD000028B70BDD4E9040129F036FA0028F4D030
:103FE00002A817F07DF902AA2146284658F074F974
:103FF0000028EAD0184902A817F054FA034600280E
:10400000E3D1DFED160A00900246B0EE600A1448D4
:1040100002A90AF017F8D8B1D6F8940E03685B6AC3
:104020009847044608B10020D0E70E480222042138
:1040300005F01AFC60B1DFED090A09480094234637
:10404000B0EE600A224602A909F0FCFF0028EAD17E
:104050000420BBE7B84B0020C4740020000000001F
:10406000847B0020B82B002008B591F82030032B6A
:104070001CD1D1ED027A9FED0E7A91ED060A0D4B1F
:10408000F0EEE77AF4EEC77ADFED0B7AD3F8940E10
:10409000F1EE10FA4CBF0121002120EE270A0FF0AB
:1040A00095F9002814BF0020042008BD0220FCE779
:1040B00000000034B84B00200000C84210B52DEDC0
:1040C000028BD1ED007AF5EEC07AF1EE10FA82B0F3
:1040D0000C4604DA042002B0BDEC028B10BD9FED4B
:1040E000197AF4EEC77AF1EE10FAF3D891ED030ADB
:1040F0009FED158AF0EEC07AF4EEC87AF1EE10FA70
:1041000019D5D4ED037A1148D4ED010A94ED000AD3
:10411000F4EEC87AD4ED027AFDEEE77AF1EE10FA09
:10412000CDED017A9DF90410ACBF0122002202F00E
:1041300013F80020CFE7F7EE000A27F0D3FF00289E
:10414000C8D0DEE70000B44300000034EC7E00205D
:1041500091ED010AB5EEC00AF1EE10FA08B501DCE6
:10416000042008BD9FED107A104BD1ED007AD3F8F2
:10417000940E20EE070A9FED0E7A0368F4EEC77ADC
:10418000F1EE10FA05DDDB6E98470028E8D000203C
:10419000E7E79FED087AF4EEC77AF1EE10FACCBFAC
:1041A0009B6E5B6EF0E700BF0000C842B84B00207A
:1041B0009A9939403333F33F08B5D1ED007A9FED3A
:1041C000157AF0EEE77AF4EEC77AF1EE10FA1DD523
:1041D000D1ED017AF0EEE77AF4EEC77AF1EE10FA5B
:1041E00014D50D480222032105F03EFB80B10A4898
:1041F0000121FDF7CFFF094890F8603B012B03D068
:1042000000F65C302EF0AEFD002000E0022008BD7C
:104210000420FCE700000034B82B0020B86B00201D
:1042200010B5D1ED007AFCEEE77A17EE903A9CB229
:10423000012C02D0022C06D04CB9064821465EF073
:10424000B9FB002010BD044803F04EF9F9E7042043
:10425000F8E700BFE0750020B82B00201FB5D1EDB6
:10426000017A0B7CFCEEE77ACDED027AD1ED007A93
:104270000093FCEEE77AD1ED030ACDED037A91EDE0
:10428000020A9DF808309DF80C20014602480DF006
:1042900087FE05B05DF804FBB82B002010B50A4C72
:1042A00094F8AD3EDB070CD402220521A4F50050A2
:1042B00005F0DAFA28B902221146A4F5005005F0FB
:1042C000D3FA002010BD00BFB84B002010B5D1EDCF
:1042D000007AFCEEE77A044617EE903A13F0FF03FB
:1042E0000FD10F4BD3F8940E03689B6F984708B11A
:1042F000002010BD0B4A2046062155F0F7F9042096
:10430000F7E7012B09D1064BD3F8940E0368DB6F56
:1043100098470028ECD1044AEDE70220E9E700BF06
:10432000B84B0020104A0C08204A0C089FED0B7A6D
:1043300001F10C03F1EC017AF4EE677AF1EE10FA78
:104340000AD6F0EEE77AF4EEC77AF1EE10FA03DC63
:104350009942EFD1012070470020704700007A4455
:1043600030B52DED028B8DB00023054603930493E9
:10437000059311F09BFC03A911F072FA58B311F0E8
:1043800095FC00F55A7393E8070006AC84E8070033
:10439000DDED060A9DED070A2D7CF1EE600AB1EE17
:1043A000400AA9F069F82046B0EE408A2BF0A0FD43
:1043B000DFED0B7A089B0B93012228EE278A0C2352
:1043C000CDE90032A82109AA28468DED098A8DED94
:1043D0000A0A52F059FF0DB0BDEC028B30BD00BF90
:1043E000E02E6542242938B505460FD003D81B2995
:1043F00007D1012412E04029FBD0A1F14203012B97
:10440000F7D92846BDE8384058F028BB0C2152F0B7
:104410005FF9044610B12846FFF7A2FF204638BDD9
:1044200038B5194C94F8AD3EDB070D460AD4D4F8E4
:10443000B83E93F8CB303BB90122114604F6EC307C
:10444000FDF700FD002038BD94F9883E002B4FF0A9
:10445000020212DA0521A4F5005005F005FA002841
:10446000F0D095ED000ADFED097AD4F8940E20EE35
:10447000270A01210EF0AAFFE4E70921A4F5005064
:1044800005F0F2F9DEE700BFB84B00200000C8429B
:1044900010B5214C94F8AD3EDB070ED4D4F8B83EED
:1044A00093F8CB304BB194F9883E002B07DA012208
:1044B000082104F6EC30FDF777FD002010BDD1EDAA
:1044C000007A9FED167AF0EEE77AF4EEC77AF1EE15
:1044D00010FA0BD512480222112105F0C5F9A0B936
:1044E000022211460E4805F0BFF9E6E7D4F8940E13
:1044F00003681B6898470428DFD0D4F8940E03683B
:104500001B6898471428E5D1D7E7064840F6C41140
:1045100008F0C0FAD1E700BFB84B0020000000341B
:10452000B82B0020707A002070B58B8BC12B05460C
:104530000C463CD8BB2B0CD8542B6AD02ED8113B40
:1045400099B2052918D921462846BDE8704059F08E
:104550001DB9BC3B052BF6D801A151F823F000BFD3
:104560004D4601085B4601084745010847450108DB
:10457000F745010801460108052BE4D801A151F8CF
:1045800023F000BF374601084745010847450108A9
:1045900047460108A945010813460108732B22D09C
:1045A000B22B24D0552BCED10222092145E04AF26C
:1045B0001146B34237D00AD8D12B26D0B3F5967F17
:1045C00035D0D02BBFD1BDE87040FFF729BE4AF2ED
:1045D0001246B34223D04AF21346B342B3D1BDE8E8
:1045E0007040FFF755BFBDE87040FFF767BDBDE8FD
:1045F0007040FFF7ADBD2146BDE87040FFF7D0BC6D
:104600002146BDE87040FFF761BEBDE87040FFF78E
:1046100025BE21462846BDE87040FFF725BDBDE810
:104620007040FFF7FDBEBDE87040FFF737BEBDE844
:104630007040FFF7C1BD022205210A4805F014F9B8
:1046400048B9042070BD02220621F6E7022106487F
:1046500006F06EFAF4E70020F4E70221024806F0C3
:1046600031FAEDE7B82B0020D876002008B591ED9F
:10467000007AF6EE007AB4EEE77AF1EE10FA06DD93
:10468000044801220521FDF78FFC002008BD04200D
:10469000FCE700BFA457002030B52DED028BCD788C
:1046A00093B0272D28BF27250C462722002108A8D4
:1046B000ABF0DCF82A4604F10C0108A8ABF08CF84A
:1046C000424BD3F8940E03685B6A9847002841D0A8
:1046D0009DF8465068063DD400244FF07E532906CD
:1046E000049307940694059427D504A82AF0DAFACF
:1046F000EA0701940294039405F006032ED4002BDC
:104700002ED10D9B01930E9B02930F9B0393304878
:1047100009F046FA9DED100A044630B340F2ED4030
:10472000B7EE001AFFEE000A27F0E0FD2848234606
:1047300001AA04A909F03CFA0CE0099B04930A9B26
:1047400005930B9B069304A80C9B07932AF0B0FAE1
:104750000028CDD113B0BDEC028B30BD062BD6D0D6
:1047600001211B4809F0B8F9F4E7DFED1A0A4FF40C
:104770009E60B7EE001A27F0B9FDF6EE000AB0EE23
:10478000408A27F0AFFCE8B9B6EE000A124BB4EE4F
:10479000C08AF1EE10FAD3F8443908DD38EE400A49
:1047A00030EE008A93ED070A28EE000ABEE730EEED
:1047B000480AD3ED087A30EE000AF0EEE77A27EEE9
:1047C000C00AB3E79FED030AB0E700BFB84B002073
:1047D000847B002000000000B86B00202DE9F0432E
:1047E0009DB0814608460EA9FEF79EFF844BD3F884
:1047F000940E03685B6A984750B19DF86C30012BAA
:1048000009D0DA1F022A06D97E48012109F064F98D
:104810001DB0BDE8F083BDF86840A20504F00706AE
:1048200004F0380704F4E07501D5002DF0D04FF006
:104830000008CDF81480CDF81880CDF81C803EBB60
:104840009FED716A9DED107ADDED117ADDED0F6A55
:1048500027EE067A67EEC67A66EE866A083B012B7B
:10486000CDED056A8DED067ACDED077A04D867485F
:1048700006AA05A9FDF708FE9DF86C30073B022B40
:1048800006D863487DF0BCFE014605A82AF052FF19
:10489000CDF82080CDF82480CDF82880F7B9DDED63
:1048A000147A129B0893F1EE677A139B099308A977
:1048B0004846CDED0A7AFFF739FD0028A4D09FEDD8
:1048C000520A08A82AF06AFF9DF86C30083B012BB9
:1048D00004D84E4809AA08A9FDF7D6FDCDF82C80CA
:1048E000CDF83080CDF83480EDB99FED476A9DED6D
:1048F000167ADDED177ADDED156A9DF86C3027EE3E
:10490000067A67EEC67A66EE866A083B012BCDED25
:104910000B6A8DED0C7ACDED0D7A04D83B480CAACC
:104920000BA9FDF7B1FD14F4806233D1DFED397AC4
:104930009DED180A9DF86C1020EE270ADFED327A03
:104940000839012920EE270A8CBF0021012114F427
:10495000006305BFDFED2F7ADDED190ADFED2E0ACA
:1049600060EEA70A04BFDFED287A60EEA70AAEB9B1
:10497000002F35D1B3FA83F3B2FA82F25B09520900
:104980000291019300920BAB08AA05A91D4809F0FA
:1049900011FA3DE79FED200A0021D8E77FB9B3FA6D
:1049A00083F35B0901200093B2FA82F3CDE9011091
:1049B0005B0914480BAA08A909F094FC28E7002D0C
:1049C0007FF422AF0120B3FA83F3B2FA82F2CDE989
:1049D00000105B090B4852090BA909F02BFC17E7E3
:1049E000002D3FF411AFB3FA83F3B2FA82F2CDE9AE
:1049F00000165B09520905A9024809F05DFA07E7AC
:104A0000B84B0020847B00200000C842B82B002057
:104A1000D4740020E02E6542000000002DE9F0472C
:104A2000A2B08046084614A9FEF77EFE7E4BD3F85E
:104A3000940E03685B6A9847C0B1BDF88040A30537
:104A400004F0070904F4E07700D57FB10CAE3046DE
:104A500016F046FCB9F1000F29D1DDE9150128F067
:104A6000F3FC30B97148012109F036F822B0BDE8F5
:104A7000F0879DF8841009AA404657F017FC0028DB
:104A8000F0D0DDED177A9FED6A7A099B009367EE0F
:104A9000877A10ADFDEEE77ADDE9151217EE903A50
:104AA000284616F03DFC95E80F0086E80F0000252B
:104AB00014F0380A06950795089514D1DDED1A7A99
:104AC000189B0693F1EE677A199B079306A9404657
:104AD000CDED087AFFF72AFC0028C3D09FED540AD9
:104AE00006A82AF05BFE09950A950B959FB99FEDE4
:104AF000506A9DED1C7ADDED1D7ADDED1B6A27EE17
:104B0000067A67EEC67A66EE866A8DED0A7ACDED94
:104B1000096ACDED0B7A14F4806805BFDFED457AA4
:104B20009DED1E0A9FED440A20EE270A04BFDFED2B
:104B3000407A20EE270A14F4006405BFDFED3D7AC9
:104B4000DDED1F0ADFED3C0A60EEA70A04BFDFEDD2
:104B5000387A60EEA70AB9F1000F31D1BAF1000F2F
:104B600052D13046CDED050A8DED040A16F0E8FB72
:104B700003289DED040ADDED050A3FF473AF10A98B
:104B80003046CDED050A8DED040A1095119512956C
:104B900016F036FD00283FF465AFB4FA84F46409DA
:104BA000B8FA88F3DDED050A9DED040ACDF804A0FE
:104BB00000945B0906AA10A91C4809F06BF955E797
:104BC000BAF1000F0FD10123B4FA84F4CDE901A3A7
:104BD0006409B8FA88F3154800945B0909AA06A984
:104BE00009F080FB42E7002F7FF43CAF0123CDE9C1
:104BF0000073B8FA88F2B4FA84F30C485B095209DE
:104C000009A909F017FB31E7002F3FF42BAFB4FAE5
:104C100084F3B8FA88F2CDF800905B095209314666
:104C2000024809F00FFA21E7B84B0020847B0020EE
:104C30000000C842E02E65420000000010B44B7A2C
:104C40008C7ACA7A43EA042343EA0243542B07D0FE
:104C5000562B09D0522B0BD15DF8044BFFF71CBD2E
:104C60005DF8044BFFF7BABD5DF8044BFFF7D6BE05
:104C70005DF8044B57F022BC2DE9F0432DED028B7B
:104C800000F500560446D6F8940EDFED4B8A036813
:104C900091B05B69984704F580490027002840F0EF
:104CA0008780D9F84039D3EDDE7A93EDD88AFDEECE
:104CB000E77A28EE288A17EE903A1DB204F52D58AF
:104CC00008F1340801A940460DF032FF18B94FF041
:104CD00043FA3A4B01933722002102A8AAF0C6FDFD
:104CE000A3238DF8083095238DF8093085F04AFE0E
:104CF000D9F83839CDF80B00D6F8B80ED3F8DC2047
:104D0000D3F8E030CDF80F104430CDF81320CDF8B3
:104D1000173050F053FE0346DFED290A93ED000AE9
:104D2000B7EE001A9F2027F0E1FA10EE103AD6F8FD
:104D3000B80ECDF81B3003681B69984710EE103A87
:104D400004F59246CDF81F301C3618EE103A304666
:104D5000CDF823307DF058FC20EE280A404610EEB6
:104D6000103ACDF82730D9F8E838CDF82B30019B30
:104D7000CDF82F300DF0FEFE10EE103A3046CDF893
:104D80003330CDF83770ADF83B507DF049FCBDEEC7
:104D9000C00A372210EE103A02A904F57C60ADF883
:104DA0003D304EF02BFB11B0BDEC028BBDE8F08323
:104DB00008EE107A002581E70AD7233C2292CA7FA9
:104DC0000000000010B500F58044D4F8380976F0F2
:104DD00003FBD4F84019D4F83809BDE8104076F048
:104DE00061BB000070B54FF4805104460DF0EAFF3E
:104DF00000284ED004F5804604F57C65D6F83809C5
:104E000003689B689847692100F1940228464EF098
:104E10008DF9D6F838090368DB6898476A2100F1F4
:104E2000940228464EF082F9D6F8380903681B69C7
:104E300098476B2100F1940228464EF077F9D6F896
:104E400040296C21284602F52A724EF06FF9202184
:104E500020460DF0B7FFE0B104F50053D3F8940EEF
:104E600003681B69984778B1D6F8402928469032E4
:104E70006E214EF05BF9D6F840292846BC32BDE8D9
:104E800070406F214EF052B9204609F093FF002880
:104E9000EAD170BD08B510F009FFBDE8084010F078
:104EA00091BC00007FB50E464FF6FF7104461546D3
:104EB0000DF088FFE0B1102200216846AAF0D6FC70
:104EC000A3238DF8003095238DF8013003238DF84E
:104ED000023085F057FD1022CDF80300CDF8071001
:104EE00004F57C6069468DF80B6003954EF006FB77
:104EF00004B070BD7FB50E464FF6FF7104461546EF
:104F00000DF060FFE0B1102200216846AAF0AEFC6F
:104F1000A3238DF8003095238DF8013004238DF8FC
:104F2000023085F02FFD1022CDF80300CDF80710D8
:104F300004F57C6069468DF80B6003954EF0DEFA4F
:104F400004B070BD30B52DED048B87B004460D461E
:104F5000182200216846B0EE409AF0EE608AB0EE6A
:104F6000418AAAF083FCA3238DF8003095238DF8A5
:104F7000013006238DF8023085F004FD1822CDF8AB
:104F80000300CDF8071004F57C6069468DF80B50DE
:104F90008DED039ACDED048A8DED058A4EF02EFA43
:104FA00007B0BDEC048B30BD10B54FF48011044642
:104FB0000DF008FF30B104F593500830BDE8104003
:104FC0000FF0F6B810BD00002DE9F0438FB0144685
:104FD000054689463122002101A8DDE9167698466A
:104FE000AAF044FCA3238DF8043095238DF80530F6
:104FF00008238DF8063085F0C5FC236804936368A8
:105000000593A36806933B68CDF81D307B68CDF807
:105010002130BB68CDF825303368CDF8293073686E
:10502000CDF80700CDF80B10CDF82D303122B36844
:105030008DF80F9001A905F57C608DF81C80CDF8E6
:1050400031304EF0DBF90FB0BDE8F08370B52DEDD7
:10505000068B8CB0144605460E462C22002101A872
:10506000B0EE409AF0EE608AB0EE418AB0EE61AAEE
:10507000F0EE429AAAF0FAFBA3238DF804309523B0
:105080008DF805300B238DF8063085F07BFCDFEDC5
:105090001A7A94ED007ACDF8070027EE277A29EEE8
:1050A000279A8DED077A94ED017ACDF80B1027EE53
:1050B000277A68EEA78A8DED087A94ED027A8DF84A
:1050C0000F6028EE278A67EE277A2C2201A905F5C2
:1050D0007C608DED049ACDED058A8DED068ACDEDCF
:1050E000097A8DED0AAACDED0B9A4EF087F90CB036
:1050F000BDEC068B70BD00BFE02E6542A02070475E
:1051000070B5144B88B004466946D3F8B80E04F560
:105110007C6504F500561E227EF01EFB6A460E4991
:1051200028464EF007FBD6F8940E03681B68984794
:1051300096F80421014628464EF020FB04F59350D2
:10514000083010F0F1FF04F590701EF011FF08B068
:1051500070BD00BFB84B002032970C082A4B2B4A79
:1051600070B54360002343618361C361C363284B0F
:10517000426303644FF08042264B436404468263DB
:10518000583059F023F8244E244BA365A825601904
:1051900059F0D2F966513035B5F56A7FF7D104F58B
:1051A0006A705AF075FD002104F5F66080F0C4FEC7
:1051B0001B4BC4F864389FED1B1ADFED1B0A9FEDF3
:1051C0001B0A04F6780076F0F9FE9FED161A9FEDA3
:1051D000180AF0EE410A04F5096076F0EFFE9FED43
:1051E000111A9FED130AF0EE410A04F6A80076F0BA
:1051F000E5FE20460F4945F01DFB20460E4945F0CF
:1052000019FB204670BD00BFF83700200000C841E0
:105210000AD7233C0000E0409C940C08B0940C0892
:10522000EC780020000000009A99993E0000B443F9
:1052300000804A4360880C08C08A0C0870B54C4D49
:105240004C49ADF50E7DD02206465AA8AAF0C4FA04
:105250000FCD0EAC0FC40FCD0FC40FCD0FC495E80A
:105260000F0084E80F0000245AAB18190021B7EE94
:10527000000A103444F09AFFD02CF5D13E4B0FCBEE
:1052800002AC84E80F0001A9204644F043FF90B12E
:105290009DF90430DFED396AE06807EE103AB8EEA8
:1052A000C77AF0EE007AE7EE267AB7EE000A80EED3
:1052B000270A45F05FFE00240EAB181900211034B8
:1052C000B7EE000A44F072FF402CF5D12C49902231
:1052D00036A8AAF081FA0022092136A845F012F872
:1052E00096F97469D6B9274D0FCD1EAC0FC40FCDFA
:1052F0000FC40FCD0FC495E80F0084E80F003246AD
:1053000004211EA844F0FEFF9FED1F0A1F4845F030
:1053100031FE1F48B7EE000A45F02CFE1D4C9FEDF4
:105320001E0A0FCC06AD0FC594E80F0085E80F00EC
:10533000002106A844F03AFF9FED170A00212846F5
:1053400044F034FF04F1100160221EA8AAF044FAD0
:1053500000241EAB18190021B7EE000A103444F0E7
:1053600025FF602CF5D15AF0A7FA0DF50E7D70BD22
:10537000F83A0C08283A0C08383B0C08CDCCCC3D48
:10538000483B0C08D83B0C080000000048870C087C
:1053900057870C08183C0C08000034422DE9F047F0
:1053A00090B00DF106011D205AF078FB002800F0A6
:1053B0009E809DF80630614A0133DBB211210BA8B3
:1053C0008DF8063084F0B2FC00220DF107010BA825
:1053D00044F0D2FB9DF80630594A112105460BA82E
:1053E00084F0A4FC00220DF107010BA844F0C4FBDB
:1053F0009DF80630534A112106460BA884F096FC0E
:1054000000220DF107010BA844F0B6FB9DF8063011
:105410004D4A03F03F03112107460BA884F086FC98
:1054200000220DF107010BA844F0A6FB8046002DD9
:105430005DD0002E5BD0002F59D0002857D02846D1
:1054400044F0B2FD002852D1304644F0ADFD0028B2
:105450004DD1384644F0A8FD002848D1404644F0DC
:10546000A3FD002843D1394C94E80F000DF10C0C3A
:1054700010348CE80F0094E80F000DF11C0989E846
:105480000F0002A9604644F045FE98B3BDF80840FD
:1054900002A9484644F03EFE00284AD0BDF8083034
:1054A00054BB23B340F2E2449C420FFA84FA0FFA51
:1054B00083F927D80DF10A013046ADF80A9046F07D
:1054C0004FF80DF10A012846ADF80AA046F048F859
:1054D0000DF10A013846ADF80AA046F041F8002364
:1054E0000DF10A014046ADF80A3046F053F810B00D
:1054F000BDE8F0870024CBE740F2D662002B08BF5E
:105500001346D1E70DF10A013046ADF80AA046F086
:1055100027F80DF10A012846ADF80A9046F020F868
:105520000DF10A013846ADF80A9046F019F801234A
:10553000D6E7002CDBD040F2D663B5E768870C08CD
:1055400074870C0880870C088D870C08983C0C0821
:1055500037B500F505517822083104464CF046FB7A
:1055600000220C21244844F0CDFE2046FFF716FF10
:1055700004F505500022B7EE000A02211C3044F069
:1055800049FF012504F501511C4A0095002308310B
:10559000452044F0BBFE1A4A1368D90705D41949BF
:1055A000156004F5FF5310330B6004F506501549E0
:1055B00001223C30012544F0FBFE134A00950023F4
:1055C00004F57C61FD2044F0A1FE104B1A68D2075F
:1055D00005D40F4A1D6004F58C540C3414600C483B
:1055E000012144F001FF45F02BFB0A4A138843F0E8
:1055F0000103138003B030BDA0870C08B0AF0D08C5
:10560000E47E00200022002070340D08E87E002097
:105610000C220020288100200F299DBF302303FB8E
:105620000100503000207047014B93F98F01704703
:10563000B84B0020024B93F8AD0E00F0010070470C
:10564000B84B0020044BB3F85431DB075ABF006954
:10565000C0F3401000207047B84B0020014BD3F836
:10566000D40A7047B84B002008B503689B68984778
:1056700030B9044B93F9AC0EB0FA80F0400908BD84
:105680000020FCE7B84B002038B50D1E2DDB174C71
:1056900094F8E02AEBB29A4227D3D4F8DC3A0122FC
:1056A000595DA4F5005004F0DFF8F0B158F00EFF9A
:1056B000032159F0C3FEC0B958F008FF0D2159F07D
:1056C000BDFE90B994F97431EB40DB075CBF94F9EF
:1056D0008E11E940A4F5005048BF0221BDE83840D2
:1056E00058BF01F00101FCF76BBD38BDB84B00207D
:1056F000022A10B50C4605D1BDE8104009483522F4
:1057000004F0B2B8084BD3F8940E03681B689847AE
:10571000A04205D158F0DAFEBDE8104058F060BE56
:1057200010BD00BFB82B0020B84B002029B10229C2
:1057300007D1044BC3F88C1E7047024B0122C3F8FB
:105740008C2E7047B84B002031B1022907D1044B91
:10575000012283F8902E7047014B83F8901E70470A
:10576000B84B002010B500F50053DFED186AD3F8F0
:10577000CC2AD3F8C83AB2F90820B3F908309FED23
:10578000147A07EE902AF8EEE77A0446C7EEA60AE6
:1057900000F593500121083007EE903AF8EEE77AD1
:1057A00060EE870A87EEA60A20EE070A10F01CFBBF
:1057B0004EF0D2FC26214EF00BFC04F53150054A88
:1057C000BDE8104006212C3050F066BD0000C842F4
:1057D00035FA8E3C6C920C0800F58042002382F86A
:1057E0005439044A00F5315013720621024A2C3014
:1057F00050F052BD9D80002078920C08F8B500F55D
:105800008045044695F85419002955D02B4B2C4A55
:10581000D3F8940E904204D1D3F8B83E93F8CB302D
:1058200023B92046BDE8F840FFF7D6BF254E95F8CE
:10583000557904F50053012093F9882E3072C7BBC7
:10584000002A39DB85F855090139C9B285F85419A0
:10585000D3F8CC2AD3F8C83AB2F90820DFED1A6A97
:10586000B3F908309FED197A07EE902AF8EEE77A3F
:10587000B1FA81F1C7EEA60A04F593504909083040
:1058800007EE903AF8EEE77A60EE870A87EEA60A0E
:1058900020EE070A10F0A8FA95F8543963B904F518
:1058A000315033720A4ABDE8F84006212C3050F0DE
:1058B000F3BC002AC8DAB4E7F8BD00BFB84B00203B
:1058C0006C7D00209D80002000007A4535FA8E3CDA
:1058D0008C920C086D2900F3E380012901DC59F05A
:1058E000FBBB8B1E6B2BFAD80FF2040C5CF823F079
:1058F000FF5A0108F95A0108FF5A0108FF5A010826
:10590000DF580108FF5A0108DF580108DF58010875
:10591000F95A0108DF580108FF5A0108F95A01082D
:10592000F95A0108DF580108FF5A0108FF5A010817
:10593000FF5A0108DF580108DF580108F95A010829
:10594000FF5A0108F95A0108DF580108F95A0108FD
:10595000F95A0108DF580108DF580108DF5801082B
:10596000DF580108DF580108F95A0108FF5A0108F9
:10597000DF580108DF580108DF580108FF5A010805
:10598000DF580108F95A0108DF580108DF580108FB
:10599000FF5A0108F95A0108DF580108DF580108C9
:1059A000DF580108FF5A0108FF5A0108FF5A010891
:1059B000DF580108DF580108FF5A0108DF580108C5
:1059C000DF580108FF5A0108FF5A0108FF5A010871
:1059D000DF580108DF580108FF5A0108FF5A010883
:1059E000DF580108DF580108DF580108DF580108B7
:1059F000DF580108DF580108FF5A0108FF5A010863
:105A0000FF5A0108FF5A0108FF5A0108FF5A01080E
:105A1000DF580108F95A0108F95A0108DF5801084E
:105A2000DF580108DF580108DF580108DF58010876
:105A3000DF580108FF5A0108F95A0108DF58010828
:105A4000DF580108DF580108DF580108DF58010856
:105A5000DF580108DF580108DF580108DF58010846
:105A6000DF580108DF580108DF580108DF58010836
:105A7000DF580108FF5A0108DF580108DF58010804
:105A8000DF580108DF580108DF580108DF58010816
:105A9000DF580108DF580108DF580108F95A0108EA
:105AA000A12921DC96297FF71AAFA1F197030A2BD0
:105AB0003FF615AF0FF2040C5CF823F0FF5A010813
:105AC000FF5A0108DF580108FF5A0108DF58010892
:105AD000DF580108DF580108DF580108F95A0108AA
:105AE000F95A0108FF5A0108B42908D0DB2903D06C
:105AF000B2297FF4F4AE7047002359F0BFBA704763
:105B000070B563298AB000F3D180012904DC0AB0A2
:105B1000BDE8704059F082B88B1E612BF7D801A404
:105B200054F823F0235D0108375D0108575D010833
:105B30005F5D01080F5B01088F5D01080F5B0108C5
:105B40000F5B01083D5E01080F5B01080F5B010858
:105B5000455D0108635E01080F5B0108395E0108BD
:105B60009D5E0108AB5E01080F5B01080F5B010839
:105B7000BB5E0108C95E0108D75E01080F5B010822
:105B8000F95E01080B5F01080F5B01080F5B01085C
:105B90000F5B01080F5B01080F5B01081D5F010827
:105BA000375F01080F5B01080F5B01080F5B0108FD
:105BB0003B5F01080F5B01080F5B01080F5B0108E9
:105BC0000F5B01083F5F01080F5B01080F5B0108D5
:105BD0000F5B01080F5B01080F5B01080F5B0108F9
:105BE0000F5B01080F5B01080F5B01084F5F0108A5
:105BF0000F5B01080F5B0108AF5E0108B35E01088F
:105C0000B75E01080F5B01080F5B01080F5B01081D
:105C10000F5B01080F5B01080F5B01080F5B0108B8
:105C20000F5B01080F5B01080F5B0108435F010870
:105C3000475F01084B5F01080F5B0108535F0108D4
:105C4000575F01080F5B0108995F01085B5F01085E
:105C50000F5B01080F5B01080F5B01080F5B010878
:105C60000F5B01080F5B01080F5B0108FB5F010878
:105C70000F5B01080F5B01080F5B01080F5B010858
:105C80000F5B01080F5B01080F5B01080F5B010848
:105C90000F5B01080F5B01080F5B01080F5B010838
:105CA0000F5B01080F5B0108116001089F291DDCD3
:105CB00096297FF72CAFA1F19703082B3FF627AF6A
:105CC00001A454F823F000BF156001081960010811
:105CD0000F5B01082D6001080F5B01080F5B0108D5
:105CE0000F5B01080F5B010809600108B42900F08F
:105CF000D780DB2917D0B2297FF409AF002A00F042
:105D00007581022A0FD1AD4BD3F8940E03689B6FB7
:105D1000984740B957F018F9A94A042150F0BCFA45
:105D200001E0022A01D001242EE035220E21A548EF
:105D300003F09AFDF7E7111E18BF0121A148FCF7F7
:105D40003FFAF0E7012A04D0022A14BF0021022101
:105D5000F4E71146F2E70621FFF7CAFCE3E7022A5F
:105D6000E1D1964DD5F8940E0368DB6A9847044656
:105D70000028D8D0D5F8D03AB3F90830002BD2D1CA
:105D8000A5F50050FFF7EEFC20460AB070BD022AD0
:105D9000C9D18A4D8C4BD5F8942E9A42C3D0D5F8F0
:105DA000B83E93F8CB30002BBDD005F50054B4F9C4
:105DB000903B2BB9D5F8D03AB3F90830002BB2D0CC
:105DC0001C22002103A805AEA9F050FD304615F0B5
:105DD00087FAB4F9903B93B91623ADF80E30D4F896
:105DE00010397A48642BB8BF642303A906932AF0BC
:105DF0002BFC20B14EF0B0F927214EF0E9F804F663
:105E00000C1494E80F0086E80F00D5F8D03A6F48DC
:105E1000B3F90830002BCCBF1023152303A9ADF82C
:105E20000E302AF011FC00283FF47DAF4EF094F9BB
:105E300027214EF0CDF876E703218DE7022A04D022
:105E40005E4B002283F8E42A6DE76148192145F092
:105E5000DBFF04460028F3D0584B012283F8E42AE4
:105E600092E7012A0BD0022A11D0002A7FF45BAFFF
:105E7000524B83F8B8214EF06FF92B21D9E74F4BE5
:105E8000019283F8B8214EF067F92C21D1E74B4BF2
:105E900083F8B8214EF060F92D21CAE70F215BE7A6
:105EA0004C48114683F040F93DE7092154E70421AD
:105EB00052E7052150E717214EE7901E414241412C
:105EC00045485CF077FD2EE7022A7FF42CAF3D4871
:105ED00001F00AFB27E7012A06D0022A07D0002A90
:105EE0007FF421AF1146EBE711460192E8E73A480B
:105EF00001215CF05FFDEAE7384B911ED3F8383999
:105F00004A424A4183F820200DE7931E59425941E5
:105F1000324BD3F8380977F05DF904E7274B013AA3
:105F200093F88A1E012A8CBF0022012262F3041119
:105F300083F88A1EF7E611210EE712210CE71521DE
:105F40000AE7002108E7102106E7022104E7012102
:105F500002E7072100E70B21FEE6022A1F4B0ED1C4
:105F6000012483F8804A4EF0F7F84A214EF030F8C9
:105F700056F0EAFF1A4A062150F08EF904E7002293
:105F800083F8802A4EF0E8F84B214EF021F856F0C5
:105F9000DBFF144A0621C1E6012A09D0022A0AD0F1
:105FA000002A7FF4C0AE01210F480CF0F9FDBAE6DB
:105FB00001920021F8E71146F6E700BFB84B002038
:105FC000C7920C08B82B0020D87600201477002048
:105FD000C8380020EC780020E0750020B86B002065
:105FE000A4920C08B5920C082C570020184BD3F83B
:105FF000940E0368DB6F984795E61146FFF796FB12
:10600000144803F0D7FF8EE61146FFF79DFB8AE6A2
:106010001B21A1E61C219FE6022A7FF484AE0E48D4
:10602000FCF7ACFE56F090FF0C4AB3E7114658F06F
:1060300015FD0B4873F0A6FF044600283FF473AE2D
:10604000034A92F88B3E43F0020382F88B3E9BE6B4
:10605000B84B00205C760020B82B0020E0920C08A2
:10606000A457002010B5044604487CF0CBFA04F194
:106070000801BDE8104027F065B900BFD4740020C6
:1060800038B504462DED028B11487CF0C1FA054667
:1060900029F094F80F48B0EE408A0CF02DFE90B134
:1060A000DFED0D7AB4EEE78AF1EE10FA0BDDD5EDF7
:1060B000000A95ED010AA7F0DFF9DFED087A20EE7E
:1060C000270A84ED080ABDEC028B94ED080A38BD5E
:1060D000D4740020B82B002000401C46E02E6542FE
:1060E000074B93F97501022805D0032806D0003824
:1060F00018BF0120704781F00100704704207047ED
:10610000B84B002003688B4216D00429C0E9001365
:1061100002D007290ED07047084B9FED097A03F58E
:106120008D63D3ED007AF8EEE77A67EE877AC0EDFB
:10613000087A704700238362704700BFB83B002095
:106140000AD7233C08B50246FFF7CAFFBDE808405E
:1061500001461046FFF7D6BF70B52DED048B0446FF
:10616000F0EE408AB0EE608A0D46164684F002FCDE
:106170009FED329ADFED329AE06176B3236843B93E
:10618000304B03F58D63D3ED007AF8EEE77AC4ED7A
:10619000097A68EE898A002DB7EE000AFFEE007AD0
:1061A000B8BFB0EE670A68EE808AC4ED058A264B58
:1061B000B4EEE98AF1EE10FAD3F8380930DA75F066
:1061C000E7FF20EE090A84ED060ABDEC048B2046A9
:1061D0000321BDE87040FFF795BF94ED090A98EEE2
:1061E000890A26F02DF8002D84ED050A0BDAB4EEAD
:1061F000E90AF1EE10FADADBDFED147A30EE670A25
:1062000084ED050AD3E7D2D0DFED117AB4EEE70AC8
:10621000F1EE10FACBD8DFED0D7A30EE270AEFE77A
:1062200075F0B6FFB4EE480AF1EE10FA48BFB0EED2
:10623000408A28EE098A84ED068AC6E70000C84233
:1062400000000034B83B0020B86B002000A00C47D1
:10625000000000B410B52DED028B0446B0EE608A4C
:10626000F0EE408A84F086FBDFED090AE06168EE1B
:10627000A08A68EE200AC4ED098ABDEC028BC4ED49
:106280000A0A20460621BDE81040FFF73BBF00BFC9
:106290000000C84208B54A680346084642B98A6801
:1062A00032B9C96821B9BDE808400748FFF74ABFBD
:1062B00003F1080115F0A4F928B1BDE8084002482F
:1062C0000221FFF71FBF08BDEC7E002008B50721A3
:1062D000FFF718FF80ED0A0A08BD000008B5036843
:1062E000032B23D1D0ED057A9FED127AF0EEE77AF9
:1062F000F4EEC77AF1EE10FA1AD50F4B90ED090AB9
:1063000003F58D63D3ED007AF8EEE77A37EEC00A35
:1063100025F096FFDFED097AB0EEC00AB4EEE70A89
:10632000F1EE10FA94BF0120002008BD0120FCE727
:106330000020FAE700000034B83B0020000048438A
:1063400030B50368023B85B00446082B6FD8DFE800
:1063500003F0050D30374D6341636300FFF782FEA4
:1063600084ED090A94ED090A05B030BD84F002FB02
:10637000E369DFED320AE061C31A07EE903AF8EE06
:10638000677A94ED050A67EEA07AD4ED060AF1204B
:1063900020EEA71A67EEE00A25F0A8FFD4ED057AF3
:1063A00077EEC07AC4ED057AD4ED097A37EE800A2B
:1063B000D6E7FFF765FEDFED227A20EE270ACFE76A
:1063C000204B03F56E63D3ED007AF8EEE77AC0ED6B
:1063D000097AC7E71C4DD5F84C097AF0ADFA0028C8
:1063E000C0D0D5F84C391B6B6362BBE784F0C2FAAE
:1063F000E3699FED127AD4ED0A6AE061C31A07EEF1
:10640000903AF8EE677A67EE877A94ED097AA6EE0D
:10641000A77A84ED097AA5E70B4B9FED0C0AD3F818
:1064200038096C3029F066F984ED091A9AE7064BB1
:10643000D3F84039D3F84433D6E700BF6F12833A1C
:106440000000C842B84B0020B86B00209F0CB34539
:106450000368092B08D8DFE803F0050A05050505E0
:10646000070705100023836290ED0A0A7047044B6A
:10647000D3F84039D3F84833F5E7C36AF3E700BFF0
:10648000B86B0020F8B50023214FCB6297F8AD3EE2
:10649000204E13F0010F04460D462DD1D7F8940E6F
:1064A00003685B6F984738B3D7F8940E03F08EFB00
:1064B000DFED197A85ED0B0AB0EEC00AB4EEE70AFB
:1064C000F1EE10FA03D409213046FFF71BFE114804
:1064D000FFF736FF0F4884ED000AFFF7B9FF336876
:1064E00084ED010A0A2B0FD8DFE803F00C1010101E
:1064F0001010100C100C0C003368092BE7D1054864
:106500000021E2E70223A3602046F8BD0123FAE759
:10651000B84B0020EC7E002000000034034B012229
:106520001A6000229A60DA601A617047EC7E0020DF
:1065300013B501A904460CF07BFA04F5804320B999
:10654000012283F8FD2902B010BDDDED017ADFEDF7
:10655000096A03F51F62B8EEE77AD2ED007A67EEBA
:10656000A67AB4EEE77AF1EE10FA54BF01220022C7
:10657000E7E700BF0000C8422DE9F04F2DED068B84
:1065800000F5005700F5935997F9C6318BB00646D0
:1065900000F5804409F1080933B1D7F8B83E93F803
:1065A000CB80B8F1000F0FD10021A4F8741A48462F
:1065B0000FF0E2FD94F8751A48460BB0BDEC068B5F
:1065C000BDE8F04F0FF0E2BD84F0D4F98346D4F873
:1065D00040099FED978A90EDDBAA78F0CDFB07ADDF
:1065E000002800F0CD80D4F8403903F55C7393E8BF
:1065F000070085E8070028468DED098A29F078FC18
:10660000B0EE409A30460CF077FB06F5924A0AF15C
:106610001C0A002800F0B78050467BF0F9FF07C83D
:1066200085E8070028468DED098A29F061FCF0EE27
:10663000409AD7F8940E03681B689847122840F0D8
:10664000AB80002384F8743AD7F8940E03685B6932
:10665000984728B1D7F8D03AB3F90830002B0CDCB2
:1066600097F9883E002B08DAC4F878BA50467BF0D8
:10667000CBFF04F67C2383ED000A94F8743A5BB1F7
:10668000D4F8780A41F28833ABEB000B9B4540F21B
:106690009180002384F8743AD4F838099FED650A94
:1066A0006C3029F027F88DED070ACDED080A8DED45
:1066B000091A95E8070004AB01AD9FED5F0A83E876
:1066C000070085E80700284629F014F83046B0EEA8
:1066D000408AF0EE608A8DED040ACDED050A8DED5D
:1066E000061A0CF009FB002876D0DFED547AF4EEA0
:1066F000E79AF1EE10FA94BF01250025D4F840097D
:1067000078F03AFB30B1DFED4D7AB4EEE79AF1EE76
:1067100010FA0AD9002D66D1D7F8940E03681B68C9
:106720009847022866D04FF00008D4F8400978F066
:1067300045FC0546002876D0B5EEC0AAF1EE10FA69
:1067400070D5DFED3F7AB4EEE7AAF1EE10FAACBFF8
:106750000126002650467BF063FF66B9DFED397AEB
:10676000B0EEC00AB4EEE70AF1EE10FA5DD8002DE3
:1067700008BF4FF0000894F8741A84F8758A16E779
:10678000B0EE489A3EE730460CF088FA00287FF4D5
:1067900043AFDFED279A4CE7D7F8B83E93F8CB30FC
:1067A000002B3FF451AF97F9883E002BBFF64CAF5A
:1067B000012347E750467BF027FF04F67C23D3ED07
:1067C000007A30EE670ADFED207AB4EEE70AF1EEE8
:1067D00010FA3FF75EAF5FE730460CF05FFA054610
:1067E000002882D18AE7D4F8400978F0C5FA002859
:1067F00092D19AE7B0EE680AA6F01CFCF0EE408A4F
:10680000B0EE480AA6F016FCDFED107A20EE280A5A
:10681000B4EEE70AF1EE10FACCBF4FF001084FF0EA
:10682000000882E700252E4694E7B046A3E700BFA4
:10683000000000009F0CB345D30237390000FA4234
:106840000000C8C2000070420000484255CF7D3FA2
:1068500038B504460CF050FA04F59355083548B99C
:1068600020460CF01BFA014620B92846BDE8384006
:106870000EF004BF04F50054D4F8940E03689B6C2A
:10688000984720B9D4F8940E0368DB6C984701460A
:10689000EBE7000030B5044689B0684604F593552F
:1068A00014F01EFD083504A814F01AFD69462846A8
:1068B0000EF09EFF98B104A928460EF0E9FF70B1D2
:1068C000059B019323680022DB6C694620469847AC
:1068D00028B104F5255001212C307FF0F9FD09B0D5
:1068E00030BD000000F5805292F8E424D2070BD4AA
:1068F00000F50052D2F8B82E92F8CB1009B1FFF78C
:10690000C9BF03689B6C18477047000030B587B05B
:10691000044602A8019114F0E3FC04F5935002A987
:1069200008300EF065FF019A18B90025284607B017
:1069300030BD236802A9DB6C204698470546002835
:10694000F3D004F5255001212C307FF0C1FDEDE797
:10695000F0B5044685B004F59356684608360F46F0
:10696000154614F0BDFC694630460EF091FF10B993
:10697000002005B0F0BD394630460EF0F1FD00288C
:10698000F6D0002DF5D004F58054284694F8E43470
:1069900043F0020384F8E434EBE700002DE9F04F04
:1069A0002DED0A8BBDB0044624220E4618A8002106
:1069B000A8F05CFF2422002121A8A8F057FF242280
:1069C00000212AA8A8F052FF04F500552422002136
:1069D00033A8A8F04BFF0023CDE90D330F9395F8B2
:1069E000893E13F0080837D143F0080395F8C42A0C
:1069F000079285F8893E15F0A7FD90F9213003B381
:106A000090F84033EBB104F25457384615F0ACFC23
:106A1000C24694F876355FFA8AF18B421FD9384620
:106A200015F080FC0AF1010A81460028F1D1C84A1C
:106A30000221304652F05AFE95F8893E69F3C303AD
:106A400008E0C44A0221304652F050FE95F8893ED3
:106A50006FF3C30385F8893E4FF001083AE304F56C
:106A60002F532C33012118460BEE903AFBF790F888
:106A7000814608B9B84ADBE720460BF069FED5F835
:106A8000D03AB3F90890B9F1000F01D0B34AD9E771
:106A900095F9883E002B01DBB14AC9E7204601F099
:106AA00075FE04F53B53243318464A460CA90CEEF8
:106AB000103A11F0BDFF002814BF022301230393F5
:106AC000F123CDE913398F210A23CDE90031307C40
:106AD000ADF85490032313AA4D2150F0D5FBA14BE0
:106AE0009FEDA18A01225A720621A04A304652F037
:106AF000FDFD039B022B0CBF9D4A9E4A062130469A
:106B00004FF0000952F0F2FD85F88291494638466F
:106B100015F074FB94F876355FFA89F18B420CD945
:106B200013AA38468DED138A8DED148A8DED158AE2
:106B300009F1010915F0E4F9ECE7384615F014FC09
:106B40004FF0000A4FF07C0B94F876255FFA8AF933
:106B50004A4519D94946384615F0C4F8C0B20BFB6E
:106B600000403CAA0C2300F2E45003FB092C07C8A8
:106B7000ACF1900C8CE807003CAA02EB890909ED06
:106B80002F8A0AF1010ADFE741F288310AA821F0D1
:106B90008FFED5F8B80E9FED749A03689FED76AA24
:106BA0009B6ADFED76AA9847D5F8B80E01217CF0F4
:106BB000D7FC734B1B680293D86A036801211B68DA
:106BC000984783F0D7FE059083F0D4FEF0EE499A03
:106BD0000690002504F50059079A99F8C43A9342A3
:106BE00040F0D68094F89618384615F09BFB0028A4
:106BF00000F0CE80D9F8B83E93F8CB300493002B48
:106C000000F0C68041F288310BA821F051FE83F0DC
:106C1000B1FE059BC01A132840F2D78083F0AAFE6C
:106C2000059020460BF094FD59F052F9824659F038
:106C3000E9F8D9F8D03AD9F8B80EB3F9083000EE2F
:106C4000103AB8EEC00A20EE0A0A7EF063F9504608
:106C500059F0E0F8384615F087FB1CEE100A12F0E8
:106C6000D1F8D9F8D03ADFED400AB3F9083000EE98
:106C7000103AB8EEC00AA22020EE0A0AB7EE001AB7
:106C800025F034FBB4EEE90AF1EE10FA1CEE100A1E
:106C90004FF000020CA958BFF0EE409AF0EE408A87
:106CA00011F0C6FE08B900230C939DED0C8ADFEDB0
:106CB000357AB4EE498AF1EE10FAF4EEE78A48BF6D
:106CC000B0EE498AF1EE10FA80F28D809FED2E9A97
:106CD000DFED2E8A4FF0000A94F876355FFA8AFBD2
:106CE0005B4540F294814FF00C0918AB09FB0BF99E
:106CF00003EB0900B0EE490A28F0FCFC594638467F
:106D0000CDED110A8DED121A8DED100A14F0EAFF87
:106D10007C23C0B203FB0040B0EE680A00F2E450EE
:106D200028F0E8FC3CAB13A910A899448DED130A98
:106D3000CDED140A8DED151A28F0B0FC0AF1010A08
:106D400009ED240A49ED230A09ED221AC4E700BF20
:106D5000DD940C08CC940C08DBA80C08EB940C0810
:106D6000FD940C089D8000200000000008950C0890
:106D70001D950C08833E0C086F12833A0000C84230
:106D8000E07E002000000034A4707D3F0AD7233C41
:106D9000D9F8B80E03689B6A9847D9F8B80E002155
:106DA0007CF0DEFB029BD86A036800211B689847D1
:106DB000002D40F05F813046C94A052152F096FC13
:106DC0002946384615F01AFA70E1029B986A036862
:106DD00005215B6898470BA821F076FDB0EE498A43
:106DE000B0EE489AF6E64FF000094FF00C0B04F5B0
:106DF000B26A94F876255FFA89F39A4222D9194645
:106E00003846089314F06EFF089B0BFB03F13CAB74
:106E10005A18A2F16C034FF07C0CC0B2CDE90832D5
:106E20000CFB00A018AB1944543028F04DFC089B13
:106E3000099A09F1010902ED1B0AC3ED010A83ED6C
:106E4000021AD6E7039B012B4FF0000A46D19FEDB3
:106E5000A5BA9FEDA59A4FF00C0B94F876355FFA22
:106E60008AF5AB4240F286800BFB05F53CAB03EBA9
:106E70000509A9F14803089321ABB0EE680A581937
:106E800028F048FC089B09ED120AC3ED010A83EDC6
:106E9000021A33ABB0EE4B0A581928F02BFC2AAB80
:106EA00058198DED100AB0EE490ACDED110A8DED9D
:106EB000121A28F01FFC13A910A88DED130ACDEDAE
:106EC000140A8DED151A28F0FFFB0AF1010A09EDED
:106ED000090A49ED080A09ED071ABEE79FED819AF4
:106EE0009FED81BAF0EE088A94F876355FFA8AF958
:106EF0004B4564D99DED0C0AB4EEE80AF1EE10FAA8
:106F000035DB0C2303FB09F93CAB03EB090521AB93
:106F100003EB090028F0FEFB33AB45ED110A05ED4C
:106F2000101A05ED120A03EB0900B0EE490A28F029
:106F3000E1FB2AAB03EB09008DED100AB0EE4B0A22
:106F4000CDED110A8DED121A28F0D4FB13A910A86B
:106F50008DED130ACDED140A8DED151A28F0B4FB52
:106F600005ED090A45ED080A05ED071A049D0AF129
:106F7000010AB9E74FF000094FF00C0A94F8763592
:106F80005FFA89F5AB4241D933AB0AFB053028F0F3
:106F9000AFFF1BEE900AF0EE408A72F0EFFF07EEB3
:106FA000900AB8EE677A3CABC8EE877A03EB8505AA
:106FB00009F1010967EEAA7A45ED2F7ADEE74FF075
:106FC000000A4FF00C0B94F876355FFA8AF94B45BE
:106FD0001DD933AB0BFB093028F08AFFC8EE297AA4
:106FE0000AF1010A1BEE900A67EE808A72F0C6FF72
:106FF00007EE900AB8EE677A3CABC8EE877A03EBEF
:10700000890967EEAA7A49ED2F7ADCE7049D83F0BF
:10701000B1FC069BC01AB0F5FA7F27D983F0AAFC11
:1070200004F50053DDED0D7AD3F8D03A0C9A1B89A4
:107030001392FCEEE77A339A1492ADF85C30349AEE
:10704000159217EE903A359A1692ADF85E30F0220E
:107050001423CDE90032B121069013AA307C50F000
:1070600013F96BF0D9FD317C6BF0D0FC0BA821F04B
:107070002BFCB5E60399384615F0C0F800254FF013
:107080000C0A94F87635E9B28B4207D933AB0AFB88
:107090000132384614F034FF0135F2E7384614F077
:1070A00041FF124A0621304652F020FB104B0025CA
:1070B00020465D7201F05CFB04F50650023043F09F
:1070C0008FFC99F8893E65F3C30389F8893E0AA8C5
:1070D00021F0FAFB40463DB0BDEC0A8BBDE8F08FD5
:1070E000B5FF0D08A4707D3F0AD7233C25950C08F9
:1070F0009D8000207FB54C4BD3F8903ADB070446C7
:1071000000F18F8000F50055D5F8B83E93F8C12006
:10711000002A40F0868093F8CB30002B7ED095F982
:10712000883E002B7ADB00F5804696F8803A002BEB
:1071300077D1D6F838099FED3D0A6C3028F0DAFA9D
:10714000CDED020A60EEA00ADFED397A8DED010A7D
:10715000E0EE000A8DED031AF4EEE70AF1EE10FA04
:107160005CDCD6F838399FED337AD3ED377AF4EE1C
:10717000C77AF1EE10FA04D5D5F8B83E1B7A002B89
:107180004CD0B5EE007AF4EEC77AF1EE10FA45D4A1
:1071900004F592401C307BF043FADFED277AB4EE21
:1071A000E70AF1EE10FA39D8D6F838399FED237A8C
:1071B000D3ED367A67EE877AB3EE0E7AF4EEC77ABD
:1071C000F1EE10FA2ADA1E4AB4F9A410138801333A
:1071D0009BB2138019B9B4F8A210A4F8A410B4F8A3
:1071E000A41099421DD8002616804CF0B5FF01224C
:1071F00019214CF00DFFD5F8B80E03685B6998476C
:10720000431C04F531500F4A31462C304FF044F8FE
:10721000D5F8B83E012283F8C12002E0084B0022D5
:107220001A8004B070BD00BFB84B00209F0CB3455E
:107230004054094A6666663F000000B4E02E65428D
:10724000267F00203C950C0870B52DED028B4A4B33
:10725000D3F8903A9B0784B004461FD400F58045CC
:10726000DFED468AD5F8380903681B699847D0EDE9
:10727000017AF4EEE87AF1EE10FA0FDB04F5005330
:1072800004F59546D3F8B82E92F8C110043649B1EA
:10729000002303A9304603934EF092FB04B0BDECEB
:1072A000028B70BD92F8CB20002AF1D093F9883E72
:1072B000002BEDDB95F8803A002BE9D1D5F83809A1
:1072C00003681B699847D0F8A430D5F838090393B0
:1072D00003681B69984704F58C7200F1A4013046DD
:1072E0004EF010FCDDED037AB0EEC08AF0EEE77AE6
:1072F000F4EEC87AF1EE10FA03D503A930464EF049
:107300005FFBD5F8380903681B699847D0ED040A7C
:10731000F4EEE80AF1EE10FAC0DBF6EE087A60EE61
:10732000A77AF4EEC87AF1EE10FA1DD583F022FBAD
:10733000D5F8903A42F21072C31A9342AED9DFEDFB
:10734000107AC5F8900A68EE277A04F5315417EEE2
:10735000900AF9F7D9F82C34CDE90001094A002147
:1073600020464EF099FF99E79DED030A24F0BAFEFE
:107370000028DBD192E700BFB84B002000000034AA
:107380000000C84258950C0810B5044600F594401A
:1073900028305BF021FB04F594400121BDE810404A
:1073A000483064F071B80000F8B500F58045044637
:1073B00095F9283A4BB300F5005695F83C2A96F813
:1073C000883EDB43C3F3C01363F3C30200F5944765
:1073D00000F5924085F83C2A1C307BF021F9DFED66
:1073E0003E7A283720EE670A38465BF075FB95F841
:1073F000803A53B938465BF01BFBD6F8B83E93F899
:10740000CB301BB9354B00221A80F8BD95F83C3AB9
:10741000DB07FAD4D6F8940E03689B6B98470028D4
:10742000F0D096F9883E002BECDB2C4E33884BB91C
:10743000B5F92E3A33B1642213FB02F3D5F81029C3
:107440009A42E2DB38465BF063FBD5F838399FEDB2
:10745000247AD3ED367A67EE877AB3EE0E7AF4EEBD
:10746000C77AF1EE10FA05D83388002BCDD0013B56
:107470003380CAE7B4F9A4301BB9B4F8A230A4F839
:10748000A4303388B4F8A420B4F9A4001549934279
:107490003CBF013333803388D5F8E828012B01D174
:1074A0000A60B2E709689142ACDD18B9B4F8A220CD
:1074B000A4F8A420B4F8A4209A42A6D800233380CC
:1074C0004CF04AFE02220C214CF0A2FD2046BDE801
:1074D000F840FFF759BF00BF0AD7233C247F0020A4
:1074E000E02E6542207F002008B500F5804292F929
:1074F000283A6BB300F5005393F9883E002B0EDA5F
:1075000000F53150134A06212C304EF0C5FE4CF0E8
:1075100023FE0322BDE808400F214CF079BDB2F9EB
:107520002E3A8BB1D2F81029642113FB01F39A4251
:107530000ADA00F53150084A01212C304EF0ACFE39
:107540004CF00AFE0222E5E7BDE80840FFF71CBF49
:1075500008BD00BF70950C0882950C08F0B52DEDA4
:10756000028B00F500555B4ED5F8B83E93F8CB3052
:107570008DB0044633B195F9883E002B02DB95F9B6
:107580009E312BB9002333800DB0BDEC028BF0BDD2
:1075900000F5804797F8803A002BF3D101F05AFBB1
:1075A00000287DD1D5F8940E03689B6B984700287E
:1075B000E8D004F591406C304EF024FA28F098FCA5
:1075C000F0EE087AB4EEE70AF1EE10FAF0EE408A37
:1075D000D8DA04F5805303F5966203F2B443D3ED91
:1075E000007A92ED000A20EE270AA5F0DDFEDFED1D
:1075F0003A7A20EE270AB2EE0E7AB4EEC70AF1EE1E
:1076000010FABFD9D7F8383993ED368A28EE278A91
:10761000F3EE0E7AB4EEE78AF1EE10FAB2D904F581
:107620009350002309A9083009930A930B930EF095
:107630003BF900283DD13388B4F9A42001339BB233
:107640003380002A40D0B4F8A420B3EB420F9BDB78
:107650004CF082FD01220C214CF0DAFC1F4B002281
:1076600018EE900ACDE90623F8F74EFF1C4BCDE942
:107670000401002218EE100ACDE90223F8F744FFB6
:1076800004F531542C34CDE90001164A204600217E
:107690004EF002FE01220C211348FAF785FC73E735
:1076A000D5F8940E0368DB6C984700287FF47AAF16
:1076B00068E709A828F01CFCF2EE047AB4EEE70AA9
:1076C000F1EE10FAB7DB5DE7B4F8A220A4F8A4202D
:1076D000B9E700BF1C7F0020E02E65420000084093
:1076E00000003E4098950C08A4570020F0B52DED01
:1076F000028B8BB0002307930893099305AB0446D4
:10770000019300F5935007AB009302AA04AB03A9C1
:1077100008300DF0E1FF04F50056054686F8600CD0
:1077200028B9002528460BB0BDEC028BF0BD83F0D4
:1077300015F9D6F8643C9FED2F7AC31A07EE903AFC
:10774000F8EE677A074667EE877A04F5305006AAA6
:1077500002A93C30CDED067A4EF0D4F904F5315053
:1077600006AA03A908308DED020A4EF0CBF904F504
:10777000315006AA04A914308DED030A4EF0C2F967
:1077800096ED688AC6F8647CB5EEC08AF1EE10FA10
:10779000C7D9DDED080A9DED070AA5F0D1FCDDEDA6
:1077A000090AA5F0CDFCDDED037A38EE087AB4EED7
:1077B000C08AF1EE10FAB4EEE77A94BF01230023F9
:1077C000F1EE10FA0AD80233DDED027AB4EEE78A60
:1077D000F1EE10FA0AD8002BA3D0A3E7B4EEE78AA3
:1077E000F1EE10FA9CBF0133DBB2EDE7012B99D823
:1077F00097E700BFBD37863570B500F500550446E4
:1078000095F8AD3E43F0040385F8AD3E4CF0A4FC82
:10781000012211214CF0FCFBD5F8B83E93F8CB3097
:10782000002B41D0D5F8940E03681B6898470928AF
:107830000AD1204607F0BEFA30B104F5A04010305E
:10784000BDE8704007F09EBA184BD3F8940E036859
:107850001B69984740B995F99D31032B24D1062126
:10786000204607F093FA0DE095F99D110229F6D113
:1078700095F8AD3EDB07F2D40622204601F0F4FF76
:107880000028ECD00A4BD5F8940E01225A730368F5
:107890001B6C9847034604F53150064ABDE870401A
:1078A00002212C304EF0F8BC70BD00BFB84B002058
:1078B0009D800020CC950C0808B500F5005292F888
:1078C000AD3E590717D56FF3820382F8AD3E0A4BE0
:1078D0005A7B42B1002200F531505A730221074A07
:1078E0002C304EF0D9FC4CF037FCBDE808400022AB
:1078F00011214CF08DBB08BD9D800020F0950C0837
:10790000F0B5054685B005F593576846083713F07E
:10791000E7FC694638460DF0BBFF80B105F5005322
:10792000D3ED687A374CF5EEC07AF1EE10FA08D84C
:10793000354A002328462380D373FFF7BDFF05B0E7
:10794000F0BD2846FFF7D2FE064628460BF0A6F902
:1079500010B928460BF07CF9A378002E18BF002040
:107960000343DBB2A370002BE9D06378A8BB83BBD1
:1079700023780133DBB2082B237003D14EB3384692
:107980000DF016FF2378092B02D138460DF008FFC1
:107990002378092B1DD94FF4857323804CF0DCFB31
:1079A000022210214CF034FB82F0E4FF6368C01A1D
:1079B00047F23053984209D905F53150134A022154
:1079C0002C304EF069FC82F0D5FF60602846FFF74E
:1079D00013FF0D4B6278DA73B1E72678002EF8D0EA
:1079E000013EF6B22670002BF3D0002EF1D1667066
:1079F0004CF0B2FB324610214CF00AFB2846FFF750
:107A00005BFFE6E7287F00209D80002008960C0899
:107A100000F5005393F8AD3E5B0701D5FFF7ECBED0
:107A20007047000073B5044600F5935001A9083073
:107A300004F500550DF09AFCD5F8283C8342064623
:107A40000CD004F58043D3F8380975F065FFC5F80C
:107A5000286C4CF081FB3E214CF0BAFA04F58056BC
:107A600095F92C1C96F9782596F8783591421BD01B
:107A7000FF2B19D004F58043D3F8380975F04CFF7B
:107A800096F8783585F82C3C4CF066FB95F82C2C54
:107A900018214CF0BDFA04F5315095F92C3C034AFD
:107AA00004212C304EF0F8FB02B070BD18960C0883
:107AB0002DE9F0438FB0054682F05CFF002305936B
:107AC00006930793089309930A930B930C930D93D2
:107AD00005F5935804AB019308F1080803AB009334
:107AE00006460BAB08AA05A940460DF0D5FDDFED13
:107AF000477A9DED077AB4EEE77AF1EE10FA074681
:107B000030DB9DED0A7AB4EEE77AF1EE10FAACBF05
:107B10000124002405F50059404699F8603C002BEB
:107B200008BF00270DF0CAFD8046EFB9444699F919
:107B30002C3A012B29D164B1D9F8B83E93F8CB4047
:107B40003CB1D9F8940E03685B69984780F0010056
:107B5000C4B299F8303CCBBBCCB9C9F8346C0FB087
:107B6000BDE8F0830024D5E7002CDFD005F53150C7
:107B700008304DF023FF90ED007AF7EE007AB4EE76
:107B8000E77AF1EE10FAD2DCD0E70024E1E7D9F889
:107B9000340C301AB0F57A7FE1D9C9F8383C0124A9
:107BA00005F5804389F8304CD3F8403983F80C440C
:107BB0004CF0D2FA22461D214CF02AFA144A05F55F
:107BC000315002212C304EF067FBC8E714B1C9F8E0
:107BD000386CC4E7D9F8380C43F69823361A9E421D
:107BE000BDD905F58043C9F8344C89F8304CD3F839
:107BF000403983F80C44C9F8384C4CF0ADFA2246B1
:107C00001D214CF005FA034AD9E700BF00000034FB
:107C100030960C084A960C080B4B10B5012204460E
:107C20005A7282F0A7FE04F58042D2F86C3AC31A69
:107C3000142B08D9C2F86C0A04F590501430BDE832
:107C400010403FF0DFBF10BD9D8000202DE9F743BD
:107C5000044604F5005500F50650002318300DF1D8
:107C600007018DF8073043F029FCD5F8B80E90F9DC
:107C7000C030026883B3083BDBB2012B96692BD975
:107C80003221B04704F1100011F036FA1F4B04F511
:107C900031581F684FF0000908F12C08F86A036892
:107CA000DB69984701281CD182F064FE41F28733DA
:107CB000A0EB09029A42064605D9154A062140461C
:107CC0004EF0EAFAB1462046FFF7A6FFB86A03680D
:107CD00003215B689847E1E79369B5F8AC119847D1
:107CE000D0E70121D5F8B80E7BF03AFCD5F8B80EF4
:107CF0000368DB6A984757F089FDF86A03681B68D8
:107D0000012103B0BDE8F043184700BFE07E00202A
:107D100068960C0870B5044600F531502DED028BC5
:107D2000174A184E9FED188A06212C304EF0B4FAEF
:107D30002046FFF78BFF2046FFF76EFF20460AF034
:107D400007FD3368986A036803215B68984758F019
:107D5000BFF8054658F056F804F50053D3F8D02A7A
:107D6000D3F8B80EB2F9082000EE102AB8EEC00A17
:107D700020EE080A7DF0CEF8284658F04BF8DAE7F6
:107D80008C960C08E07E00206F12833A2DE9F047B4
:107D9000044600F531502DED028B2A4ADFF8AC90F5
:107DA00006212C304EF078FA2046FFF74FFF58F0AE
:107DB0008FF804F50056054658F024F8B7EE000A8F
:107DC000D6F8B80E7DF0A6F8284658F023F882F0D1
:107DD000D1FD41F2873A074682F0CCFDC01B5045E9
:107DE000D9F8008017D99FED188A284658F00AF86C
:107DF000B0EE480AD6F8B80E7DF08CF8284658F058
:107E000009F82046FFF708FFD8F828000368032187
:107E10005B689847E9E7284657F0F4FFB7EE000A99
:107E2000D6F8B80E7DF076F8284657F0F3FF2046D6
:107E3000FFF7F2FED8F82800036803215B68984733
:107E4000CAE700BFBC960C0800000000E07E0020DE
:107E50002DE9F34100F500550446D5F8B83E93F9F5
:107E6000C030032B29D0354F652600F58048013EF0
:107E700016F0FF060CD0D8F8683A4BB93B68986A00
:107E8000036814215B68984720460AF061FCEEE71E
:107E900004F52F5001212C30F9F77AFE95F998312D
:107EA00070B953B1092B08D08DF8070004F50650BE
:107EB0000DF10701183043F001FB02B0BDE8F0817D
:107EC000032B34D8DFE803F002252D30D5F8D03A63
:107ED000B3F9082040F2B5339A422ADD04F5065082
:107EE00001250DF1070118308DF8075043F0E6FA2F
:107EF00004F53150124A02212C304EF0CDF9114BCD
:107F00005D720E4B1C68A06A036805215B68984788
:107F1000F9E7D5F8D03AB3F9082040F2B5339A42E0
:107F200007DD2046FFF7F6FE2046FFF72FFF092B5F
:107F3000C3D000238DF80730B8E700BFE07E0020F3
:107F4000E0960C089D80002000F531500B46024A57
:107F500004212C304EF0A0B900970C0810B504464F
:107F60004CF0FAF8002205214CF052F804F531509B
:107F7000034ABDE8104004212C304EF08DB900BFFB
:107F80000C970C0813B50B464AB100F5315000921E
:107F90000421054A2C304EF07FF902B010BD02B02A
:107FA000BDE81040FFF7D0BF24970C0808B500F5D6
:107FB0003150064A04212C304EF06EF94CF0CCF8CA
:107FC000BDE80840002208214CF022B838970C0880
:107FD00038B504460D4682F0CDFC04F500533DB99A
:107FE000D3F8A42EC3F8A80E0AB9C3F8A40E38BD5E
:107FF000D3F8A82E801A642882BF0022C3F8A82EC6
:10800000C3F8A42EF3E7000037B5044600F592400C
:108010001C307AF0EBFA04F50052C0F3803592F888
:108020008A3EC3F34001A9421DD065F3410304F524
:10803000315482F88A3E2C346DB14CF08DF8022216
:108040000B214BF0E5FF094A0221204603B0BDE8B1
:1080500030404EF021B94CF07FF82A460B214BF00E
:10806000D7FF034AF0E703B030BD00BF50970C08BC
:108070006C970C0838B50A460C460621054601F0F7
:10808000F3FB28B1054A137843F00803137038BD99
:1080900021462846BDE8384006F078BEBC80002066
:1080A00038B50A460D461521044601F0DDFB28B11E
:1080B000094A137843F00803137038BD04F53150B2
:1080C00004212C30054A4EF0E7F829462046BDE849
:1080D000384006F05BBE00BFBC8000207C970C08D7
:1080E00038B50A460D461521044601F0BDFB28B1FE
:1080F000094A137843F00803137038BD04F5315072
:1081000004212C30054A4EF0C7F829462046BDE828
:108110003840FFF7AFBF00BFBC800020A4970C0819
:1081200038B50A460D461B21044601F09DFB28B1D7
:10813000094A137843F00803137038BD04F5315031
:1081400004212C30054A4EF0A7F829462046BDE808
:108150003840FFF78FBF00BFBC800020BA970C08E3
:1081600038B50A460D461121044601F07DFB28B1C1
:10817000094A137843F00803137038BD04F53150F1
:1081800004212C30054A4EF087F829462046BDE8E8
:10819000384006F0FBBD00BFBC800020CC970C0827
:1081A00010B500F5005494F88A3E9A0623D4D4F80A
:1081B000940E03681B689847032808D005D8022846
:1081C0000ED194F8880EC00914E01B28F9D194F858
:1081D000880E00F0A000A0F180035842584109E049
:1081E000B4F8880E20F4FE4020F07F0080B2003802
:1081F00018BF012010BD0120FCE7000038B500F5D4
:108200000055044695F8AD3E184A43F0080300F5C2
:10821000315085F8AD3E02212C304EF03DF84BF048
:108220009BFF012217214BF0F3FE2046FFF7B8FF1A
:1082300040B104F52F500122BDE8384015212C3003
:10824000F9F7B2BED5F8940E03681B689847062864
:1082500006D104F5A2402830BDE8384007F09CBFA5
:1082600020460B21BDE83840FFF704BFE0970C081B
:1082700070B500F500550646D5F8A42ED5F8A83EF1
:108280009B1A41F28832934211D9D5F8940E0368B3
:108290001B6D9847044695F8AD3EC3F3C003A34257
:1082A00013D034B13046BDE87040FFF7A7BF0024BB
:1082B000F1E74BF051FF224617214BF0A9FE95F84C
:1082C000AD3E64F3C30385F8AD3E70BD0B46013B84
:1082D0001146062B18D8DFE803F00406080A0C1331
:1082E000150006F053BDFFF7C5BEFFF7F9BEFFF757
:1082F000D7BE00F52F50012214212C30F9F754BEBF
:10830000FFF70EBFFFF72CBF7047000070B50446A3
:1083100004F500554BF020FF012205214BF078FEBB
:1083200095F88231072B98BF304A204694BFD65C1F
:108330000126FFF735FF68B12D4A2E492046FFF789
:1083400021FE04F52F50012210212C30F9F72CFECC
:10835000002614E0D5F8940E0368DB6C9847A8B1AA
:1083600004F5405393F80D2482B193F90C34012B9A
:108370000CDC214A21492046FFF704FE0126314644
:1083800020460322BDE87040FFF7A0BFD5F8940E49
:108390000368DB6C984718B1D5F8303A190715D443
:1083A000D5F8940E03681B689847032803D1D5F8C5
:1083B000303ADA070DD4D5F8940E03685B6A984713
:1083C00068B90C492046FFF7BFFDD8E70A4A0949BA
:1083D000D1E70B4A07492046FFF7D4FDB8E7D5F8A7
:1083E000303A5B07EDD5074AF4E700BFC8980C08A0
:1083F00000980C080A980C0810980C0823980C0890
:1084000033980C0843980C0870B5044615464BF099
:10841000A3FE012206214BF0FBFD2046FFF7C0FE24
:1084200098B104F52F50012207212C30F9F7BCFD3B
:10843000134A14492046FFF7A5FD0025294620468A
:108440000422BDE87040FFF741BF04F50056EDB2CD
:10845000D6F8940E0368DB6C984758B1D6F8303ADA
:108460001B0707D535B1084A06492046FFF78AFDA4
:108470000125E3E703492046FFF766FDDEE700BF7D
:1084800000980C0862980C0810980C08F8B504467F
:1084900004F500554BF060FE012208214BF0B8FDB9
:1084A00055F014FF95F87131072B9CBF364AD65C06
:1084B000D5F8B83E93F8CB7088BF02265FB9334930
:1084C0002046FFF741FD0026314620460522BDE843
:1084D000F840FFF7FBBE2046FFF762FE60B104F5EF
:1084E0002F50012212212C30F9F75EFD284A27492E
:1084F0002046FFF747FDE6E7D5F8940E0368DB6CEE
:10850000984778B104F5405393F80D2452B193F98C
:108510000C34012B06DC1F4A1F492046FFF732FDB1
:108520000126D1E7D5F8940E0368DB6C984718B1A3
:10853000D5F8303A190713D4D5F8940E03681B68A0
:108540009847032803D1D5F8303A9A070BD4D5F8C9
:10855000303ADB0609D40D492046FFF7F5FCB3E7B6
:108560000C4A0A49D9E70D4AC1E7D5F8940E0368C9
:10857000DB69984705460028EDD1094A03492046A2
:10858000FFF700FD2E469FE7D0980C084B840C089F
:1085900000980C0810980C085C980C086A980C0855
:1085A0007F980C0870B500F50055044695F97131B7
:1085B000ABB3D5F8186E96B382F0DCF905F68823D4
:1085C00093ED000ADFED167A9FED161ADFED160A1D
:1085D000861B20EE270A8D2023F088FEBCEEC00A01
:1085E00010EE103A9E420CD295F8AD3E9A0716D581
:1085F00020460021F9F732FE2046BDE87040FFF723
:10860000D5BC0CD995F8AD3E9B0708D42046012176
:10861000F9F724FE2046BDE87040FFF737BF70BD74
:1086200000007A440000804F000000002DE9F34173
:10863000074600F592401C3079F0D8FF07F500544A
:10864000C0F38048019082F095F994F8B03E43451C
:10865000454606460DD007F5315084F8B08E2C30D3
:10866000002D3FD03A4B3B4AC4F8B46E02214DF086
:1086700013FE94F8B03E43B394F8B13E2BBBB4F96B
:108680009E3A9FED350A9FED351ADFED350A07EE6C
:10869000903AF8EEE77A40F2571027EE800A23F07E
:1086A00025FEBCEEC00AD4F8B40E10EE103A361A0D
:1086B0009E420AD9012307F5315084F8B13E294A78
:1086C000234B02212C304DF0E7FD94F99D3A002B0D
:1086D00094F8AD3E0DDC6FF3451384F8AD3E02B067
:1086E000BDE8F0811A4B204AC4F8B48E84F8B18EEC
:1086F000BCE7C3F34012AA42F1D065F3451384F8F6
:10870000AD3E9B06EBD5194BD3F8940E03681B695D
:1087100098470028E3D04BF01FFD01221F214BF0AA
:1087200077FC3846FFF73CFD48B107F52F50012292
:1087300021212C3002B0BDE8F041F9F735BC94F8A6
:108740009D1A3222384602B0BDE8F041FFF7BEBDA7
:1087500098980C08A7980C0800007A440000804FF5
:1087600000000000BD980C08B2980C08B84B00201F
:1087700008B5044B01221A7082F0F0F8024B186021
:1087800008BD00BF317F0020347F0020014B002254
:108790001A707047317F00202DE9F041044682F0C5
:1087A000DDF82A4BB4F8BE201988294E91420546BF
:1087B0000ED01A80274B18603378A3B10024347090
:1087C0004BF0CAFC22461321BDE8F0414BF020BC1F
:1087D0003378214FDBB93B782BB11E4B1F4A1B6806
:1087E000C31A934201D8BDE8F0810123337004F528
:1087F0000053D3F8B80E90F8CB3013B103689B6ADE
:1088000098474BF0A9FC012213214BF001FC3B7867
:10881000002BE8D03378002BE5D00E4A10491368BE
:10882000EB1A8B42DFD904F500541560D4F8B80E6A
:1088300090F8CB30002BD6D000217AF091FED4F8FE
:10884000B80E0368BDE8F0415B6A1847327F00202C
:10885000307F0020347F0020317F002080841E0084
:1088600040420F002DE9F04100F500550446D5F8CF
:10887000940E95F884700368DB6C9847014650B9F4
:1088800095F9883E002BA5BFD5F8B83E93F8CB00EC
:10889000012180F0010104F5015808F10808404663
:1088A0005FF034FCD5F8B83E93F8CB300646002B89
:1088B0007BD0002865D03E4B93F9883E002B04DB2B
:1088C00002463C4940465EF0FBFF95F94E7057B1B9
:1088D00095F9883E002B0EDA04F52F5001220F2166
:1088E0002C30F9F761FB4BF037FC3246BDE8F04124
:1088F00009214BF08DBBD5F8940E03685B6998474E
:1089000058B195F9893E002B07DA95F8AD3EDA07A4
:1089100003D495F88430DB07DED5314640465FF05E
:108920005BFCDFED257AB4EEE70AF1EE10FA05DD27
:108930000A220921204600F097FFD4E7023F032FC7
:1089400011D801A353F827F031890108598901088A
:10895000778901087D8901080A221521204600F047
:1089600083FF0028BFD10A220621204600F07CFFA9
:108970000028B8D1DCE70A221121F6E70A221521E6
:10898000F3E797B195F884307BB9094B93F9883EAA
:10899000002B06DB04F53150084A05212C304DF040
:1089A0007BFC4BF0D9FB0022A0E7BDE8F08100BFC3
:1089B000B84B0020D8980C080000C842E1980C0879
:1089C00070B500F5005300F592451C3586B093F85C
:1089D000301C0446284679F0B7FD02A812F080FC4E
:1089E00004F5935002A908300CF002FF04F580430F
:1089F000049AC3F81429059AC3F81829284679F06F
:108A0000F5FD82061AD5284679F0FEFD04F592455B
:108A1000FDEEC07A0C3504F5805417EE901A022250
:108A2000284617EE906A12F061FC94F8E434DB07F4
:108A300006D401223146284612F058FC06B070BD1B
:108A40000121284612F0E4FC0028F2D0F6E70000ED
:108A500070B500F5804486B0B4F89C3A8B420D4660
:108A6000164603D1D4F8983A934221D081F082FF80
:108A7000D4F8943AC31A132B1AD9C4F8986AA4F8F4
:108A80009C5AC4F8940A4BF067FB044681F07AFFC5
:108A9000084B094A1B68CDE90453084B0193084B66
:108AA0000093CDE90201074B074920464BF0E0F85F
:108AB00006B070BD387F0020F8980C0810990C089B
:108AC000D06E0C080C520C080B990C0838B500F548
:108AD00000540D4694F8893EC3F380138B420BD0AB
:108AE00021B14BF039FB11214BF072FA94F8893E19
:108AF00065F3861384F8893E38BD0000F0B52DED8E
:108B0000048B00F500558BB0D5F8B83E93F8CB3008
:108B1000064600F58044002B67D095F9883E002B6F
:108B200063DBD5F8940E03685B699847002861D130
:108B3000D4F838099FED430A6C3026F0DBFD0AAA11
:108B4000CDED080A8DED091A8DED070A12E907002F
:108B500004AB01AF83E8070087E80700384626F03A
:108B600037FBD4F8383906F591406C30D3ED368AAE
:108B7000B0EE409A4CF046FF27F0BAF9D4F84039ED
:108B8000D5F8940ED3EDDB9A0368DB6CB0EE408A27
:108B90009847DFED2D7AB4EEE79AF1EE10FA02DC99
:108BA00095F8903E0BB1002838D0DFED287A68EEBA
:108BB000A78AF3EE0E7AF4EEE78AF1EE10FA2DDCD6
:108BC000F0EE087AB4EEE78AF1EE10FA26DCF5EE64
:108BD000C09AF1EE10FA21DAD4F8380903689B6FD5
:108BE00098470BB0BDEC048BF0BDD4F8380903688E
:108BF0009B6F0DE0D5F8D02AD4F83809B2F90820D7
:108C00000368002A03DCD5F88C2E022AF0D1DB6F32
:108C10000BB0BDEC048BBDE8F0401847D4F83859D0
:108C2000DFED0B0A2B68D3F88060D4F8403940F2AE
:108C3000AB1093EDC90AB7EE001A23F057FB284694
:108C4000B047CEE79F0CB3450080BB44E02E6542A1
:108C50000000000000F5005090F8900E70470000F2
:108C6000F8B500F50054064694F8883EB1EBD31FE2
:108C70000D4644D0224B00221A6000293BD04BF015
:108C80006BFA12214BF0A4F994F8883E65F3C713F0
:108C900085F0010784F8883E6AF0FEF839466AF0EC
:108CA000D7F837B194F806311BB981F063FEC4F8E8
:108CB000080184F8067115B3B4F854315B071ED56A
:108CC000D4F8B83E93F8CB30CBB1D4F8940E036807
:108CD0005B69984798B9D4F8940E036820219B6982
:108CE000984760B106F52F500122BDE8F8400D21EC
:108CF0002C30F9F759B94BF02FFA1C21C2E7F8BD17
:108D0000387F00202DE9F04F2DED0A8B00F500553E
:108D10008DB0D5F8B83E93F8CB60044600F5804797
:108D20001EB90121FFF79CFF0BE095F9882E002A60
:108D300065DAD5F8940E03689B6C984706460028C0
:108D400041D04FF0000B95F9882EB24E002AC0F2A8
:108D50005581D6ED007AB4F9A420B8EE677A1AB935
:108D6000B4F8A220A4F8A420B4F8A430DFEDAA6AD5
:108D700007EE903AF8EEE77A67EEA67AB4EEE77A75
:108D8000F1EE10FAACBF012100212046FFF79EFE54
:108D900095F9882E002A95F8892EB8BF4BF0010B63
:108DA000530697F8802A48BF4BF0020B0AB14BF0EC
:108DB000080B3268594620460DB0BDEC0A8BBDE861
:108DC000F04FFFF745BED5F8B83E204693ED0C8A2C
:108DD000F9F714FBB4EEC80AF1EE10FAB1D5D5F8E4
:108DE000B83E93F8A130032BABD149F0C1FC4FF44E
:108DF0008011422249F074FC3146204692E797F8F0
:108E000080AABAF1000F03D0824A0023136098E7CA
:108E1000D7F8380993F8079003685B6F9847804646
:108E20000090D5F8940E03685B69984720B1D5F897
:108E30008C3E022B00F0E480B9F1000F0CBF4FF024
:108E4000000B4FF4007BB7EE00BAB8F1000F02D070
:108E50004BF4806B009604F5944808F148084046AE
:108E600062F032FB0130D7F838099FED6C0A9FEDB4
:108E70006CCADFED6C8A0CBF012302236C3008EE54
:108E8000103A26F037FC0CABCDED0A0A8DED0B1A2B
:108E90008DED090A13E907000DF10C0E0DF1180C08
:108EA0008CE807008EE80700704626F091F9D7F8A5
:108EB0003829DFED5D7A92ED36AA2AEE27AAB4EEC4
:108EC000CC0AF3EE0EBAF1EE10FA04F59140B4EECE
:108ED000EBAAC8BF4BF4807B6C30F1EE10FAC8BF30
:108EE0004BF4807BF0EE40AA4CF08CFD27F000F8AC
:108EF000B8EEC88A04F59240B4EEC80AF1EE10FA52
:108F000000F11C0098BF4BF0800BF0EE409A79F016
:108F100087FB68EE288AB0EEC09AB4EEE89AF1EECC
:108F200010FA204648BF4BF0400B09F0F7FC002830
:108F300046D14BF0200B0196404662F0C5FA01285D
:108F40004FD14BF0100BB2463249B9F1000F53D05C
:108F5000009B002B50D0F4EECCAAF1EE10FA4BDCC3
:108F6000B4EEEBAAF1EE10FA46DCF4EEC89AF1EE9C
:108F700010FA41D8B4EEE89AF1EE10FA3CD5019B14
:108F8000D3B3BAF1000F37D00A68B4F9A40007EEE2
:108F9000902AB8EE677A18B9B4F8A200A4F8A40031
:108FA000B4F8A43007EE903AF8EEE77A67EE8B7AE1
:108FB000B4EEE77AF1EE10FA19D501320A60C2E692
:108FC00004F52B502C304CF0F9FCDFED187A90EDC5
:108FD000007AB4EEE77AF1EE10FAAAD400230193F6
:108FE000AAE7404662F070FA0130ADD1A9E701214D
:108FF0002046FFF735FEA6E60022DFE70121C4E6A2
:10900000B9F1000FB0EE08BA0CBF4FF0000B4FF4EF
:10901000007B1DE7387F0020CDCC4C3E9F0CB34534
:109020000080BB440000C842E02E65420000484377
:1090300030B500F5AD531833044693E8070089B006
:1090400002AD85E807009FED1D7ADDED047A77EE2D
:10905000877A9FED1B7ACDED047AD4ED2B7AF0EE72
:10906000E77AF4EEC77A04F59140F1EE10FA00F1D8
:109070006C000BD5B4F9A23007EE903AF8EEE77A1F
:10908000F7EE006A86EEA77A84ED2B7AD4F8AC303E
:10909000019301AA29464CF05BFD2046FFF732FE02
:1090A0002046FEF781F92046FEF758FA2046FEF7E3
:1090B00021F82046FEF7C8F809B030BD0AE81C4187
:1090C0000000003410B504462DED028B1D2056F033
:1090D0001DFD60B304F50053D3F8940E00F0C2FAFE
:1090E000192108EE100A04F5516042F083FE0228AF
:1090F0001AD00338012808D804F52B502C304CF036
:109100005DFC90ED008ABDEEC88AB8EEC88A9FED7E
:10911000090A28EE000ABDEC028B04F594404830A1
:10912000BDE8104062F056BA9FED038AEDE7BDEC52
:10913000028B10BD0AD7233C00000000134A0260D6
:10914000134A426002F1740181601249C16002F564
:10915000205101610839416124398161A2F56E61B4
:10916000C1610D49016202F55761416202F5186162
:10917000816202F68411C16202F6881102F68C1235
:109180004263064A01638263704700BF44AA0C0829
:10919000004D0020FC740020F0740020D02C002032
:1091A0001C2953D8DFE801F0130F171B27232F1FAB
:1091B000522B52335252373B3E424652524A52523F
:1091C000525252524E0000F595402430704700F53F
:1091D000A3403430704700F595406430704700F587
:1091E00096402030704700F59D407C30704700F578
:1091F000A0405830704700F59F404C30704700F554
:10920000A0401030704700F5A2402830704700F5AC
:109210009E403C30704700F59E407830704700F526
:109220009940FAE700F5A1401430704700F59D40E1
:109230003830704700F5A3407030704700F5A44007
:109240004030704700F5A5405C3070470020704703
:1092500073B50B6805461B6C08460C4616469847C6
:10926000034605F531500F4A009604212C304DF08D
:1092700013F84AF071FF236805461B68204698479B
:109280000A21024628464AF0C3FE074B93F8893E5E
:109290009B0641BF054A137843F00403137002B0E4
:1092A00070BD00BF14990C08B84B0020BC80002092
:1092B00038B50C4A182305460C4649F0CBF878B16E
:1092C00021462846FFF76CFF30B10146064A284682
:1092D000FFF7BEFF002038BD284649F001F8F9E746
:1092E0000120F8E794990C0834990C0810B500F5A2
:1092F0000054002384F8803B084B00F5804093F82D
:10930000881ED0F83809C90972F0B2FFD4F8940E5B
:109310000368BDE81040DB68184700BFB84B002069
:1093200070B50546086803685B690C4616469847A1
:1093300090B1306803685B69984768B905F50053D8
:10934000D3F8B82E92F8CB2032B193F9883E002B97
:1093500002DB2846F9F768F804480AF093F8206819
:109360000368BDE870409B68184700BFF87F002085
:1093700070B500F500550446D5F8940E0B4E036801
:10938000DB6998473074D5F8940E03681B689847DA
:10939000F070D5F8940E03685B6C9847014604F5AD
:1093A00090501430BDE870403EF076BC9D800020A7
:1093B00070B52DED028B244B93F8AD3EDB0782B0E8
:1093C00006460D461446B0EE408AF0EE608A06D599
:1093D00000232B60236002B0BDEC028B70BD55F002
:1093E00075F8037F002BF3D0F36A9FED181A1B6802
:1093F0009FED170AB3F9083007EE103AB36A1B68FD
:10940000B3F9083007EE903AB8EEC77AF8EEE77A8B
:1094100067EE000A68EE811A27EE800A28EE011A2C
:1094200001A9684623F04CFEDFED0A6A9DED007A43
:10943000DDED017A27EE267A67EEA67A85ED007AD1
:10944000C4ED007AC7E700BFB84B00200AD7233C21
:10945000530469390000C84270B52DED028B88B005
:10946000002302930393364B93F8AD3E13F0010FA4
:109470000646B0EE408A06AD02AC03D155F026F8A0
:10948000037F5BB994E8030085E803009DED060ABD
:10949000DDED070A08B0BDEC028B70BDB36ADFEDED
:1094A000296A1B68B3F9083007EE903AF36A1B6823
:1094B000B3F9083007EE103AB8EEC77AF8EEE77A5B
:1094C00027EE267A67EEA67AF1EE476ACDED026ABC
:1094D000DFED1D6ACDED037AB0EEC77AB4EEE67A21
:1094E000F1EE10FA06D5F0EEE77AF4EEE67AF1EE58
:1094F00010FAC7D403AA21461448F8F7C5FFDDEDDA
:10950000027A9DED037AF0EEE77AB0EEC77AF4EED8
:10951000477AF1EE10FACCBFB0EE670AB0EE470A18
:10952000204625F0A3FD04A88DED040ACDED050A23
:1095300025F04EFE204688EE000A25F0C7FDA1E783
:10954000B84B00205304693900000034B82B0020C8
:10955000094B93F9882E002A0CDAB5EEC00AF1EE19
:1095600010FA07D9D3F8B83E93F8A100C31E5842A9
:109570005841704700207047B84B0020436A1B6871
:1095800093F8CB3043B1054B93F8880E00F0A00060
:10959000203818BF0120704701207047B84B0020C9
:1095A00010B5436A04461868D1B1022179F0E8FF8A
:1095B000236A9FED0C1A18680368F0EE410ADB6A13
:1095C000B0EE410A9847236A074A1868D2ED540A58
:1095D00003689FED040A5B6EBDE810400021184748
:1095E0000121E3E700000000B84B002010B5436AFA
:1095F00004461868002930D0022179F0C1FF236A9F
:10960000186872F005FE636A1B6893F8A130012B9D
:1096100004D8236A0121186873F094FB6369186801
:1096200076F0A0FC6369186876F0FCFC63699FED36
:109630000C0A186876F022FF6369186876F090FFCC
:10964000236A9FED071A18680368BDE81040DB6ABB
:10965000F0EE410AB0EE410A18470121CDE700BF04
:109660000000000013B5044601A90C4809F0E0F918
:1096700010B1019802B010BD6369186875F07CFBE9
:1096800018B9074BD3F81009F4E7064801AA0321DB
:1096900011F062FE0028F4D0EBE700BFB82B0020E9
:1096A000B86B0020C474002070B504462DED028B09
:1096B00000296AD18368B3F96258642DB8BF642564
:1096C000FFF7D0FFA8426268A4BF324B93F8895ECF
:1096D000B2F93430ACBFC5F380150125002BDBBFD8
:1096E00063691B685B4293EDC48AC8BF07EE903A7A
:1096F000B2F93230C8BFB8EEE78A002BB8BF5B4280
:109700009BB25B4207EE903AA368F8EEE77AB3F9B2
:109710006268F4EEC87AF1EE10FAD8BFB0EE678A4C
:109720002046642EB8BF6426FFF79CFF6369A26BD6
:109730001B68D2ED001A93EDC61AD3ED0E0A311A4A
:1097400000EE101AB8EEC00A23F0A8F86368B3F967
:109750003230002BB8BF5B429BB25B4201EE103A45
:1097600040F29720B8EEC11AF0EE480A22F0BEFD92
:1097700063692946186875F0A3FBBDEC028B636929
:10978000BDE87040186876F0EBBE9FED030A002537
:10979000EEE700BFB84B002000000000436A1868E5
:1097A00003681B691847000038B52DED028B03686C
:1097B0000446D3F880309847236B2A481B68F0EEA4
:1097C000408AB3F9085009F049F84FF47A72041E40
:1097D0004FF000012846D8BF4FF4FA7422F0C4FDC0
:1097E0008442B6EE000A2ADD07EE900AB8EEE77A68
:1097F00007EE904A27EE007AF8EEE77A87EE278A9E
:109800004FF46D7038EEC00AF5EE087AB1EE400AFA
:1098100080EE270AB7EE001AFEEE000A22F066FD7F
:10982000F7EE007A77EEC07A28EE000A20EE080AFA
:1098300020EE080AA7EE880ABDEC028B38BD031B98
:1098400007EE103AC4F57A74B8EEC77A07EE904A7C
:1098500027EE007AF8EEE77A87EE278A38EE008A5C
:10986000CEE700BFB82B00202DE9F04F2DED028B85
:1098700000F5804900F5005599F8A04A89F8A02A1A
:109880000646D5F8940E036883B01B6888461746D1
:10989000984740451FD11A2F85F8047107D130B978
:1098A00005F66425D9F838392A68C3F8FC208B4BB3
:1098B00093F8893E980606D40124204603B0BDECF7
:1098C000028BBDE8F08FBC42F6D0854A137843F096
:1098D00002031370F0E7022F0DD0B8F11B0F12D165
:1098E00006F596403946203003B0BDEC028BBDE84A
:1098F000F04F01F053B941463046FFF7D9FC04461A
:109900000028EAD1D9E741463046FFF749FC044632
:10991000019018B9304648F0E3FCCEE7D5F8B83EE0
:1099200093F8CBB003685B699847019A06F59E43AC
:109930003C338BF0010A9A4208BF0120BBF1000FB3
:1099400008D10198036851465B689847044648BBB4
:10995000644A22E095F9883E002B80F2B18000280D
:1099600000F0AE80DFF874B1DBF8940E03685B6939
:1099700098470446002840F0A3800198FFF714FFA1
:10998000ABF50050B0EE408AF8F738FDB4EEC08A6F
:10999000F1EE10FA40F39480534A01993046FFF7F4
:1099A00057FC8AE706F53A5101AA14313046FFF711
:1099B000B7FC0198C5F8940E85F8047103681B681C
:1099C00098473A46014606F57C6049F0D7FE06F511
:1099D000315000212C3053F0B1FE95F94E3023B1B7
:1099E00006F5015008305EF01BFCD5F8940E0368B4
:1099F0001B689847C21E5042504105F6342289F830
:109A0000C809D9F838391268C3F8F82005F6642275
:109A1000D9F838391268C3F8FC20B8F1010F02D028
:109A2000B8F10B0F06D105F64C25D9F838392A685C
:109A3000C3F8FC203046FFF79BFC284B93F8893E87
:109A40009B063FF542AF37E795F84830002B3FF4CF
:109A500078AFB5F86430D9077FF573AF95F88430E7
:109A6000002B3FF46EAFD5F8B83E93F8CB30002B07
:109A70003FF467AF95F804310A2B7FF462AF95F994
:109A8000883E002BFFF65DAF184A01993046FFF77C
:109A9000DFFB002411E7164809F040F90028D3D174
:109AA000D5F8940E03685B6998470028CCD00198DC
:109AB00003685B69984704460028C5D10D4A6CE7E6
:109AC000019803681B6998470028E4D0084809F00A
:109AD00013F904460028DED1074A5EE7B84B0020A0
:109AE000BC800020B6FB0D085C990C0880990C081E
:109AF000B82B00206E990C08C2AE0D080148FFF784
:109B0000B3BE00BFB82B002013B504468DED010A8B
:109B100061F072FC6369A26B1B6892ED001A93ED11
:109B20000E0AD3EDC60A01A960F0F4FA9DED010A10
:109B300002B010BD436A186803685B6A18470000EA
:109B400038B5436A1C6894F8CB10054661B92046C5
:109B500079F016FD6B6A1B6893F8A10018B1012813
:109B600014BF0320022038BD164803783BBBFFF723
:109B7000EFFC20BB144A92F8883E03F0A003202B90
:109B800017D0B5EEC00AF1EE10FA10D592F88A3E61
:109B90005B070CD40121204679F0F2FC6B6A1B684C
:109BA00093F8A130012B0CBF02200320DBE7022138
:109BB000F1E72046022179F0E3FC0420D3E70120FD
:109BC000D1E700BFF87F0020B84B002010B52DED85
:109BD000028B134B93F8AD3EDB07044604D59FED93
:109BE000110ABDEC028B10BD54F070FC037F002BFA
:109BF000F5D0636B186854F093FDA368DFED0A7A23
:109C000003F6AC0292ED008A03F50B63D3ED000A74
:109C100028EE278A23F00EFA28EE000AE1E700BFBB
:109C2000B84B0020000000000000C8420148F8F7CF
:109C300059BC00BFB82B00200148F9F7D5B800BFC8
:109C4000B82B00200148FFF70FBE00BFB82B002043
:109C500070B57E4D2DED028B95F8893E8CB00026B7
:109C6000044658060496059603D56369186874F08F
:109C7000F7FE95F8AD3ED9075DD463689B899A07D6
:109C80001BD573484BF09AFEDFED727A90ED007AA7
:109C9000B4EEE77AF1EE10FA0FDD4AF05DFA3D21FD
:109CA0004AF096F96C4809220521FFF7DDFD20B93D
:109CB000092202212046FFF7C5FF636893F954305B
:109CC000CBB365489FED658AF9F78EF8E3689FEDA1
:109CD000647A1B68D3ED0A7AF4EEC87AF1EE10FAD2
:109CE000B8BFF0EE477AB6EE000A27EE800A2046AB
:109CF000FFF7B2FB8DED040AB0EEC00AB4EEC80A5D
:109D0000F1EE10FACDED050A06D5F0EEE00AF4EE1C
:109D1000C80AF1EE10FA0ED495F88A3E1B0704D457
:109D20004AF01AFA49214AF053F995F88A3E43F06D
:109D3000080385F88A3E95F88B3E09966FF38203F7
:109D400085F88B3E60690A9609AE324604A9006820
:109D5000012374F0EFFE6369186876F063F96369B4
:109D6000186875F03BFAA3688DED060ACDED070A79
:109D70008DED081AD3ED007AF5EEC07AF1EE10FA07
:109D800051DDB5F944319FED378A00EE903AF8EE97
:109D9000E00A2046CDED030AFFF764FCA368DDED81
:109DA000030AD3ED001A9FED2B0AB7EE002A07EE47
:109DB000900A31EE822AB8EEE71A22EE082A61EE06
:109DC000881A22F0D3F9DFED287A20EE270ADFED9A
:109DD000277A20EE270AA3F083FADFED257A20EE1A
:109DE000270A06A820EE088A25F0F2F9B4EEC08A08
:109DF000F1EE10FA17D5C8EE006A63699DED067A98
:109E0000DDED077A27EE267A67EEA67A8DED067AE3
:109E1000CDED077A1B68D3F88823C3F89423D3F8D1
:109E20008C23C3F89823236A12491C683046FCF738
:109E300029FB0B9B009396E80C0006A9204672F0C4
:109E400099FA0CB0BDEC028B70BD00BFB84B00207E
:109E5000B874002000002F44B82B0020000000340C
:109E600000007A430000C8420AD7233C35FA8E3CF2
:109E70000AE81C41EC7E002013B504460191FFF76F
:109E8000E7FE0199204602B0BDE81040FFF70CBC88
:109E90000148FEF7E5BE00BFB82B00200048704720
:109EA000245800200148F8F70BBB00BFB82B002056
:109EB00030B50F4D87B0002304466946D5F84009F8
:109EC00000930193029375F0A1F9D5F8400902A916
:109ED00075F0F0F9009B0393019B04930222029B0F
:109EE000059303A9204611F007FD204607B030BDB9
:109EF000B86B00200020704700207047002070479A
:109F000000207047002070470020704700207047F5
:109F10000020704700207047002070479FED010A25
:109F2000704700BF0000000000207047002070470D
:109F300000207047012070470020704700207047C4
:109F400001207047002070470120704701207047B2
:109F500000207047012070470120704700207047A3
:109F600000487047AC990C0800487047AC990C0841
:109F7000836893F8C038DB0706D5002380F83C30AF
:109F8000024B0222C3F88C2E01207047B84B0020F0
:109F900090F83C3043B9836893F8C038DB0742BF80
:109FA000034B0122C3F88C2E002380F83C3070470D
:109FB000B84B0020012380F83C3070472DE9F04376
:109FC0002DED0C8BF0EE409A20EE000A97B00025A4
:109FD000A0EEA00A04468946B0EE41CAF0EE60AA9F
:109FE00090461F46019502950395049505950695A3
:109FF000A3F08CFBF7EE00CAB4EEEC0AF1EE10FA17
:10A00000C8BFCCEE807AA36803F67C0203F5086330
:10A0100092ED009A9FEDC5DAD3ED000AC4BF69EE58
:10A02000A79A6AEEA7AAB0EE690A23F003F8A3681C
:10A0300029EE0D9A03F67C0203F50863D2ED008A3F
:10A04000D3ED000A29EE009AB0EE6A0A22F0F2FF80
:10A05000A36868EE8D8A03F6940203F69803D3EDA5
:10A06000000A92ED008A68EE808AB0EE4C0A22F077
:10A07000E1FF636828EE0D8A93F9703028EE008ABC
:10A08000002B00F0D980236A9FEDA90A18686C3074
:10A0900025F030FBB0EE60AACDED080A8DED091A6F
:10A0A0008DED070A22F0CCF8BDEEC0BAA14940F60A
:10A0B000B8321BEE100A22F047F9434207EE903AFD
:10A0C0006368F8EEE77A93ED1A7A67EE877AB0EE76
:10A0D0004A0ACDED017A22F0B3F8FDEEC0BA40F69F
:10A0E000B83294491BEE900A22F02EF9424263687E
:10A0F000039507EE902A93ED1B7A93F97030F8EEF2
:10A10000E77A022B67EE877ACDED027A6ED18A4B21
:10A11000B3F944310AEE103AB8EECBBAB8EECAAA97
:10A12000236AB4EECABAF1EE10FA1A683DDDA368EC
:10A13000DFED820AA16B92ED051AD1ED001A03F64C
:10A140007C0393ED007A27EE0D7A3AEE4B0AC7EEC8
:10A15000200A22F0A3FBDDED017A37EE800A8DEDB7
:10A16000010AB8EEEB0A236AB4EECA0AF1EE10FA5D
:10A170001A6834DDA368A16B92ED061AD1ED001ABE
:10A1800003F67C03D3ED000A20EE8DDADFED6B0AD7
:10A190003AEE400ACDEE200A22F080FBDDED027A95
:10A1A00037EE800A8DED020A20E0B1EE4A0AB4EEE5
:10A1B000C0BAF1EE10FAD4D5A368A16BDFED5F0A47
:10A1C000D1ED001A92ED051A03F67C0393ED007AA7
:10A1D00027EE0D7A30EE4B0AC7EE200AB9E7B1EE52
:10A1E0004AAAB4EECA0AF1EE10FAC3D4236AD3F82D
:10A1F00000C00CF184030FCB12AD85E80F000EAE4A
:10A200000AAD86E80F0085E80F0004AB01AA2946D5
:10A21000604672F04BFD636893F97030022B16D1E3
:10A22000DDED047A39EE279ADDED057A78EEA78A1E
:10A23000DDED067A38EE278A89ED009AC8ED008AAE
:10A2400087ED008A17B0BDEC0C8BBDE8F083F0EE13
:10A25000E99AF0EEEAAAF4EEE9AAF1EE10FA48BFA4
:10A260006D46CDED009ACDED0AAAD5ED007ADFED71
:10A27000340AB0EECCCAF4EECC7AF1EE10FAD8BFC4
:10A2800035468DED0ECA95ED007ADFED2E7A87EE1C
:10A29000270AAD20B7EE001A3CEEC00A22F026F8DD
:10A2A000E369D3ED937A04A820EE270A25F022FA79
:10A2B000F0EEC07A8DED061AB0EEC91A31EE671ACB
:10A2C0008DED040AB0EEC11A39EE000ACDED050A93
:10A2D000B520F1EE410A22F009F8B0EE409A9DED6A
:10A2E000050AB0EEE81AF0EEC07A31EE671A38EEE1
:10A2F000800AB0EEC11AF1EE410ABA2021F0F6FF51
:10A30000F0EE408A9DED060AB0EEC81AF0EEC07A73
:10A3100031EE671A38EE000AB0EEC11ABF20F1EE36
:10A32000410A21F0E3FFB0EE408A85E70000C84211
:10A330009F0CB34548F4FFFFB84B002000007A445F
:10A340000000000000A08C4530B52DED028B836A23
:10A350003E4D044687B0186854F0E2F9E36A186885
:10A36000B0EE408A54F0DCF9636B8DED010A186899
:10A3700054F0D6F905ABB0EE401A03A92046DDED46
:10A38000010A04AAB0EE480AFFF718FE636A1868CB
:10A3900090F8CB10002939D179F0F2F82046FFF778
:10A3A00003FA636A1B6893F8A1100129B0EE408A92
:10A3B0003BD0032942D051B9236A0121186873F0B8
:10A3C00077FB236A186871F00DFF9FED218A236ADD
:10A3D000A268186892F8C02803689DED030ADDEDB5
:10A3E000040A9DED051A92074CBFDB6B9B6B9847E7
:10A3F000236AD5ED540A1868036800215B6EB0EE3D
:10A40000480A984707B0BDEC028B30BD95F9893EEC
:10A41000002B06DBD5F88C3E022B04D190F8A1303E
:10A420000BB90121B8E70221B6E7236A186873F077
:10A430003FFB236A186871F0EBFEC6E7D979002963
:10A44000C5D12046FFF724FDC1E700BFB84B00206F
:10A4500000000000836893ED140AB5EEC00AF1EE27
:10A4600010FA01DCFFF79AB970470000704700004E
:10A47000002070470120704702207047002070477D
:10A4800000207047012070470020704781F00100D4
:10A490007047000001207047012070470048704756
:10A4A000449A0C0800487047509A0C0838B5436924
:10A4B0000446186874F082FD18B96369186875F06D
:10A4C00001FF636920461D68FFF7ECFC6368B3F980
:10A4D0003820B3F9363000EE903A434201EE102AAC
:10A4E00000EE103AB8EEC11AF8EEE00AB8EEC00A73
:10A4F000284674F04FFC636920461D68FFF7D2FCC4
:10A500006368B3F93820B3F9363000EE903A43422D
:10A5100001EE102A00EE103A2846B8EEC11AF8EE05
:10A52000E00AB8EEC00A74F0AFFC012038BD0000AC
:10A5300030B52DED028B0446436985B01D68FFF7E9
:10A54000B1FC6368B3F93820B3F9363000EE903AC5
:10A55000434201EE102A00EE103AB8EEC11AF8EEAE
:10A56000E00AB8EEC00A28465B4D74F013FC2046A2
:10A57000FFF762FBB5F9443108EE103A236A186818
:10A5800003689B6E9847B8EEC88AF0EE400A02AAAC
:10A5900001A9B0EE480A2046FEF70AFF2046FFF761
:10A5A00015FB236B1B68B3F90830F0EE408A00EE10
:10A5B000103A2046B8EEC00AFFF738FB2046B0EE4E
:10A5C000408A8DED030AFFF76DFC6368B3F93630FE
:10A5D00001EE103A434200EE903AB8EEC11AF8EE9E
:10A5E000E00A2B20B0EE480A21F080FE20468DEDD7
:10A5F000030AFFF7A5FA042813D8DFE800F0032FB9
:10A60000252A4B00236A186871F0ECFD236A0021AB
:10A61000186872F097FB63699FED300A186875F04F
:10A620002DFF236ADDED020A18689DED010A03681B
:10A63000B0EE681ADB6A98476369186875F090FF96
:10A6400005B0BDEC028B30BD236A0121186872F0A1
:10A6500079FB236A186871F0DBFDDCE7204D2B786D
:10A6600063B963689FED1F1ADFED1C0A93ED040ABE
:10A67000452021F03BFE284608F0ECFE20469DEDEB
:10A68000030AFFF741FA16488DED030A03A908F003
:10A690001BFFC6E7636A0221186878F071FFB5F9FD
:10A6A0004431114800EE103A02AA01A9B8EEC00ADE
:10A6B0005FF060FA20469DED030AFFF725FA0B488C
:10A6C0008DED030A08F0D0F963699DED030A18685F
:10A6D00074F0E6FBA5E700BFB84B002000000000C7
:10A6E000F87F002000007A44907500202C5700204D
:10A6F0000020704790F8B931002B14BF1B200320B5
:10A7000070470000002070470120704790F89001CA
:10A71000062804D0A0F1090358425841704701208F
:10A7200070470000012070470120704790F8B90180
:10A73000034A044B002814BF10461846704700BF58
:10A74000E89A0C08C5C10D0890F8B901034A044BFA
:10A75000002814BF10461846704700BFF49A0C0832
:10A76000C5C10D0890F890010A3818BF0120704744
:10A7700090F8B9312BB9044BD3F8800A00F00100EE
:10A7800070470020704700BFB84B002090F8903110
:10A7900023B9034B187880F0010070470020704700
:10A7A000DC7F002038B590F89041012C054601D09F
:10A7B000002038BDC368186803681B6998470028E3
:10A7C000F6D1EB681B68204683F8B848F1E7000033
:10A7D000C3681B68002283F8B82801207047000076
:10A7E00070B52DED028B002380F8B931B0F87030D0
:10A7F000012B84B004460D4601D8002946D0636A77
:10A80000254E1B6893F8CB3073BB2448072384F88C
:10A8100090310368022B02D10021FBF773FC9FEDFE
:10A82000208AE368F0EE480A1868B0EE481AF0EEA5
:10A83000481AB0EE480A012577F018F984ED738ABA
:10A8400084ED748A84ED758A84F8B85104F59A70A1
:10A8500025F038FC134803F0B3FD96F88A3E6FF3F9
:10A86000C30386F88A3E11E096F9883E002BCCDAC5
:10A8700004F13C0027F0D8FC05460028C5D120464D
:10A88000FFF70CFB084A02214BF006FD284604B0F6
:10A89000BDEC028B70BD00BFB84B0020EC7E0020E9
:10A8A00000000000847B0020FC9A0C0810B50446D0
:10A8B000064890F8603B012B03D100F65C3025F090
:10A8C00069FC002384F8B93110BD00BFB86B0020CB
:10A8D00010B52DED028B094B0446D3F84409B0EEB8
:10A8E000408A76F05BFC9FED060A28EE008A012084
:10A8F00084ED748ABDEC028B10BD00BFB86B0020E4
:10A900000AD7233C10B52DED028B094B0446D3F832
:10A910004409B0EE408A76F051FC9FED060A28EE1D
:10A92000008A012084ED758ABDEC028B10BD00BF4A
:10A93000B86B00200AD7233C10B52DED028B094BD4
:10A940000446D3F84409B0EE408A76F045FC9FED0A
:10A95000060A28EE008A012084ED738ABDEC028B82
:10A9600010BD00BFB86B00200AD7233CC3681B682A
:10A97000186974F065BD000038B5D0F8943104460C
:10A980000D461BB97FF0F6FFC4F894017FF0F2FF8B
:10A99000D4F89431C01A4FF47A73B0FBF3F0B4F8E2
:10A9A0009231984209D32046FFF778FA2B88044A5F
:10A9B00006214BF071FC012038BD0020FCE700BFF0
:10A9C000189B0C0890F89031052B05D1054BD3F856
:10A9D0004C39D86874F0ACBCC36818680368DB688D
:10A9E000184700BFB86B002008B590F89031052BD0
:10A9F0000BD1094BD3F84C39D868243024F0E8FB4C
:10AA0000BCEEC00A10EE100A08BDC36818680368DF
:10AA10009B689847F4E700BFB86B002090F890312E
:10AA20008B4206D00A2B80F8901102D10148FCF726
:10AA3000EFBF7047B82B002073B501231E4E80F87E
:10AA40007530D6F8943E834205460A4614D1012457
:10AA500085F8B941D6F8940E019203681B689847AF
:10AA6000019A0146154848F089FE96F8893E9A06F3
:10AA70001BD4204602B070BD01910321FFF7E2F81C
:10AA8000019A04460028E2D185F8750049F064FB7C
:10AA90001B220A2149F0BCFA96F8893E9B06E8D5AC
:10AAA000074A137843F0040303E0054A137843F0A0
:10AAB00002031370DDE700BFB84B0020783B002095
:10AAC000BC80002030B585B004460D46014668467E
:10AAD000FFF7EEF9694604F13C0028F057F9C8B9D0
:10AAE00049F03AFB1B220A2149F092FA0D4B93F8E8
:10AAF000893E9B0604D50C4A137843F00403137077
:10AB00002046FFF7CBF9094A04214BF0C5FB002092
:10AB100005B030BD2946204605B0BDE83040FFF7FE
:10AB20008BBF00BFB84B0020BC8000202C9B0C08C2
:10AB300030B585B004460D4601466846FFF7B8F9C2
:10AB4000694604F13C0028F045F9C8B949F004FB16
:10AB50001B220A2149F05CFA0D4B93F8893E9B06B3
:10AB600004D50C4A137843F0040313702046FFF712
:10AB700095F9094A04214BF08FFB002005B030BD48
:10AB80002946204605B0BDE83040FFF755BF00BF5D
:10AB9000B84B0020BC800020689B0C087FB50546A0
:10ABA0000E4605F13C0401466846FFF781F9694607
:10ABB000204628F00FF9C0B92046694628F0E6F88B
:10ABC000044690B949F0C8FA1B220A2149F020FA3C
:10ABD0000D4B93F8893E9B060FD42846FFF75EF98C
:10ABE0000A4A04214BF058FB04E031462846FFF79F
:10ABF00023FF0446204604B070BD054A137843F095
:10AC000004031370E9E700BFB84B0020A09B0C08B9
:10AC1000BC80002030B5044685B00F4808F06CF8C1
:10AC20000546B0B1072384F89031002301930293C5
:10AC30000393E36801A9186876F04AFAE368186894
:10AC4000036801A95B680022984704480021FBF7CC
:10AC500059FA284605B030BDB82B0020EC7E002004
:10AC6000F0B5424FD7F81829D7F814392DED028BDB
:10AC70001343D7F81029134387B005460C460CD16F
:10AC800047F076FD40F275124FF4801107B0BDEC2D
:10AC9000028BBDE8F04047F023BD806977F0B4FC3B
:10ACA0002046B0EE408A10F04BFB03283AD1EB6807
:10ACB00001A9186876F0E8FA064698B3DDED017A46
:10ACC0006368009338EE678A294BDFED2A7A93F99F
:10ACD000883E9FED290A2948002BA8BFB0EE670ADD
:10ACE00038EE008A009BBDEEC88A002118EE102ABB
:10ACF0009342ACBF00930092FBF704FA6B691868AB
:10AD000075F0E0FADDED007A1D48B8EEE70A31464D
:10AD100008F056FE00212846FFF780FE07B0BDEC84
:10AD2000028BF0BD94E80F0002AE86E80F00D7F862
:10AD3000143904936A46D7F818390593022130462E
:10AD400010F00AFB78B949F007FA0222152149F000
:10AD50005FF9DDED037AF8EEE77A77EE887AFDEEBB
:10AD6000E77ACDED007A0026AEE700BFB86B002091
:10AD7000B84B0020000000000000C842EC7E00201C
:10AD8000DC7F002030B52DED028BC36887B0044610
:10AD900018680D4676F06CFA00284BD194F8902193
:10ADA00000230093019302936AB93148039303A9E6
:10ADB0000493059308F034FE28B1039B0093049B91
:10ADC0000193059B029394ED730A9FED2A8AE36831
:10ADD000DDED000A9DED011ADDED021A1868B4EEF2
:10ADE000C80AF1EE10FAAABFDFED237A9FED230A1D
:10ADF00020EE270A76F03AFED4ED747AF4EEC87AA3
:10AE0000F1EE10FA07DBE3689FED1B0A186827EEE6
:10AE1000800A76F0C3F9D4ED757AF4EEC87AF1EED3
:10AE200010FA07DBE3689FED140A186827EE800A22
:10AE300076F0C4F9E3682946186876F03FFD0546C8
:10AE400088B10F4B1B68022B09D0032B03D10D4B8C
:10AE500093F975311BB10A480021FBF773F9012101
:10AE60002046FFF7DBFD284607B0BDEC028B30BD66
:10AE7000DC7F0020000000340000C8420000000019
:10AE8000EC7E0020B84B002010B52DED028BC3687E
:10AE9000DFED348A1B684269D3ED0A0A9FED328ADE
:10AEA00093ED060AF4EEE80A0446F1EE10FA106893
:10AEB000B8BFF0EE480A73F053FDE36862691B689F
:10AEC0001068D3ED0A0A93ED060AF4EEE80AF1EEF3
:10AED00010FAB8BFF0EE480A73F0BAFD636918685B
:10AEE00073F04AFF18B96369186874F085FFE36866
:10AEF00062691B68106893ED080A93ED0C1AD3ED94
:10AF0000070AB0EEC00A73F045FFE36862691B6888
:10AF1000106893ED080A93ED0C1AD3ED070AB0EE12
:10AF2000C00A73F0B1FF6369186874F047F818B984
:10AF30006369186875F0C6F900210C48FBF7E2F860
:10AF40000B4860F0DFFB0B4AB2F88A3E23F48163C2
:10AF5000A2F88A3EBDEC028B20460221BDE81040DB
:10AF6000FFF75CBD0000003400007A43EC7E002057
:10AF700000760020B84B002010B50C4B0446D3F8E7
:10AF80004C0990ED0B0A90F8502000F11C0175F06F
:10AF9000E7FD07480368022B02D00821FBF7B2F84F
:10AFA00020460521BDE81040FFF738BDB86B0020F2
:10AFB000EC7E0020F0B52DED028B4A4DDFED4A8A84
:10AFC000B0EE408A8FB00446D5F84C090E461746BD
:10AFD00075F03CFCF0EEC87AF4EEE87AF1EE10FA87
:10AFE00007D49FED420AD5F84C0928EE000A75F007
:10AFF00093FCD5F84C0990ED0B0AB0EEC00A0FB1E6
:10B00000B1EE400A75F078FC0023D5F84C0907939F
:10B0100002AA07A90893099375F09AFCDFED347A28
:10B020009DED027AB4EEE77AF1EE10FA56DD0222D7
:10B0300007A90AA810F060FC71680191304610F071
:10B040007FF9019902460AA810F050F9E3680AA9AD
:10B05000186876F033FC10B92648FDF7CFF8A069E0
:10B0600077F0D0FA02684368D5F84C09049303A935
:10B070001C30039223F0DEFF05A88DED050ACDED0F
:10B08000060A24F0A5F81C4B1B68022B1BD0D5F830
:10B090004C391948D3ED0A7AF4EEE87AF1EE10FA59
:10B0A000B8BFD3ED047AF4EEC07AF1EE10FA4FF0A7
:10B0B000000110D5DFED117AB4EEE70AF1EE10FAD7
:10B0C00009DDFBF73FF804212046FFF7A7FC0FB08E
:10B0D000BDEC028BF0BDFBF715F8F4E72046FFF757
:10B0E0004BFFF4E7B86B0020000000340000C842BA
:10B0F00000009643B82B0020EC7E00200000FA43AD
:10B1000008B50748D0F8803A9B0704D50121A0F57F
:10B110000050F7F73FF8BDE80840024808F0B2BA1F
:10B12000B84B0020DC7F002030B589B00446FEF724
:10B1300025FA30B10021204609B0BDE83040FEF7C5
:10B1400055BA636A0221186878F01AFAE368186839
:10B1500003685B69984701461048FCF739FF63694B
:10B16000186875F0FDF9236A1D686369186874F042
:10B1700035F805AC20460A498DED020ACDED030AEB
:10B180008DED041AFBF77EF9079B009394E80C0001
:10B1900002A9284671F0EEF809B030BDB82B0020A6
:10B1A000EC7E002038B50446FEF7E8F9054628B1E4
:10B1B00020460021BDE83840FEF718BA636A022134
:10B1C000186878F0DDF929462046BDE83840FEF7DA
:10B1D00053BE00000148002105F0F8BBE07C0020D0
:10B1E00030B5174D9FED170A05F5804389B0044629
:10B1F000D3F84C0975F014FD01462846FCF7E8FE2B
:10B200006369186875F0ACF9236A1D68636918688A
:10B2100073F0E4FF05AC20460B498DED020ACDED3D
:10B22000030A8DED041AFBF72DF9079B009394E8B0
:10B230000C0002A9284671F09DF809B030BD00BF8E
:10B24000B82B002000000000EC7E002030B589B053
:10B250000446FEF793F930B10021204609B0BDE85D
:10B260003040FEF7C3B9636A0221186878F088F9A4
:10B27000E368186803685B69984701461048FCF763
:10B28000A7FE6369186875F06BF9236A1D68636926
:10B29000186873F0A3FF05AC20460A498DED020A39
:10B2A000CDED030A8DED041AFBF7ECF8079B009334
:10B2B00094E80C0002A9284671F05CF809B030BD92
:10B2C000B82B0020EC7E002030B52DED028B83B032
:10B2D0000446FEF753F920B9636A1B6893F8CC3033
:10B2E00043B90021204603B0BDEC028BBDE83040DD
:10B2F000FEF77CB994F89831DA071DD4E3681D682D
:10B300002B6828469B689847D5ED097A94F89831C0
:10B31000B4EEE70AF1EE10FA4CBF0122002262F30C
:10B32000000384F8983107D4204603B0BDEC028BAB
:10B33000BDE83040FFF7F8BE94F898319B0734D44D
:10B34000E368DFED458A1B686269D3ED0A0A9FED69
:10B35000438A93ED060A1068F4EEE80AF1EE10FA5B
:10B36000B8BFF0EE480A73F0FBFAE36862691B6845
:10B370001068D3ED0A0A93ED060AF4EEE80AF1EE3E
:10B3800010FAB8BFF0EE480A73F062FB6369186800
:10B3900073F0F2FC18B96369186874F02DFD94F825
:10B3A000983143F0020384F898312D4BD4F8A02152
:10B3B000D3F810399B1A07EE903AB8EEE78AF1EE0F
:10B3C000047AB0EEC87AB4EEE77AF1EE10FA38D526
:10B3D00094F8983143F0040384F89831204684EDC2
:10B3E000678AFEF735FC6369A26B1B68D2ED001A11
:10B3F00093EDC61AD3ED0E0AB1EE480A21F04EFACB
:10B4000063691B6840F2AA4093EDC31AD3EDC40AE6
:10B4100020F06CFF2046FEF777FB12488DED010A05
:10B4200007F022FB63699DED010A186873F038FD8F
:10B430006369186803B0BDEC028BBDE8304075F05D
:10B440008FB8D4ED677A68EE277AF5EEC07AF1EE20
:10B4500010FAC3D5BCE700BF0000003400007A43F7
:10B46000B86B00202C57002030B52DED028B83B037
:10B470000446FEF783F820B9636A1B6893F8CC3062
:10B4800043B90021204603B0BDEC028BBDE830403B
:10B49000FEF7ACB86369DFED347A1B6894ED710A8E
:10B4A00093EDC31AD3EDC40A20EE270A40F2C4403C
:10B4B00020F01CFF2046FEF727FB236A186803686C
:10B4C0009B6EB0EE408A9847284BB3F9443107EEA3
:10B4D000903AB4F8BC316425F8EEE77A13FB05F333
:10B4E000B4EEE70A07EE103A94F9BE31F1EE10FA25
:10B4F000D8BFF0EE407A13FB05F39FED1D0AF8EE7E
:10B50000C76A07EE103AF4EE407AB8EEC77AF1EE69
:10B5100010FA58BFB0EE670A6846CDED006A8DEDAF
:10B52000017A23F0A7FE236ADDED010A1868B4F85A
:10B53000C03102689DED000A126B13FB05F301EEAA
:10B54000103A0121B8EEC11A90476369B0EE480A7B
:10B55000186873F0A5FC6369186875F001F803B00A
:10B56000BDEC028B30BD00BF0000C842B84B0020CC
:10B5700000007A4430B590F8B83185B00446F3B194
:10B5800068460FF0ADFE404869460AF081F950B1B7
:10B5900004F13C0027F0E6FB002384F8B83104F501
:10B5A0009A7024F08FFD94F890310A2B2DD8DFE8A3
:10B5B00003F0294C50544C582C5C602C640000F56E
:10B5C0009A7024F07FFD04F13C0590B194F840306E
:10B5D000012B0ED194F89031012B0AD1284627F087
:10B5E0002FFA50B12046FEF759FC284A02214AF0B2
:10B5F00053FE284627F052FAD5E72046FEF74EFCC8
:10B60000234AF3E72046FFF77BFD94F844303BB92B
:10B6100094F8463023B994F840309A1E534253416F
:10B6200094F8B9216AB363BB84F8B931194CD4F8E2
:10B63000940E03681B6898472D220146A4F582509A
:10B6400005B0BDE8304048F099B82046FFF76CFDE2
:10B65000DBE72046FFF7A6FDD7E72046FFF7BAFD58
:10B66000D3E72046FFF7BCFDCFE72046FFF7EEFD0E
:10B67000CBE72046FFF728FEC7E72046FFF7F4FE9A
:10B68000C3E705B030BD00BF203E0020EC9B0C0896
:10B69000149C0C08B84B00202DE9F0412DED028BD5
:10B6A000074684B008460E460FF04AFE032880463F
:10B6B0006D4628D1FB68186875F040FC012822D13E
:10B6C0002148294607F0B4F90446B0B17B69DDEDA5
:10B6D000007A1B68F8EEE77A93EDF27A77EEC77A94
:10B6E0004246FDEEE77A17EE901AC829CDED007AB2
:10B6F000B8BFC82130460FF0F9FD204604B0BDECBC
:10B70000028BBDE8F081114B0FCB85E80F0030466E
:10B710000FF016FE014628460FF07AFE0446002878
:10B72000EBD07B69DDED017A1B68B8EEE78AD3EDDB
:10B73000F27A284638EE678A0FF002FEBDEEC88A1C
:10B74000024618EE101AD5E7B82B0020C47400206A
:10B7500010B543699FED126A1B68D3EDF06A93ED53
:10B76000F17AD3EDF27A86B066EE866A27EE067A33
:10B7700067EEC67A68460C46CDED006A8DED017A1B
:10B78000CDED027A23F07AFF03A920468DED030A5E
:10B79000CDED040A8DED051A10F0DEF806B010BDEF
:10B7A0000AD7233C30B5083204461D460FCA84E848
:10B7B0000F00134301BFAB68A360EB68E3606368ED
:10B7C00085B093B920460FF0BBFD03AA0146284679
:10B7D0000FF0C2FD60B10399019120460FF0B0FD5A
:10B7E0000199024620460FF081FD204605B030BD8C
:10B7F000696801912846F1E730B50B6985B00446C8
:10B800000BB94B6953B30023C4F8B43108310FC9E5
:10B810006D4685E80F0029462046FFF73DFF98B9A1
:10B82000124B0122D3F8101928460FF05FFD48F0A3
:10B8300093FC0222152148F0EBFB2046FEF72EFB7D
:10B840000B4A02214AF028FD29462046FFF79AFAC2
:10B8500010B90848FCF7D2FC05B030BD0123C0F890
:10B86000B43105B0BDE83040FFF70EBBB86B002027
:10B87000489C0C08B82B002070B51A4B04460E46A5
:10B880000FCB88B06D4685E80F0020462946FFF7AC
:10B890005FFFE368186875F0EBFC98B1E36818681F
:10B8A00003681B69984768B1E3682946186875F012
:10B8B00051FB38B946F05CFF40F295624FF48011BD
:10B8C00046F00EFF214604A82B463246FFF76AFFDA
:10B8D00004A92046FFF756FA10B90348FCF78EFC7E
:10B8E00008B070BDC4740020B82B002070B5154B93
:10B8F0000C4606460FCB88B06D4685E80F002946FA
:10B900003046FFF725FF2B462246314604A8FFF7B5
:10B9100049FF6288A388122A4FEA132305D1227EA9
:10B92000D20744BF03EB83035B00227A07EE903A11
:10B93000C2F34002B8EE670A04A93046FFF73AFBAB
:10B9400008B070BDC474002038B504460D46FFF73A
:10B9500093FF0023C4F89431AB88A4F8923138BD2A
:10B960007FB50D460446FFF787FF05F108010FC9B3
:10B970006E4686E80F00134306D1234BD3F81429F3
:10B98000D3F818390292039304F5D072012130469E
:10B990000FF0E2FC94F8983170B923F0050343F0FE
:10B9A000050384F898312046FEF778FA174A0621F5
:10B9B0004AF072FC04B070BD23F0070384F898319C
:10B9C0000023C4F89C31E36862691B68106893ED3A
:10B9D000080A93ED0C1AD3ED070AB0EEC00A73F013
:10B9E000D9F9E36862691B68106893ED080A93ED62
:10B9F0000C1AD3ED070AB0EEC00A73F045FA08211D
:10BA00002046FFF70BF8D5E7B86B0020749C0C08B4
:10BA10002DE9F0438DB06D4688461C460746134617
:10BA20000A4601462846DDE91469FFF7BBFE95E8A2
:10BA30000F0084E80F0007A80FF052FCB8F804309C
:10BA4000F3B9B8F80010013105AA89B207F13C003A
:10BA500026F0A2FBA0B1234605AA39462846FFF7E7
:10BA6000A1FE95E80F0086E80F00BDF81630A3F19F
:10BA700052025342534189F800300DB0BDE8F083C3
:10BA800094E80F0086E80F000023F4E770B58B8878
:10BA900092B004460D461646002B44D10DA80FF077
:10BAA0001FFC298801310BAA89B204F13C0026F061
:10BAB00073FB002837D0BDF82E10132903D014D8FB
:10BAC0001039012913D833462A46214603A8FFF727
:10BAD00069FE03AB214607A80BAAFFF763FEE368E4
:10BAE00007A9186875F02AFF01E0522901D012B0A9
:10BAF00070BD07AD03A80FF0F3FB28460FF0F0FB75
:10BB00000DF10B03CDE90053324603AB0BA92046E0
:10BB1000FFF77EFFE0689DF80B3000682A4603A916
:10BB200075F0E2FEE3E70120E1E7000070B5214B8C
:10BB300004460E460FCB88B06D4685E80F002046C0
:10BB40002946FFF705FEE368186875F091FB98B188
:10BB5000E368186803681B69984768B1E368294679
:10BB6000186875F0F7F938B946F002FE40F216622F
:10BB70004FF4801146F0B4FD214604A82B4632460E
:10BB8000FFF710FE04A92046FFF7FCF820B90A4889
:10BB9000FCF734FB08B070BD0023C4F89431B388BF
:10BBA000A4F8923104AA31462046FFF76FFF00281F
:10BBB000F0D1ECE7C4740020B82B0020F0B5324B74
:10BBC00004460E460FCB91B004AD85E80F00204629
:10BBD0002946FFF7BDFDE368186875F049FB98B189
:10BBE000E368186803681B69984768B1E3682946E9
:10BBF000186875F0AFF938B946F0BAFD4FF4DF6256
:10BC00004FF4801146F06CFD0CAF08A80FF068FBF4
:10BC100038460FF065FB0DF10F03CDE900732A469E
:10BC200008AB31462046FFF7F3FEE0689DF80F3081
:10BC300000683A4608A976F09DF920B91348FCF748
:10BC4000DDFA11B0F0BD0023C4F89431B388A4F834
:10BC5000923108AA31462046FFF718FF0028EDD0A0
:10BC60000B4B1B68022B09D0032B03D1094B93F913
:10BC700075311BB106480021FAF764FA012120460C
:10BC8000FEF7CCFEDDE700BFC4740020B82B002017
:10BC9000EC7E0020B84B002037B504460D467EF000
:10BCA00069FEC4F8A801D5ED027AF5EEC07AF1EE8E
:10BCB00010FA17DD9FED137A67EE877AFCEEE77ACC
:10BCC000C4ED697A2046FEF7E9F8D4F8A4214FF4D0
:10BCD0007A73B2FBF3F30C4A062103B0BDE830409F
:10BCE0004AF0DABA5BF032FD0023009395F90D209B
:10BCF00095F90E3095F90C105BF0C4FCC4F8A40162
:10BD0000E0E700BF00007A448C9C0C0810B5B1F944
:10BD10000A30A0F8BC3191F90C3080F8BE31B1F98D
:10BD20000D30A0F8C031B1F90F3007EE903AF8EEBF
:10BD3000E77A0446C0ED717A7EF01CFE0A21C4F851
:10BD4000C8012046BDE81040FEF768BE38B504467D
:10BD50000D467EF00FFEC4F8B001D5ED027A9FEDDE
:10BD6000047A67EE877AFDEEE77AC4ED6B7A38BD28
:10BD700000007A444A7C06480B46003A91F91010BC
:10BD8000D3ED030A93ED020A18BF0122FAF7E4B9D2
:10BD9000EC7E002070B51B4E0446D6F8940E036866
:10BDA00086B01B680D469847042806D16B88102B77
:10BDB0000FD0732B20D000201CE0D6F8940E03681F
:10BDC0001B6898470328F6D194F89031062BF2D1DE
:10BDD000ECE705F108010FC902ACDFED0B0A84E8BE
:10BDE0000F00002309480093B0EE600A1A4621466E
:10BDF00002F028F906B070BD20462946FFF7BAFFC9
:10BE00000120F7E7B84B002000000000847B0020F1
:10BE100038B5D1F8093007EE903AF5EEC07AF1EE78
:10BE200010FA05460C4605DD0B7A022B03D01ED90D
:10BE3000032B0ED038BD154B9FED150AD3F84409DE
:10BE400027EE800A75F0AAF9D4F80930C5F8D03188
:10BE5000F0E70E4B9FED0E0AD3F8440927EE800A57
:10BE600075F0ACF9D4F80930C5F8D431E2E7074BE6
:10BE70009FED070AD3F8440927EE800A75F0ACF964
:10BE8000D4F80930C5F8CC31D4E700BFB86B002036
:10BE90000000C84210B5044C237813B103485FF08A
:10BEA0002BFC207810BD00BFDC7F00200076002036
:10BEB00013B5094B01910446D3F8440903681B6983
:10BEC000984730B10199204602B0BDE81040FEF716
:10BED00053BD02B010BD00BFB86B002090F8983180
:10BEE00013F0010018BFC3F380007047094A0346EE
:10BEF00092F8650168B192F86421043A012A07D8E2
:10BF00005B6A1B6893F8A100431E58425841704772
:10BF100000207047B87B002010B504467EF02AFD53
:10BF2000D4F8B031C01AD4F8AC3123EAE3739842A4
:10BF30004FF0000084BFC4F8AC01012010BD000028
:10BF400010B503680446DB6D9847D4F8AC3123EA9A
:10BF5000E37398424FF000003CBFC4F8AC010120ED
:10BF600010BD000008B504480321FAF7CBF8BDE87E
:10BF700008400148FAF7B2B9EC7E002070B51C4BBE
:10BF80000446D3F8440903681B690E4698470546E2
:10BF900010B90025284670BDD4F894315BB97EF005
:10BFA000E9FCB4F89231C4F8940123B1114A5378F2
:10BFB00043F0010353707EF0DDFCD4F89421B4F813
:10BFC0009231801A4FF47A72B0FBF2F09842E0D3CB
:10BFD00023B9084A537843F0010353702046FDF714
:10BFE0005DFF3388044A06214AF056F9D2E700BFC4
:10BFF000B86B0020BC800020189B0C0810B590F88E
:10C000009031042B0446164B0AD1D3F84409036837
:10C010001B69984718B12046FEF7AEFF002010BDFF
:10C020000A79D3F84C39DFED0F6A93ED0E6A07EE0B
:10C03000902A0A7E920748BF9FED0B7AF8EE677A46
:10C0400048BF67EE877A86EE267AB0EEC77AB4EEFE
:10C05000E77AF1EE10FAACBF01200020DFE700BF65
:10C06000B86B0020DB0FC9400000803B13B5094BC3
:10C0700001910446D3F8440903681B69984730B11D
:10C080000199204602B0BDE81040FEF775BC02B031
:10C0900010BD00BFB86B002010B504467EF06AFCEE
:10C0A000D4F8A831C01AD4F8A43198424FF0000057
:10C0B00084BFC4F8A401012010BD000038B50546B6
:10C0C0000C467EF057FCD5F8C831C01A23894FF4CE
:10C0D0007A725343984294BF0020012038BD00007B
:10C0E000C368186808B190F8B808704710B5012106
:10C0F00004460A4803F0EAFF28B120460321BDE8C0
:10C100001040FEF78BBC46F033FBBDE8104040F218
:10C110006B124FF4801146F0E3BA00BFE07C0020C0
:10C1200090F89031022B04D0032B04D1034803F084
:10C130009DBF012070470020704700BFE07C0020B9
:10C1400038B50C4BD3F8805A90F89031032B044645
:10C1500005F004050AD1084803F0A0FF94F89031D7
:10C1600035B110B9023B5842584138BD0020F5E7BF
:10C170000120FAE7B84B0020E07C002010B50F4A00
:10C18000137843F0800313700D4B93F9882E002A27
:10C19000044609DBFEF73EFD70B920460822BDE8E3
:10C1A00010400921FDF74EBDBDE8104001220E21CF
:10C1B00003F6EC30F5F7F8BE10BD00BFBC800020E0
:10C1C000B84B0020F8B5D0F8B44105465CB1012C5D
:10C1D0001AD046F0CDFA40F643024FF4801146F0F3
:10C1E0007FFA012407E0184BD3F8440903681B6960
:10C1F000984710B900242046F8BD2846FEF744FEB3
:10C200000123C5F8B431F6E7104F97F9883E002BAB
:10C21000F0DA436A1B6893F8A160012EEAD13C3042
:10C2200026F010F804460028E5D1D7F8B83E93F878
:10C23000CB3033B132460D2107F6EC30F5F7B4FEC2
:10C24000D9E73446D7E700BFB86B0020B84B0020D1
:10C2500038B5674BD3F8942E664B9A4204460D4688
:10C2600001D0002096E04B885D2B75D8512B2FD83C
:10C27000103B9AB20F2A49D92046FDF70FFE6B8872
:10C280005D4A04214AF008F87DE0BC3B0D2BF3D851
:10C2900001A252F823F000BF87C3010887C3010839
:10C2A00079C2010879C2010879C2010879C201087E
:10C2B00079C2010887C3010879C2010887C3010850
:10C2C00079C2010879C2010879C2010887C301084F
:10C2D000523B0B2BD0D801A252F823F0D3C3010854
:10C2E00079C201089DC30108B1C3010879C20108E0
:10C2F00079C2010879C2010879C2010879C201082E
:10C3000079C2010879C20108D9C301080F2BB3D83B
:10C3100001A252F823F000BFABC3010863C20108B9
:10C32000B9C30108BFC30108CDC30108B1C30108E7
:10C330009DC3010879C2010879C2010879C20108C8
:10C3400079C2010879C2010879C2010879C20108DD
:10C3500079C20108C5C30108732B46D006D8702BDB
:10C3600040D0722B88D1FFF7EBFD1AE04AF2CF6282
:10C37000934234D080D8C92B0DD8BB2B85D8B23B83
:10C38000012B3FF679AF2046FDF788FD29884EF056
:10C39000A5F8012038BDCF2BF5D06DE72046FFF77B
:10C3A00079FD00283FF45DAFEDE7FFF7E7FDF8E723
:10C3B0002046FFF707FFF4E7FFF720FEF1E7FFF75E
:10C3C00077FDEEE7BDE83840FFF788BDFFF78EFD4B
:10C3D000E7E7FFF74BFEE4E7FFF75EFEE1E7FFF775
:10C3E0006DFEDEE7FFF798FDDBE7FFF7BBFDD8E763
:10C3F000B84B0020D87600209C9C0C0890F8903117
:10C40000032B0BD0062B06D0012B0AD1C36818686A
:10C4100003681B681847044801F006BA034803F094
:10C42000AFBE0020704700BF847B0020E07C00206E
:10C430008B88012B05D00B693BB94B692BB9CB68B5
:10C440001BB904480021FAF761BA024800220831FA
:10C45000FAF77EBAB82B002010B54B885D2B044646
:10C460000A464BD8512B05D8103B99B20F291FD93A
:10C47000002091E0523B0B2BFAD801A151F823F098
:10C48000D3C5010871C401088DC50108A3C5010801
:10C4900071C4010871C4010871C4010871C40108A4
:10C4A00071C4010871C4010871C40108DBC5010829
:10C4B0000F2BDDD801A151F823F000BF9BC5010867
:10C4C000ADC50108B5C50108BDC50108CDC5010848
:10C4D000A3C501088DC5010871C4010871C4010814
:10C4E00071C4010871C4010871C4010871C4010854
:10C4F00071C4010871C40108C5C50108B32B76D009
:10C5000016D8732B70D00ED8702B6AD0722BAFD187
:10C51000D1ED027A9FED3A7A67EE877AFDEEE77AFF
:10C52000C0ED6B7A37E0B22BA2D1FFF771FC32E09D
:10C53000C92B23D8BB2B9BD9BC3B0D2B98D801A171
:10C5400051F823F097C5010897C5010871C4010887
:10C5500071C4010871C4010871C4010871C40108E3
:10C56000F5C5010871C40108F5C5010871C40108C9
:10C5700071C4010871C40108F5C501084AF2CF620F
:10C5800093427FF475AFFFF7C1FB04E002F10801AD
:10C590002046FEF765FB012010BD1146FFF7C6FAE5
:10C5A000F9E711462046FFF727F9F4E71146FFF7B0
:10C5B00063F9F0E71146FFF799F9ECE71146FFF749
:10C5C000C3F9E8E71146FFF7CBF9E4E7FFF78EFD83
:10C5D000E1E71146FFF7F2FADDE71146FFF75CFBF2
:10C5E000D9E7FFF7B3FBD6E7FFF7C4FBD3E7FFF7C5
:10C5F0001FFFD0E7034802F10801F9F74BFECAE735
:10C600000000C842EC7E0020704700007047000028
:10C610007047000090F8280080F00100704700008B
:10C62000024B436040F6050303817047000102049A
:10C6300090F85501704700000F20704700207047A8
:10C640000020704700207047002070470048704766
:10C65000489D0C0800487047549D0C0808B50948CF
:10C6600000F50053D3F8D03AB3F9083000EE103A91
:10C67000B8EEC00AF5F736FFBDE808400248FDF7FE
:10C6800043BA00BFB82B0020B078002010B5144882
:10C690002DED028B1C4600F5005300F58040B3F9E8
:10C6A0004431D0F8380908EE103A036882B09B6E26
:10C6B000CDE900219847B8EEC88AF0EE400ADDE9DE
:10C6C0000021B0EE480A0748FCF772FE0548FDF766
:10C6D0007DFA84ED000A02B0BDEC028B10BD00BFF4
:10C6E000B82B0020B0780020F8B51C4D05F500549B
:10C6F00005F580462846D6F84079F5F7E1FEB4F90D
:10C70000803101EE103AB4F97E3100EE903A4342A6
:10C7100000EE103AB8EEC11AF8EEE00AB8EEC00A20
:10C72000384672F037FB2846D6F84069F5F7C8FE60
:10C73000B4F9803101EE103AB4F97E3100EE903A4E
:10C74000434200EE103A3046B8EEC11ABDE8F84058
:10C75000F8EEE00AB8EEC00A72F096BBB82B0020E3
:10C7600038B5144C04F5804504F57C64D5F83809D7
:10C7700003689B689847692100F19402204646F0BF
:10C78000D5FCD5F838090368DB6898476A2100F1C1
:10C790009402204646F0CAFCD5F8380903681B69A4
:10C7A00098476B2100F194022046BDE8384046F0DE
:10C7B000BDBC00BFB82B0020014806F09DBA00BFE9
:10C7C000B82B00203C307CF09BBC000008B545F045
:10C7D000CFFFBDE8084072224FF4801145F080BFC2
:10C7E00008B545F0C5FFBDE8084066224FF480114A
:10C7F00045F076BF08B545F0BBFFBDE80840802294
:10C800004FF4801145F06CBF73B51E4E0546D6F847
:10C81000940E0268126B9047044670B396F9893EF5
:10C82000002B2DDBD6F8B83E93F8CB402CB396F80E
:10C83000883E03F0A003202B22D1D6F8940E026884
:10C8400012689047052808D0D6F8940E026812683E
:10C850009047A0F110035C425C410B4A02F61C13A6
:10C860000193D6F8E83B0093D2F84039D2F8382942
:10C87000214628467CF0F2FB0446204602B070BDFB
:10C880000024FAE7B84B0020B86B00203C30FFF7DB
:10C89000BBBF000038B5114D04461148F6F7A4FAA5
:10C8A00095F9883E002B14DA236A93F8A120012A17
:10C8B00006D0D5F8940E0021BDE83840FCF796BEAE
:10C8C0000D2105F6EC30F5F76FFB95F9883E002B4E
:10C8D000EFDB2046BDE838407CF0FCBEB84B0020C2
:10C8E000B82B00203C30FFF7D5BF00000120704777
:10C8F00001207047012070470120704711207047C8
:10C9000001207047002070470020704700207047CA
:10C9100000487047989E0C0800487047A09E0C087D
:10C9200038B5436904461D68806975F071FE23F0CF
:10C93000DFFADFED1B0A284672F012F86369A0697E
:10C940001D6875F065FE23F0D3FADFED150A284661
:10C9500072F07EF86369186873F04EFA6369DFED70
:10C96000110A18689FED0E1AB0EE600A72F012FA02
:10C970006369DFED0C0A18689FED091AB0EE600AD2
:10C9800072F082FA6369186872F018FB18B963696B
:10C99000186873F097FC00232364012038BD00BFA2
:10C9A00000803B4400007A4370B52DED028B88B0C7
:10C9B0000446FCF7E3FD70B120460021FCF716FEAB
:10C9C00063699FED310A186808B0BDEC028BBDE8C1
:10C9D000704073F053BD636A0221186876F0D0FD91
:10C9E0002A4B93F8893E5B0603D56369186872F099
:10C9F00037F89FED258A60698DED018A8DED028AF9
:10CA00008DED038A8DED048A03AA01A90068012334
:10CA100072F090F86369186873F004FB236A1D686C
:10CA20002B68DE6C6369186872F0D8FB0122CDEDCB
:10CA3000060A8DED071A05A98DED050A2846B0EE08
:10CA4000480AB0476369B0EE480A186872F028FADD
:10CA50006369186873F084FD236C8BB17DF08AFFE5
:10CA6000E36BC01A236C98420AD309480C220521B3
:10CA7000FCF7FAFE20B906480C220221FCF7F4FE6E
:10CA800008B0BDEC028B70BD00000000B84B002068
:10CA9000B82B002038B504460D467DF06BFFC4E985
:10CAA0000F0538BD072070470120704700207047F0
:10CAB000002070470120704700487047389F0C08DD
:10CAC00000487047409F0C0838B52DED028B0023BD
:10CAD00080F83C30C368DFED338A1B684269D3EDD0
:10CAE0000A0A9FED318A93ED060AF4EEE80A04463D
:10CAF000F1EE10FAB8BFF0EE480A106871F030FF9E
:10CB0000E36862691B681068D3ED0A0A93ED060AB0
:10CB1000F4EEE80AF1EE10FAB8BFF0EE480A71F050
:10CB200097FF636920461D68FDF7BCF96368B3F998
:10CB30003820B3F9363000EE903A434201EE102A25
:10CB400000EE103AB8EEC11AF8EEE00AB8EEC00AEC
:10CB5000284672F01FF9636920461D68FDF7A2F9A7
:10CB60006368B3F93820B3F9363000EE903A4342A7
:10CB700001EE102A00EE103AB8EEC11AF8EEE00A03
:10CB8000B8EEC00A284672F07FF9084BD3F84C097A
:10CB900074F002F806480821F9F7B4FABDEC028BEC
:10CBA000012038BD0000003400007A43B86B00203B
:10CBB000EC7E002030B52DED048BC3689FED898A93
:10CBC0001B684269D3ED0A7ADFED870A93ED060A06
:10CBD000F4EEC87AF1EE10FA0446A8BFF0EE670A48
:10CBE000106889B071F0BCFE636920461D68FDF7CE
:10CBF00059F96368B3F93820B3F9363000EE903A4A
:10CC0000434200EE103A01EE102A2846774DB8EE66
:10CC1000C11AF8EEE00AB8EEC00A72F0BBF8D5F817
:10CC20004C0974F0FBF8A5F5005393F8AD3ED90715
:10CC300047D4D5F84C391A8BD20742D593ED0A9ACE
:10CC4000B4EEC89AF1EE10FAB8BF93ED049AE36A15
:10CC5000186851F065FDD5F84439D3ED067AA36B19
:10CC600020EE270AD3ED007AF0EE498AE0EE278A1B
:10CC7000B0EE490AF5EEC08AF1EE10FAD8BFDFED4A
:10CC80005C8AF0EE680A1FF02DFA28B9D5F84C0935
:10CC9000B0EE680A73F040FE636893F95130272BB9
:10CCA0000FD0A36A186851F03BFDF0EEC07AF4EEA5
:10CCB000C87AF1EE10FAB0EE407A20D5002384F85D
:10CCC0003C30236B1B68B3F9083000EE103A204665
:10CCD000B8EEC00AFCF7AAFF2046FCF715FF204675
:10CCE000B0EE408AFCF74AFC002848D000212046DC
:10CCF00009B0BDEC048BBDE83040FCF777BCD5F83B
:10CD00004C399FED3C0AD3ED0F7AD3ED0B6AA36B40
:10CD100027EE800AF4EEC86AD3ED007AF1EE10FA3D
:10CD200067EE277A10DB9FED341ADFED310A5520CC
:10CD300037EE800A1FF0DAFA012384F83C30D5F888
:10CD40004C0973F0D9FDBCE79FED2C7AF4EEC76A6D
:10CD5000F1EE10FA05D89FED261ADFED290A5920C9
:10CD6000E6E7F0EEE66AF4EEC86AF1EE10FAE3D513
:10CD700094F83C30002B08BFB0EE670ADCE7636A2A
:10CD80000221186876F0FCFB1E4805F06DFEB0EE3F
:10CD9000480AD5F84C0973F043FF01461A48FBF7DF
:10CDA00017F96369186873F0DBFB236A1D68636910
:10CDB000186872F013FA05AC204614498DED020A8A
:10CDC000CDED030A8DED041AF9F75CFB079B009388
:10CDD00094E80C0002A928466FF0CCFA09B0BDEC2B
:10CDE000048B30BD0000003400007A43B86B002093
:10CDF00000000000E02E65420000B442000000B4D4
:10CE00000000B4C22C570020B82B0020EC7E00207C
:10CE100008B5064BD3F84C39D868243022F0D8F93D
:10CE2000FCEEC07A17EE900A08BD00BFB86B002078
:10CE3000024BD3F84C39D86872F07ABAB86B00203C
:10CE40000B20704701207047002070470120704779
:10CE50000020704700487047D89F0C080048704772
:10CE6000E09F0C080120704708B5DFED237AF4EE4F
:10CE7000E70AF1EE10FA2DED028BF0EE408AB0EEEB
:10CE8000608A35DDDFED1D7AF4EEE70AF1EE10FA87
:10CE90002ED5F6EE007A70EEE77ADFED196A9FED97
:10CEA000190ADFED190AF0EEE77A87EEA67A8720F5
:10CEB000B7EE001A30EE470A1FF018FADFED137ACA
:10CEC0009FED131ADFED130A20EE270A8A2020EEC9
:10CED000280A1FF00BFA30EE080ABDEC028BDFEDDA
:10CEE0000A0ABDE808408D20B7EE001A1FF0FEB90F
:10CEF0009FED050AEFE700BFAC1C5A3ED578493FCD
:10CF00008FC2753E9A99993F00000000FAEDEBBA86
:10CF10009A99993E9A9999BE70B57E4EB6F9443168
:10CF20002DED048B00EE903AF8EEE00A82B0044654
:10CF300001AA6946B0EE600AFCF73AFAA06975F0FA
:10CF400067FBE369D0ED008AD3ED946AD3ED977A5D
:10CF500090ED016AA3689FED701ADFED700A27EE6D
:10CF6000E80A68EEA68A03F69403E6EE278A0546E9
:10CF70003B20DFED6B7AB0EEE87AB4EEE77AF1EEC3
:10CF800010FA58BFB0EE677ADFED667AC7EE275A1F
:10CF9000F7EE007A77EEE57A9DED007A67EE877A14
:10CFA00093ED007A67EE877A9FED5F7AA6EE260A08
:10CFB00087EE879A1FF09AF93C209FED571ADFED14
:10CFC000570AB0EE408AB0EE680A1FF08FF9626B24
:10CFD000564B1268DFED567AB2F90820D3ED006A9D
:10CFE0009FED541ADFED540A07EE102AB8EEC77A07
:10CFF000F0EE408A27EE277ADFED507AA6EEA77A88
:10D000004520F4EE007AA7EE678ABAEE000A28EE11
:10D01000000A83ED007A8DED000A1FF067F9DDED5F
:10D02000017A9FED477A474B8DED000AF0EEE77AE3
:10D03000F4EEC77AF1EE10FA51D593ED007ADFEDF8
:10D04000427A77EE277AB2EE007AF4EEC77AF1EE02
:10D0500010FA58BFF0EE477AC3ED007A67EEA87A6F
:10D06000CDED017A636A186890F8CB10002939D1A8
:10D0700076F086FA636A1B6893F8A110012938D00C
:10D0800003293FD039B9236A18686FF05BFE236A21
:10D0900018686FF0A7F8236ADDED010A18689DEDA6
:10D0A000000A0368B0EE491ADB6A9847204695EDFE
:10D0B000028AFCF779FB2046F0EE400AB0EE480AFF
:10D0C000FFF7D2FE236A62681868D2ED020A03688D
:10D0D00001215B6E984702B0BDEC048B70BD00224D
:10D0E0001A60BFE796F9893E002BB4BF01210221E7
:10D0F000BEE7236A18686FF025FE236A18686FF090
:10D1000087F8C8E7D9790029C5D12046FCF7C0FEC9
:10D11000C1E700BFB84B002000000C4400000CC465
:10D120000000FA4400409C45000034423C7F00204F
:10D130000AD7233D00A08C4500A08CC58FC2753F47
:10D1400000000034407F00208FC2F53C0E20704765
:10D150000020704700207047002070470020704773
:10D16000002070470048704778A00C0800487047BE
:10D1700078A00C0870B52DED028B436A1B6893F8FC
:10D18000CB300446FBB9052384F848302046FCF731
:10D190000BFB636A02211868B0EE408A76F0F0F962
:10D1A00094F95030E2696BB3D2F8F8515D4394F8CA
:10D1B0004820052A4FD8DFE812F02B005F008400DA
:10D1C000B100DF001E01836A1B68B3F90830002B31
:10D1D000B8BF5B429BB2B3F57A6FD4D2C36A1B6807
:10D1E000B3F90830002BB8BF5B429BB2B3F57A6F3E
:10D1F000C9D27DF0BFFBE36CC01A40F6C41398425D
:10D20000C1D8C3E794F95150D2F8FC215543CEE779
:10D21000226A94F9511010689FED801A49F6404235
:10D220005343514300EE103A00EE901A0268F8EEB4
:10D23000E00A926BB8EEC00A9047DFED797A41F2CE
:10D2400093139D4238EE278A05DD94F950308BB157
:10D25000012384F84830236A62681868D2ED020A14
:10D260000368B0EE480ABDEC028B5B6EBDE870400F
:10D27000002118470223ECE7226A9FED681A106824
:10D2800049F64042534300EE103A0268B8EEC00A35
:10D29000926BF0EE410A9047DFED627A38EE678AD2
:10D2A00005F50C55B5EEC08AF1EE10FA05F127052B
:10D2B00043F2BA43D8BF9FED598A9D42CBD804238D
:10D2C000C7E7236A9FED551A186894F9513049F65B
:10D2D0004042534300EE903A0268F8EEE00A926B47
:10D2E000B0EE410A9047DFED4F7AE36938EE678A86
:10D2F000D3F8F831B5EEC08AF1EE10FAD8BF9FED41
:10D30000478A002BB8BF5B4242F228329342A2DD2B
:10D3100041F294139D429EDD03239AE7236A9FED19
:10D320003F1A186894F9513049F64042534300EED1
:10D33000903A0268F8EEE00A926BB0EE410A90472C
:10D34000DFED387AE36938EE678AD3F8F831B5EE65
:10D35000C08A03F50C53F1EE10FA03F1270344F2EF
:10D360004E62D8BF9FED2D8A93423FF674AF2E4B8D
:10D370009D42FFF670AFA2E7236A94ED111A186878
:10D38000D4ED100A036894ED0F0A1B6B0021984737
:10D39000DFED237A94F95020E36938EE278A1AB337
:10D3A00093ED7E7AD4ED0F7AB8EEC77A77EEC77A2E
:10D3B0009FED1E7AF0EEE77AF4EEC77AF1EE10FAFE
:10D3C0003FF649AF0D2294F849101948FCF74CFA82
:10D3D000024618B901461648FCF746FA46F0BCFE6C
:10D3E000162146F0F5FD36E793ED7F7AD4ED107AFD
:10D3F000B8EEC77ADAE70D2294F849100C48FCF72A
:10D4000033FA024618B901460948FCF72DFA46F0EE
:10D41000A3FE02220D2146F0FBFD1CE700000000E8
:10D42000CDCC4C3E8FC2753E6DEEFFFF0000FA433F
:10D43000B82B0020F7B5474D0446D5F8940E036885
:10D440005B6B984718B90026304603B0F0BD95F9DC
:10D45000893E002B5EDBA36A1B68B3F90830002B02
:10D46000B8BF5B429BB2B3F57A6FECD2636A1B68BC
:10D4700093F8CB60002EE6D095F9883E002BE2DBD6
:10D48000D5F8940E03681B689847002784F8490074
:10D4900084F848707DF06EFAE36AE064A4F8507096
:10D4A0001B68B3F90830B3F5967F42DD012384F899
:10D4B000513046F051FE152146F08AFDB5F9443150
:10D4C00001EE103AE369B8EEC11A93ED7E0A8DEDD4
:10D4D000011AF1EE410A5320B8EEC00ACDED000A60
:10D4E0001EF004FFE36984ED0F0A93ED7F0A9DEDC2
:10D4F000011ADDED000AB8EEC00A54201EF0F6FE57
:10D50000E36984ED100AD3ED807AF8EEE77AC4ED92
:10D51000117A99E7D5F8940E03681B68984701289B
:10D5200091D0D5F8940E03681B689847002892D1D3
:10D5300089E713F5967F01DAFF23B8E7A36A1B6832
:10D54000B3F90830002BACBF0123FF2384F850301F
:10D55000AFE700BFB84B00200420704701207047A0
:10D5600000207047012070470048704710A10C0848
:10D570000048704718A10C08012909D0232907D0B9
:10D58000042905D0034BD3F8840A00F0010070474A
:10D5900001207047B84B0020C36B23B990F84100BD
:10D5A00080F001007047002070470000034BD3F863
:10D5B000840A80F00400C0F380007047B84B00205C
:10D5C000012380F84230184670470000002380F89D
:10D5D000423001207047000070B52DED028BC3680A
:10D5E0000446186890F9BB3886B0B0EE408A0BB399
:10D5F00090F8BC68F6B173F0A1FC01281AD1274855
:10D6000019213EF027FC07EE900AF8EEE77AF4EED7
:10D61000C87AF1EE10FA0DDD214BB3F9E63A07EEC8
:10D62000903AF8EEE77AF4EEC87AF1EE10FA18DBE9
:10D63000002012E01B4B0FCBFDEEC87A02AD85E84F
:10D640000F0017EE901A012228460DF04FFE01AA96
:10D65000022128460DF080FEE8B906B0BDEC028B31
:10D6600070BDBDEEC88A8DED018A002529460E48A1
:10D67000E563F8F747FD6369186872F023FEDDED96
:10D68000017A0A48B8EEE70A314606F099F984F8BB
:10D6900041500120E1E70026E7E700BFC83800203D
:10D6A000B84B0020C4740020EC7E0020DC7F0020FA
:10D6B00010B52DED048BC2689FED149A1268436972
:10D6C000D2ED0A0ADFED128AF4EEC90AF1EE10FA81
:10D6D0000446B8BFF0EE680A1868B0EE408A71F0F0
:10D6E0003FF9E268636912681868D2ED0A0AF4EE3D
:10D6F000C90AF1EE10FAB8BFF0EE680AB0EE480AB7
:10D7000071F0A6F9BDEC048B012010BD00000034BF
:10D7100000007A4313B5C36842691B68F0EE400A03
:10D7200093ED080A93ED0C1ACDED010A0446B0EE14
:10D73000C00A106871F02EFBE36862691B6810680C
:10D7400093ED080A93ED0C1ADDED010AB0EEC00A64
:10D7500071F09AFB012002B010BD000010B52DED54
:10D76000028BC36842691B68044693ED0C1AD3ED23
:10D77000070A1068B0EE408A71F00CFBE36862693A
:10D780001B68106893ED0C1AD3ED070AB0EE480A37
:10D7900071F07AFBBDEC028B012010BD1FB5C36B8D
:10D7A000022B0BD0032B1DD0012B22D1C36818688C
:10D7B0000368DB6805B05DF804EB1847806974F016
:10D7C00021FF0D4B59689A6802911B68019301A9CA
:10D7D00003921FF0B7FDFDEEC07A17EE900A05B078
:10D7E0005DF804FB4369186805B05DF804EB71F05F
:10D7F0009FBD0020F3E700BF787F0020C36B012BA3
:10D800000AD003DC2BB19FED070A7047023B032BC4
:10D81000F9D84369186802E0C3681B68186971F099
:10D820000FBE00BF0000000030B5C26B012A89B0F6
:10D830000C4604D0022A0AD0002009B030BDC368CB
:10D84000186803681B6809B0BDE8304018470B4BE7
:10D85000586899681B680193094B02901B780391E3
:10D86000002B04AD18BF032201A928460EF044F88E
:10D8700095E80F0084E80F000120DEE7787F0020A4
:10D88000BC7F00207FB5C36B022B0FD0032B23D0AE
:10D89000012B25D1C368186803689B689847BCEEC4
:10D8A000C00A10EE100A07B05DF804FB806974F03E
:10D8B000A9FE0D4B014658689A6804901B680393B3
:10D8C00003A8059221F0B6FB01A88DED010ACDED6C
:10D8D000020A21F07DFCE2E7436918682430F8E78A
:10D8E0009FED020ADDE700BF787F00200000000006
:10D8F00010B52DED028B01239FED1C8AC363C36815
:10D90000044684B018688DED018AF0EE480AB0EE46
:10D91000481AF0EE481AB0EE480A8DED028A8DEDF5
:10D92000038A74F0A3F8E3688DED018A8DED028A15
:10D930008DED038A186801A973F0CAFBE3681868C3
:10D94000036800225B6801A9984730B944F010FFD2
:10D95000BB224FF4801144F0C3FE05480021F8F7C4
:10D96000F1FB04B0BDEC028B10BD00BF0000000055
:10D97000EC7E002030B589B00446FBF7FFFD70B1A6
:10D980001D4805F013FD014618B1636A1B6893F842
:10D99000CC10204609B0BDE83040FBF727BE636AD3
:10D9A0000221186875F0ECFDE368186803685B698C
:10D9B000984701461048FAF70BFB6369186872F044
:10D9C000CFFD236A1D686369186871F007FC05AC18
:10D9D00020460A498DED020ACDED030A8DED041AA9
:10D9E000F8F750FD079B009394E80C0002A9284625
:10D9F0006EF0C0FC09B030BDB82B0020EC7E0020DA
:10DA000010B52DED028BC368DFED298A1B684269D2
:10DA1000D3ED0A0A9FED278A93ED060AF4EEE80A91
:10DA20000446F1EE10FAB8BFF0EE480A106870F044
:10DA300097FFE36862691B681068D3ED0A0A93EDEB
:10DA4000060AF4EEE80AF1EE10FAB8BFF0EE480A62
:10DA500070F0FEFFE36862691B68106893ED080AC6
:10DA600093ED0C1AD3ED070AB0EEC00A71F092F9EB
:10DA7000E36862691B68106893ED080A93ED0C1A5D
:10DA8000D3ED070AB0EEC00A71F0FEF963691868B9
:10DA900072F018FC6369186872F0AEF9064800214C
:10DAA000F8F750FB054B00221A70BDEC028B10BD3D
:10DAB0000000003400007A43EC7E0020BC7F002090
:10DAC0000223C363FFF79CBF0523C363FFF798BF1F
:10DAD0000423C363FFF794BF10B50446FFF7F8FFB4
:10DAE000074A0023936053601360064A93605360B3
:10DAF0001360002384F8403084F84230012010BDC8
:10DB0000847F0020907F00200323C363FFF778BF4A
:10DB100030B50623C363C36842691B6893ED080AE6
:10DB200093ED0C1AD3ED070A044685B01068B0EEE9
:10DB3000C00A71F02FF9E36862691B68106893ED01
:10DB4000080A93ED0C1AD3ED070AB0EEC00A71F083
:10DB50009BF96369186871F031FA18B9636918683C
:10DB600072F0B0FB7CF006FF0C4D0346284601A97D
:10DB700040F8043B236A1B6800245B6F0393019405
:10DB8000029420F09DFE0023EC61AC616C616C623C
:10DB90002C6285F82C3005B030BD00BF487F0020D6
:10DBA000024BD3F8840AC0F3C0007047B84B002082
:10DBB0002DE9F0432DED028B9946C36B274C062BC4
:10DBC00085B080460E461746B0EE408A36D0FFF745
:10DBD0009FFF96E80F00224D85E80F0097E80700A9
:10DBE000103585E8070084F82D900023B9F1000F67
:10DBF00030D084ED0A8A63627CF0BCFE03AB206007
:10DC000002AA01A9304620F08DFF94ED092ADFED2C
:10DC1000157AD4ED0A1A9DED031ADDED020A9DED89
:10DC2000010AD8F83C10104822EE272A3A46F7F7A6
:10DC30000DFA05B0BDEC028BBDE8F083B9F1000F21
:10DC4000C7D194F82D30002BC3D04369186872F007
:10DC500039FBBEE7A36284ED098ACDE7487F002047
:10DC60004C7F00200AD7233CB82B002038B50B4D41
:10DC70000446284605F006FD2B786BB194F8413038
:10DC800053B90123064884F8413059F0DBFEBDE862
:10DC9000384004485DF030BD38BD00BFDC7F002057
:10DCA000004C00200076002070B52DED028B88B06E
:10DCB0000446FBF763FC054680B1294805F076FB76
:10DCC000014618B1636A1B6893F8CC10204608B06F
:10DCD000BDEC028BBDE87040FBF788BC636A9FED2A
:10DCE000218A1868022175F04BFC60698DED018A6C
:10DCF0008DED028A8DED038A8DED048A2B4603AAF1
:10DD000001A9006870F016FF63698DED008A18683C
:10DD10000368B0EE480A2A4669465B68984763691B
:10DD2000186872F07FF96369186872F019FC236A49
:10DD30001D682B68DE6C6369186871F04FFA012268
:10DD40008DED050ACDED060A8DED071AB0EE480AF5
:10DD500005A92846B04708B0BDEC028B70BD00BFD6
:10DD6000B82B002000000000A1B1DFED0F7A20EEFB
:10DD7000270A33B1DFED0D0A0D4801220021F8F723
:10DD8000EBB922B160EEA70A0948F8F763BADFEDF4
:10DD9000070AF9E722B10648B0EE600AF8F796BA2A
:10DDA0000348F8F7CFB900BF0AD7233C00000000B2
:10DDB000EC7E00202DE9F0432DED028B8BB0044664
:10DDC000164606A802220F461D46B0EE408AF0EE27
:10DDD000608A0DF091FD284806A959F0F5FF8046AC
:10DDE00058B946F0B9F90522162146F011F9404616
:10DDF0000BB0BDEC028BBDE8F083E36B032B02D0CC
:10DE00002046FFF781FE9DF858309DF854209DF87C
:10DE10005010F0EE680AB0EE480A2046FFF7A4FF63
:10DE20007CF0A8FD154BD7F800901860144BD7F87C
:10DE300004E0D7F808C0134AC3F80090C3F804E020
:10DE4000C3F808C00023137096E807000E4F0F4E6A
:10DE5000CDF80C9087E8070095E8070086E80700F2
:10DE6000CDE90076E16B0A48CDF810E003AACDF8C1
:10DE700014C0F7F7A9F8BAE7004C0020447F00204F
:10DE8000787F0020BC7F0020847F0020907F0020CE
:10DE9000B82B002010B588B0002405940694079490
:10DEA0009DF82C4002949DF82840CDE9003405AB44
:10DEB000FFF780FF08B010BD2DE9F04F2DED028B6C
:10DEC0008FB091469DF86C709DF868B0002F14BF1C
:10DED0000322022204460AA80D46B0EE408A9A4662
:10DEE000F0EE608A0DF008FD4D480AA959F06CFF6C
:10DEF000064658B946F030F90522162146F088F852
:10DF000030460FB0BDEC028BBDE8F08F454AE36BA5
:10DF1000D2F8842A12F0400F0DF11C082AD0012BF0
:10DF200002D02046FFF7E4FC5B46F0EE680A52465A
:10DF3000B0EE480A49462046FFF716FFE368186826
:10DF400003683A465B682946984700230493059383
:10DF5000069307930893099304AB0093CDF80480CC
:10DF60003B462A46E16B3048F7F72EF8012384F848
:10DF70004030C5E7022B02D02046FFF7A1FD002F5D
:10DF800049D0E3684146186873F07EF940B92268C9
:10DF900003905268012120469047039B1E46AFE73D
:10DFA000224B1B782BB963699DED070A186871F045
:10DFB000B9F852464946DFF874A0DFF884905B4612
:10DFC000F0EE680AB0EE480A2046FFF7CDFE296859
:10DFD0006A68AB68164D8AF80070164F29606A604F
:10DFE000AB600023BB607B603B60C9F80830C9F8B8
:10DFF0000430C9F800307CF0BDFC0F4B6A6829681A
:10E000001860AB680892CDE90079099307919AF8F6
:10E0100000304246A6E763699FED080AC6E700BFE5
:10E02000004C0020B84B0020B82B0020BC7F002003
:10E03000787F0020847F0020447F002000000000C3
:10E04000907F00202DE9F0472DED028B8EB0044625
:10E050006F489DF860A00E469046B0EE408A994603
:10E06000F0EE608A59F0B0FE054658B946F074F8F3
:10E070000522162145F0CCFF28460EB0BDEC028BE0
:10E08000BDE8F087634BD3F8843A590648D5E36B73
:10E09000012B02D02046FFF72BFCE36831461868BD
:10E0A00073F00CFC054618B946F056F80222E0E77A
:10E0B00053464A46F0EE680AB0EE480A414620460A
:10E0C000FFF752FED6ED027AE16B0391F8EEE76AB4
:10E0D000D6ED037ACDED056AB8EEE77AD6ED017A92
:10E0E0008DED067AF8EEE77A3046CDED077A0DF041
:10E0F00027F900220BAB089209920A920B920C921C
:10E100000D920193C21E08AB0093039953425341F1
:10E1100005AA4148F6F758FF012384F84030ABE7E1
:10E120000027E068089709970A97006805AB08AAD6
:10E13000314673F083FB054600289DD0E36B022B2C
:10E1400002D02046FFF7BCFC5346F0EE680A4A4670
:10E15000B0EE480A41462046FFF706FE9DF814300F
:10E16000002B50D0E3680BA9186873F08DF8804637
:10E1700030B9236801215B682046984745467BE714
:10E18000264B1B782BB963699DED0B0A186870F05C
:10E19000C9FF234B089A1A60099ADFF89080DFF8CC
:10E1A00090905A60DFF874A00A9A9A609DF8143033
:10E1B0008AF80030C8F80870C8F80470C8F8007011
:10E1C000C9F80870C9F80470C9F800707CF0D2FB77
:10E1D000D6ED027A134BE16B1860F8EEE76AD6EDE4
:10E1E000037ACDED0B6AB8EEE77AD6ED017A8DEDC4
:10E1F0000C7ACDE90089F8EEE77A9AF80030CDED97
:10E200000D7A0BAA85E763699FED070ABEE700BF99
:10E21000004C0020B84B0020B82B0020BC7F002011
:10E22000787F0020447F002000000000847F0020D1
:10E23000907F00202DE9F0470E4611461A46C36B29
:10E240008AB0052B9DF84C9005460DD0CDED050A02
:10E2500004928DED030A0291FFF736FCDDED050A0D
:10E26000049A9DED030A0299184C194F9DF8483005
:10E27000DFF868A0DFF868802846FFF775FD002307
:10E280000022A36063602360BB607B603B608AF810
:10E29000002096E8070088E807007CF06BFB0D4B38
:10E2A0001860B9F1000F0ED06268A3682168079169
:10E2B00008920993CDE900789AF80030E96B064896
:10E2C00007AAF6F781FE0AB0BDE8F087787F002044
:10E2D000847F0020447F0020B82B0020BC7F0020DA
:10E2E000907F00202DE9F0470F461946C36B8AB096
:10E2F000042B9DF85090054616460BD0CDED050A2F
:10E300008DED040A0391FFF7E3FBDDED050A9DEDBA
:10E31000040A03991A4C9DF84C309DF84820DFF808
:10E3200070A0DFF870802846FFF71EFD0023A36071
:10E330006360236000238AF8003097E8070088E8CC
:10E34000070096E807000F4F87E807007CF012FBF4
:10E350000D4B1860B9F1000F0ED06268A3682168F8
:10E36000079108920993CDE900879AF80030E96B8C
:10E37000064807AAF6F728FE0AB0BDE8F08700BFF6
:10E38000787F0020907F0020447F0020B82B002061
:10E39000BC7F0020847F002010B588B00024059445
:10E3A000069407949DF82C4002949DF82840CDE9EE
:10E3B0000034134605AAFFF795FF08B010BD000012
:10E3C000034B00221A6000225A609A60DA6070479C
:10E3D0009C7F002000487047787F002000487047ED
:10E3E000847F002000487047907F00200A4B9FEDFB
:10E3F0000B7AD3ED007AF4EEC77AF1EE10FAD8BFBB
:10E40000F0EE477A9FED067A67EE877AFCEEE77AC0
:10E4100017EE900A704700BF50560020CDCCCC3D7F
:10E4200000007A4470B58AB00446FBF7A7F870B1D3
:10E43000474804F0BBFF014618B1636A1B6893F8B4
:10E44000CC1020460AB0BDE87040FBF7CFB8414E73
:10E4500033780025039553B1E36803A9186872F077
:10E4600013FF20B93A48F9F7C9FE0AB070BD636AD4
:10E470000221186875F084F8374B9D605D601D605F
:10E48000364B9D605D601D607CF074FA344B1A68F9
:10E49000821A2046FFF7AAFF824207D93148036853
